Component: ARM Compiler 5.06 update 5 (build 528) Tool: armlink [4d35e2]

==============================================================================

Section Cross References

    gpioprocess.o(i.Pin_Trigger_handler_1) refers to printf1.o(i.__0printf$1) for __2printf
    gpioprocess.o(i.Pin_Trigger_handler_1) refers to host.o(i.Action_Key1) for Action_Key1
    gpioprocess.o(i.Pin_Trigger_handler_1) refers to gpioprocess.o(.data) for KeyDebunseTick
    gpioprocess.o(i.Pin_Trigger_handler_2) refers to printf1.o(i.__0printf$1) for __2printf
    gpioprocess.o(i.Pin_Trigger_handler_2) refers to esbprocess.o(.data) for PacketReceiveNGCnt
    gpioprocess.o(i.gpio_init) refers to nrfx_gpiote.o(i.nrfx_gpiote_init) for nrfx_gpiote_init
    gpioprocess.o(i.gpio_init) refers to app_error.o(i.app_error_handler_bare) for app_error_handler_bare
    gpioprocess.o(i.gpio_init) refers to gpioprocess.o(i.nrf_gpio_cfg_output) for nrf_gpio_cfg_output
    gpioprocess.o(i.gpio_init) refers to gpioprocess.o(i.nrf_gpio_pin_clear) for nrf_gpio_pin_clear
    gpioprocess.o(i.gpio_init) refers to nrfx_gpiote.o(i.nrfx_gpiote_in_init) for nrfx_gpiote_in_init
    gpioprocess.o(i.gpio_init) refers to nrfx_gpiote.o(i.nrfx_gpiote_in_event_enable) for nrfx_gpiote_in_event_enable
    gpioprocess.o(i.gpio_init) refers to gpioprocess.o(.constdata) for .constdata
    gpioprocess.o(i.gpio_init) refers to gpioprocess.o(i.Pin_Trigger_handler_1) for Pin_Trigger_handler_1
    gpioprocess.o(i.gpio_init) refers to gpioprocess.o(i.Pin_Trigger_handler_2) for Pin_Trigger_handler_2
    host.o(i.Action_Key1) refers to host.o(i.PacketSend) for PacketSend
    host.o(i.PacketSend) refers to esbprocess.o(i.esb_packet_send) for esb_packet_send
    host.o(i.Timer_1S) refers to gpioprocess.o(.data) for KeyDebunseTick
    host.o(i.Timer_1S) refers to host.o(.data) for TriggerPressedFlag
    host.o(i.esb_packet_received) refers to host.o(i.PacketSend) for PacketSend
    host.o(i.esb_packet_received) refers to printf1.o(i.__0printf$1) for __2printf
    host.o(i.esb_packet_received) refers to esbprocess.o(.data) for PacketReceiveOKCnt
    host.o(i.main) refers to host.o(i.clocks_start) for clocks_start
    host.o(i.main) refers to gpioprocess.o(i.gpio_init) for gpio_init
    host.o(i.main) refers to uartprocess.o(i.UART_Init) for UART_Init
    host.o(i.main) refers to printf1.o(i.__0printf$1) for __2printf
    host.o(i.main) refers to host.o(i.timers_init) for timers_init
    host.o(i.main) refers to esbprocess.o(i.esb_init) for esb_init
    host.o(i.main) refers to app_error.o(i.app_error_handler_bare) for app_error_handler_bare
    host.o(i.main) refers to host.o(i.timers_start) for timers_start
    host.o(i.main) refers to host.o(i.esb_packet_received) for esb_packet_received
    host.o(i.timers_init) refers to app_timer.o(i.app_timer_init) for app_timer_init
    host.o(i.timers_init) refers to app_error.o(i.app_error_handler_bare) for app_error_handler_bare
    host.o(i.timers_init) refers to app_timer.o(i.app_timer_create) for app_timer_create
    host.o(i.timers_init) refers to host.o(i.Timer_1S) for Timer_1S
    host.o(i.timers_init) refers to host.o(.constdata) for Timer_1S_timer_id
    host.o(i.timers_start) refers to app_timer.o(i.app_timer_start) for app_timer_start
    host.o(i.timers_start) refers to app_error.o(i.app_error_handler_bare) for app_error_handler_bare
    host.o(i.timers_start) refers to host.o(.constdata) for Timer_1S_timer_id
    host.o(.constdata) refers to host.o(.bss) for Timer_1S_timer_id_data
    esbprocess.o(i.esb_init) refers to nrf_esb.o(i.nrf_esb_init) for nrf_esb_init
    esbprocess.o(i.esb_init) refers to nrf_esb.o(i.nrf_esb_set_base_address_0) for nrf_esb_set_base_address_0
    esbprocess.o(i.esb_init) refers to nrf_esb.o(i.nrf_esb_set_base_address_1) for nrf_esb_set_base_address_1
    esbprocess.o(i.esb_init) refers to nrf_esb.o(i.nrf_esb_set_prefixes) for nrf_esb_set_prefixes
    esbprocess.o(i.esb_init) refers to nrf_esb.o(i.nrf_esb_set_rf_channel) for nrf_esb_set_rf_channel
    esbprocess.o(i.esb_init) refers to nrf_esb.o(i.nrf_esb_start_rx) for nrf_esb_start_rx
    esbprocess.o(i.esb_init) refers to esbprocess.o(.data) for nrf_esb_config
    esbprocess.o(i.esb_init) refers to esbprocess.o(i.nrf_esb_event_handler) for nrf_esb_event_handler
    esbprocess.o(i.esb_packet_send) refers to nrf_esb.o(i.nrf_esb_stop_rx) for nrf_esb_stop_rx
    esbprocess.o(i.esb_packet_send) refers to nrf_esb.o(i.nrf_esb_disable) for nrf_esb_disable
    esbprocess.o(i.esb_packet_send) refers to nrf_esb.o(i.nrf_esb_init) for nrf_esb_init
    esbprocess.o(i.esb_packet_send) refers to nrf_esb.o(i.nrf_esb_start_tx) for nrf_esb_start_tx
    esbprocess.o(i.esb_packet_send) refers to memcpya.o(.text) for __aeabi_memcpy
    esbprocess.o(i.esb_packet_send) refers to nrf_esb.o(i.nrf_esb_write_payload) for nrf_esb_write_payload
    esbprocess.o(i.esb_packet_send) refers to esbprocess.o(.data) for radio_started
    esbprocess.o(i.esb_packet_send) refers to esbprocess.o(.bss) for tx_payload
    esbprocess.o(i.nrf_esb_event_handler) refers to nrf_esb.o(i.nrf_esb_disable) for nrf_esb_disable
    esbprocess.o(i.nrf_esb_event_handler) refers to nrf_esb.o(i.nrf_esb_init) for nrf_esb_init
    esbprocess.o(i.nrf_esb_event_handler) refers to nrf_esb.o(i.nrf_esb_start_rx) for nrf_esb_start_rx
    esbprocess.o(i.nrf_esb_event_handler) refers to nrf_esb.o(i.nrf_esb_read_rx_payload) for nrf_esb_read_rx_payload
    esbprocess.o(i.nrf_esb_event_handler) refers to esbprocess.o(.data) for radio_tx_busy
    esbprocess.o(i.nrf_esb_event_handler) refers to esbprocess.o(.bss) for rx_payload
    boards.o(i.bsp_board_button_idx_to_pin) refers to boards.o(.constdata) for m_board_btn_list
    boards.o(i.bsp_board_button_state_get) refers to boards.o(.constdata) for m_board_btn_list
    boards.o(i.bsp_board_buttons_init) refers to boards.o(i.nrf_gpio_cfg) for nrf_gpio_cfg
    boards.o(i.bsp_board_buttons_init) refers to boards.o(.constdata) for m_board_btn_list
    boards.o(i.bsp_board_init) refers to boards.o(i.bsp_board_leds_init) for bsp_board_leds_init
    boards.o(i.bsp_board_init) refers to boards.o(i.bsp_board_buttons_init) for bsp_board_buttons_init
    boards.o(i.bsp_board_led_idx_to_pin) refers to boards.o(.constdata) for m_board_led_list
    boards.o(i.bsp_board_led_invert) refers to boards.o(.constdata) for m_board_led_list
    boards.o(i.bsp_board_led_off) refers to boards.o(i.nrf_gpio_pin_write) for nrf_gpio_pin_write
    boards.o(i.bsp_board_led_off) refers to boards.o(.constdata) for m_board_led_list
    boards.o(i.bsp_board_led_on) refers to boards.o(i.nrf_gpio_pin_write) for nrf_gpio_pin_write
    boards.o(i.bsp_board_led_on) refers to boards.o(.constdata) for m_board_led_list
    boards.o(i.bsp_board_led_state_get) refers to boards.o(.constdata) for m_board_led_list
    boards.o(i.bsp_board_leds_init) refers to boards.o(i.nrf_gpio_cfg) for nrf_gpio_cfg
    boards.o(i.bsp_board_leds_init) refers to boards.o(i.bsp_board_leds_off) for bsp_board_leds_off
    boards.o(i.bsp_board_leds_init) refers to boards.o(.constdata) for m_board_led_list
    boards.o(i.bsp_board_leds_off) refers to boards.o(i.bsp_board_led_off) for bsp_board_led_off
    boards.o(i.bsp_board_leds_on) refers to boards.o(i.bsp_board_led_on) for bsp_board_led_on
    boards.o(i.bsp_board_pin_to_button_idx) refers to boards.o(.constdata) for m_board_btn_list
    boards.o(i.bsp_board_pin_to_led_idx) refers to boards.o(.constdata) for m_board_led_list
    nrf_drv_uart.o(i.nrf_drv_uart_init) refers to memcpya.o(.text) for __aeabi_memcpy4
    nrf_drv_uart.o(i.nrf_drv_uart_init) refers to nrfx_uarte.o(i.nrfx_uarte_init) for nrfx_uarte_init
    nrf_drv_uart.o(i.nrf_drv_uart_init) refers to nrfx_uart.o(i.nrfx_uart_init) for nrfx_uart_init
    nrf_drv_uart.o(i.nrf_drv_uart_init) refers to nrf_drv_uart.o(.data) for m_handlers
    nrf_drv_uart.o(i.nrf_drv_uart_init) refers to nrf_drv_uart.o(i.uarte_evt_handler) for uarte_evt_handler
    nrf_drv_uart.o(i.nrf_drv_uart_init) refers to nrf_drv_uart.o(i.uart_evt_handler) for uart_evt_handler
    nrf_drv_uart.o(i.uart_evt_handler) refers to nrf_drv_uart.o(.data) for m_contexts
    nrf_drv_uart.o(i.uarte_evt_handler) refers to nrf_drv_uart.o(.data) for m_contexts
    nrfx_prs.o(i.UARTE0_UART0_IRQHandler) refers to nrfx_prs.o(.data) for m_prs_box_4
    nrfx_prs.o(i.nrfx_prs_acquire) refers to nrfx_prs.o(i.prs_box_get) for prs_box_get
    nrfx_prs.o(i.nrfx_prs_acquire) refers to app_util_platform.o(i.app_util_critical_region_enter) for app_util_critical_region_enter
    nrfx_prs.o(i.nrfx_prs_acquire) refers to app_util_platform.o(i.app_util_critical_region_exit) for app_util_critical_region_exit
    nrfx_prs.o(i.nrfx_prs_release) refers to nrfx_prs.o(i.prs_box_get) for prs_box_get
    nrfx_prs.o(i.prs_box_get) refers to nrfx_prs.o(.data) for m_prs_box_4
    nrfx_uart.o(i.apply_config) refers to nrfx_uart.o(i.nrf_gpio_pin_set) for nrf_gpio_pin_set
    nrfx_uart.o(i.apply_config) refers to nrfx_uart.o(i.nrf_gpio_cfg_output) for nrf_gpio_cfg_output
    nrfx_uart.o(i.apply_config) refers to nrfx_uart.o(i.nrf_gpio_cfg_input) for nrf_gpio_cfg_input
    nrfx_uart.o(i.apply_config) refers to nrfx_uart.o(i.nrf_uart_txrx_pins_set) for nrf_uart_txrx_pins_set
    nrfx_uart.o(i.apply_config) refers to nrfx_uart.o(i.nrf_uart_hwfc_pins_set) for nrf_uart_hwfc_pins_set
    nrfx_uart.o(i.interrupts_disable) refers to nrfx_uart.o(i.nrf_uart_int_disable) for nrf_uart_int_disable
    nrfx_uart.o(i.interrupts_disable) refers to nrfx_uart.o(i.nrfx_get_irq_number) for nrfx_get_irq_number
    nrfx_uart.o(i.interrupts_enable) refers to nrfx_uart.o(i.nrf_uart_event_clear) for nrf_uart_event_clear
    nrfx_uart.o(i.interrupts_enable) refers to nrfx_uart.o(i.nrf_uart_int_enable) for nrf_uart_int_enable
    nrfx_uart.o(i.interrupts_enable) refers to nrfx_uart.o(i.nrfx_get_irq_number) for nrfx_get_irq_number
    nrfx_uart.o(i.nrf_gpio_cfg_default) refers to nrfx_uart.o(i.nrf_gpio_cfg) for nrf_gpio_cfg
    nrfx_uart.o(i.nrf_gpio_cfg_input) refers to nrfx_uart.o(i.nrf_gpio_cfg) for nrf_gpio_cfg
    nrfx_uart.o(i.nrf_gpio_cfg_output) refers to nrfx_uart.o(i.nrf_gpio_cfg) for nrf_gpio_cfg
    nrfx_uart.o(i.nrfx_uart_0_irq_handler) refers to nrfx_uart.o(i.uart_irq_handler) for uart_irq_handler
    nrfx_uart.o(i.nrfx_uart_0_irq_handler) refers to nrfx_uart.o(.bss) for m_cb
    nrfx_uart.o(i.nrfx_uart_errorsrc_get) refers to nrfx_uart.o(i.nrf_uart_event_clear) for nrf_uart_event_clear
    nrfx_uart.o(i.nrfx_uart_errorsrc_get) refers to nrfx_uart.o(i.nrf_uart_errorsrc_get_and_clear) for nrf_uart_errorsrc_get_and_clear
    nrfx_uart.o(i.nrfx_uart_init) refers to nrfx_prs.o(i.nrfx_prs_acquire) for nrfx_prs_acquire
    nrfx_uart.o(i.nrfx_uart_init) refers to nrfx_uart.o(i.apply_config) for apply_config
    nrfx_uart.o(i.nrfx_uart_init) refers to nrfx_uart.o(i.interrupts_enable) for interrupts_enable
    nrfx_uart.o(i.nrfx_uart_init) refers to nrfx_uart.o(.bss) for m_cb
    nrfx_uart.o(i.nrfx_uart_init) refers to nrfx_uart.o(.constdata) for irq_handlers
    nrfx_uart.o(i.nrfx_uart_rx) refers to nrfx_uart.o(i.nrf_uart_int_disable) for nrf_uart_int_disable
    nrfx_uart.o(i.nrfx_uart_rx) refers to nrfx_uart.o(i.nrf_uart_int_enable) for nrf_uart_int_enable
    nrfx_uart.o(i.nrfx_uart_rx) refers to nrfx_uart.o(i.rx_enable) for rx_enable
    nrfx_uart.o(i.nrfx_uart_rx) refers to nrfx_uart.o(i.nrf_uart_event_clear) for nrf_uart_event_clear
    nrfx_uart.o(i.nrfx_uart_rx) refers to nrfx_uart.o(i.nrf_uart_event_check) for nrf_uart_event_check
    nrfx_uart.o(i.nrfx_uart_rx) refers to nrfx_uart.o(i.rx_byte) for rx_byte
    nrfx_uart.o(i.nrfx_uart_rx) refers to nrfx_uart.o(i.nrf_uart_task_trigger) for nrf_uart_task_trigger
    nrfx_uart.o(i.nrfx_uart_rx) refers to nrfx_uart.o(.bss) for m_cb
    nrfx_uart.o(i.nrfx_uart_rx_abort) refers to nrfx_uart.o(i.nrf_uart_int_disable) for nrf_uart_int_disable
    nrfx_uart.o(i.nrfx_uart_rx_abort) refers to nrfx_uart.o(i.nrf_uart_task_trigger) for nrf_uart_task_trigger
    nrfx_uart.o(i.nrfx_uart_rx_disable) refers to nrfx_uart.o(i.nrf_uart_task_trigger) for nrf_uart_task_trigger
    nrfx_uart.o(i.nrfx_uart_rx_disable) refers to nrfx_uart.o(.bss) for m_cb
    nrfx_uart.o(i.nrfx_uart_rx_enable) refers to nrfx_uart.o(i.rx_enable) for rx_enable
    nrfx_uart.o(i.nrfx_uart_rx_enable) refers to nrfx_uart.o(.bss) for m_cb
    nrfx_uart.o(i.nrfx_uart_rx_ready) refers to nrfx_uart.o(i.nrf_uart_event_check) for nrf_uart_event_check
    nrfx_uart.o(i.nrfx_uart_tx) refers to nrfx_uart.o(i.nrfx_uart_tx_in_progress) for nrfx_uart_tx_in_progress
    nrfx_uart.o(i.nrfx_uart_tx) refers to nrfx_uart.o(i.nrf_uart_event_clear) for nrf_uart_event_clear
    nrfx_uart.o(i.nrfx_uart_tx) refers to nrfx_uart.o(i.nrf_uart_task_trigger) for nrf_uart_task_trigger
    nrfx_uart.o(i.nrfx_uart_tx) refers to nrfx_uart.o(i.tx_byte) for tx_byte
    nrfx_uart.o(i.nrfx_uart_tx) refers to nrfx_uart.o(i.tx_blocking) for tx_blocking
    nrfx_uart.o(i.nrfx_uart_tx) refers to nrfx_uart.o(i.nrf_uart_event_check) for nrf_uart_event_check
    nrfx_uart.o(i.nrfx_uart_tx) refers to nrfx_uart.o(.bss) for m_cb
    nrfx_uart.o(i.nrfx_uart_tx_abort) refers to nrfx_uart.o(i.nrf_uart_task_trigger) for nrf_uart_task_trigger
    nrfx_uart.o(i.nrfx_uart_tx_abort) refers to nrfx_uart.o(i.tx_done_event) for tx_done_event
    nrfx_uart.o(i.nrfx_uart_tx_abort) refers to nrfx_uart.o(.bss) for m_cb
    nrfx_uart.o(i.nrfx_uart_tx_in_progress) refers to nrfx_uart.o(.bss) for m_cb
    nrfx_uart.o(i.nrfx_uart_uninit) refers to nrfx_uart.o(i.interrupts_disable) for interrupts_disable
    nrfx_uart.o(i.nrfx_uart_uninit) refers to nrfx_uart.o(i.pins_to_default) for pins_to_default
    nrfx_uart.o(i.nrfx_uart_uninit) refers to nrfx_prs.o(i.nrfx_prs_release) for nrfx_prs_release
    nrfx_uart.o(i.nrfx_uart_uninit) refers to nrfx_uart.o(.bss) for m_cb
    nrfx_uart.o(i.pins_to_default) refers to nrfx_uart.o(i.nrf_uart_txrx_pins_set) for nrf_uart_txrx_pins_set
    nrfx_uart.o(i.pins_to_default) refers to nrfx_uart.o(i.nrf_uart_hwfc_pins_set) for nrf_uart_hwfc_pins_set
    nrfx_uart.o(i.pins_to_default) refers to nrfx_uart.o(i.nrf_gpio_cfg_default) for nrf_gpio_cfg_default
    nrfx_uart.o(i.rx_byte) refers to nrfx_uart.o(i.nrf_uart_event_clear) for nrf_uart_event_clear
    nrfx_uart.o(i.rx_enable) refers to nrfx_uart.o(i.nrf_uart_event_clear) for nrf_uart_event_clear
    nrfx_uart.o(i.rx_enable) refers to nrfx_uart.o(i.nrf_uart_task_trigger) for nrf_uart_task_trigger
    nrfx_uart.o(i.tx_blocking) refers to nrfx_uart.o(i.nrf_uart_event_check) for nrf_uart_event_check
    nrfx_uart.o(i.tx_blocking) refers to nrfx_uart.o(i.tx_byte) for tx_byte
    nrfx_uart.o(i.tx_byte) refers to nrfx_uart.o(i.nrf_uart_event_clear) for nrf_uart_event_clear
    nrfx_uart.o(i.uart_irq_handler) refers to nrfx_uart.o(i.nrf_uart_int_enable_check) for nrf_uart_int_enable_check
    nrfx_uart.o(i.uart_irq_handler) refers to nrfx_uart.o(i.nrf_uart_event_check) for nrf_uart_event_check
    nrfx_uart.o(i.uart_irq_handler) refers to nrfx_uart.o(i.nrf_uart_event_clear) for nrf_uart_event_clear
    nrfx_uart.o(i.uart_irq_handler) refers to nrfx_uart.o(i.nrf_uart_int_disable) for nrf_uart_int_disable
    nrfx_uart.o(i.uart_irq_handler) refers to nrfx_uart.o(i.nrf_uart_task_trigger) for nrf_uart_task_trigger
    nrfx_uart.o(i.uart_irq_handler) refers to nrfx_uart.o(i.nrf_uart_errorsrc_get_and_clear) for nrf_uart_errorsrc_get_and_clear
    nrfx_uart.o(i.uart_irq_handler) refers to nrfx_uart.o(i.rx_byte) for rx_byte
    nrfx_uart.o(i.uart_irq_handler) refers to nrfx_uart.o(i.rx_done_event) for rx_done_event
    nrfx_uart.o(i.uart_irq_handler) refers to nrfx_uart.o(i.tx_byte) for tx_byte
    nrfx_uart.o(i.uart_irq_handler) refers to nrfx_uart.o(i.tx_done_event) for tx_done_event
    nrfx_uart.o(.constdata) refers to nrfx_uart.o(i.nrfx_uart_0_irq_handler) for nrfx_uart_0_irq_handler
    nrfx_uarte.o(i.apply_config) refers to nrfx_uarte.o(i.nrf_gpio_pin_set) for nrf_gpio_pin_set
    nrfx_uarte.o(i.apply_config) refers to nrfx_uarte.o(i.nrf_gpio_cfg_output) for nrf_gpio_cfg_output
    nrfx_uarte.o(i.apply_config) refers to nrfx_uarte.o(i.nrf_gpio_cfg_input) for nrf_gpio_cfg_input
    nrfx_uarte.o(i.apply_config) refers to nrfx_uarte.o(i.nrf_uarte_txrx_pins_set) for nrf_uarte_txrx_pins_set
    nrfx_uarte.o(i.apply_config) refers to nrfx_uarte.o(i.nrf_uarte_hwfc_pins_set) for nrf_uarte_hwfc_pins_set
    nrfx_uarte.o(i.interrupts_disable) refers to nrfx_uarte.o(i.nrf_uarte_int_disable) for nrf_uarte_int_disable
    nrfx_uarte.o(i.interrupts_disable) refers to nrfx_uarte.o(i.nrfx_get_irq_number) for nrfx_get_irq_number
    nrfx_uarte.o(i.interrupts_enable) refers to nrfx_uarte.o(i.nrf_uarte_event_clear) for nrf_uarte_event_clear
    nrfx_uarte.o(i.interrupts_enable) refers to nrfx_uarte.o(i.nrf_uarte_int_enable) for nrf_uarte_int_enable
    nrfx_uarte.o(i.interrupts_enable) refers to nrfx_uarte.o(i.nrfx_get_irq_number) for nrfx_get_irq_number
    nrfx_uarte.o(i.nrf_gpio_cfg_default) refers to nrfx_uarte.o(i.nrf_gpio_cfg) for nrf_gpio_cfg
    nrfx_uarte.o(i.nrf_gpio_cfg_input) refers to nrfx_uarte.o(i.nrf_gpio_cfg) for nrf_gpio_cfg
    nrfx_uarte.o(i.nrf_gpio_cfg_output) refers to nrfx_uarte.o(i.nrf_gpio_cfg) for nrf_gpio_cfg
    nrfx_uarte.o(i.nrfx_uarte_0_irq_handler) refers to nrfx_uarte.o(i.uarte_irq_handler) for uarte_irq_handler
    nrfx_uarte.o(i.nrfx_uarte_0_irq_handler) refers to nrfx_uarte.o(.bss) for m_cb
    nrfx_uarte.o(i.nrfx_uarte_errorsrc_get) refers to nrfx_uarte.o(i.nrf_uarte_event_clear) for nrf_uarte_event_clear
    nrfx_uarte.o(i.nrfx_uarte_errorsrc_get) refers to nrfx_uarte.o(i.nrf_uarte_errorsrc_get_and_clear) for nrf_uarte_errorsrc_get_and_clear
    nrfx_uarte.o(i.nrfx_uarte_init) refers to nrfx_prs.o(i.nrfx_prs_acquire) for nrfx_prs_acquire
    nrfx_uarte.o(i.nrfx_uarte_init) refers to nrfx_uarte.o(i.apply_config) for apply_config
    nrfx_uarte.o(i.nrfx_uarte_init) refers to nrfx_uarte.o(i.interrupts_enable) for interrupts_enable
    nrfx_uarte.o(i.nrfx_uarte_init) refers to nrfx_uarte.o(.bss) for m_cb
    nrfx_uarte.o(i.nrfx_uarte_init) refers to nrfx_uarte.o(.constdata) for irq_handlers
    nrfx_uarte.o(i.nrfx_uarte_rx) refers to nrfx_uarte.o(i.nrfx_is_in_ram) for nrfx_is_in_ram
    nrfx_uarte.o(i.nrfx_uarte_rx) refers to nrfx_uarte.o(i.nrf_uarte_int_disable) for nrf_uarte_int_disable
    nrfx_uarte.o(i.nrfx_uarte_rx) refers to nrfx_uarte.o(i.nrf_uarte_int_enable) for nrf_uarte_int_enable
    nrfx_uarte.o(i.nrfx_uarte_rx) refers to nrfx_uarte.o(i.nrf_uarte_event_clear) for nrf_uarte_event_clear
    nrfx_uarte.o(i.nrfx_uarte_rx) refers to nrfx_uarte.o(i.nrf_uarte_task_trigger) for nrf_uarte_task_trigger
    nrfx_uarte.o(i.nrfx_uarte_rx) refers to nrfx_uarte.o(i.nrf_uarte_event_check) for nrf_uarte_event_check
    nrfx_uarte.o(i.nrfx_uarte_rx) refers to nrfx_uarte.o(.bss) for m_cb
    nrfx_uarte.o(i.nrfx_uarte_rx_abort) refers to nrfx_uarte.o(i.nrf_uarte_shorts_disable) for nrf_uarte_shorts_disable
    nrfx_uarte.o(i.nrfx_uarte_rx_abort) refers to nrfx_uarte.o(i.nrf_uarte_task_trigger) for nrf_uarte_task_trigger
    nrfx_uarte.o(i.nrfx_uarte_rx_abort) refers to nrfx_uarte.o(.bss) for m_cb
    nrfx_uarte.o(i.nrfx_uarte_rx_ready) refers to nrfx_uarte.o(i.nrf_uarte_event_check) for nrf_uarte_event_check
    nrfx_uarte.o(i.nrfx_uarte_tx) refers to nrfx_uarte.o(i.nrfx_is_in_ram) for nrfx_is_in_ram
    nrfx_uarte.o(i.nrfx_uarte_tx) refers to nrfx_uarte.o(i.nrfx_uarte_tx_in_progress) for nrfx_uarte_tx_in_progress
    nrfx_uarte.o(i.nrfx_uarte_tx) refers to nrfx_uarte.o(i.nrf_uarte_event_clear) for nrf_uarte_event_clear
    nrfx_uarte.o(i.nrfx_uarte_tx) refers to nrfx_uarte.o(i.nrf_uarte_task_trigger) for nrf_uarte_task_trigger
    nrfx_uarte.o(i.nrfx_uarte_tx) refers to nrfx_uarte.o(i.nrf_uarte_event_check) for nrf_uarte_event_check
    nrfx_uarte.o(i.nrfx_uarte_tx) refers to nrfx_uarte.o(.bss) for m_cb
    nrfx_uarte.o(i.nrfx_uarte_tx_abort) refers to nrfx_uarte.o(i.nrf_uarte_event_clear) for nrf_uarte_event_clear
    nrfx_uarte.o(i.nrfx_uarte_tx_abort) refers to nrfx_uarte.o(i.nrf_uarte_task_trigger) for nrf_uarte_task_trigger
    nrfx_uarte.o(i.nrfx_uarte_tx_abort) refers to nrfx_uarte.o(i.nrf_uarte_event_check) for nrf_uarte_event_check
    nrfx_uarte.o(i.nrfx_uarte_tx_abort) refers to nrfx_uarte.o(.bss) for m_cb
    nrfx_uarte.o(i.nrfx_uarte_tx_in_progress) refers to nrfx_uarte.o(.bss) for m_cb
    nrfx_uarte.o(i.nrfx_uarte_uninit) refers to nrfx_uarte.o(i.interrupts_disable) for interrupts_disable
    nrfx_uarte.o(i.nrfx_uarte_uninit) refers to nrfx_uarte.o(i.pins_to_default) for pins_to_default
    nrfx_uarte.o(i.nrfx_uarte_uninit) refers to nrfx_prs.o(i.nrfx_prs_release) for nrfx_prs_release
    nrfx_uarte.o(i.nrfx_uarte_uninit) refers to nrfx_uarte.o(.bss) for m_cb
    nrfx_uarte.o(i.pins_to_default) refers to nrfx_uarte.o(i.nrf_uarte_txrx_pins_set) for nrf_uarte_txrx_pins_set
    nrfx_uarte.o(i.pins_to_default) refers to nrfx_uarte.o(i.nrf_uarte_hwfc_pins_set) for nrf_uarte_hwfc_pins_set
    nrfx_uarte.o(i.pins_to_default) refers to nrfx_uarte.o(i.nrf_gpio_cfg_default) for nrf_gpio_cfg_default
    nrfx_uarte.o(i.uarte_irq_handler) refers to nrfx_uarte.o(i.nrf_uarte_event_check) for nrf_uarte_event_check
    nrfx_uarte.o(i.uarte_irq_handler) refers to nrfx_uarte.o(i.nrf_uarte_event_clear) for nrf_uarte_event_clear
    nrfx_uarte.o(i.uarte_irq_handler) refers to nrfx_uarte.o(i.nrf_uarte_errorsrc_get_and_clear) for nrf_uarte_errorsrc_get_and_clear
    nrfx_uarte.o(i.uarte_irq_handler) refers to nrfx_uarte.o(i.nrf_uarte_rx_amount_get) for nrf_uarte_rx_amount_get
    nrfx_uarte.o(i.uarte_irq_handler) refers to nrfx_uarte.o(i.nrf_uarte_shorts_disable) for nrf_uarte_shorts_disable
    nrfx_uarte.o(i.uarte_irq_handler) refers to nrfx_uarte.o(i.rx_done_event) for rx_done_event
    nrfx_uarte.o(i.uarte_irq_handler) refers to nrfx_uarte.o(i.tx_done_event) for tx_done_event
    nrfx_uarte.o(.constdata) refers to nrfx_uarte.o(i.nrfx_uarte_0_irq_handler) for nrfx_uarte_0_irq_handler
    nrfx_gpiote.o(i.GPIOTE_IRQHandler) refers to nrfx_gpiote.o(i.nrf_gpiote_event_is_set) for nrf_gpiote_event_is_set
    nrfx_gpiote.o(i.GPIOTE_IRQHandler) refers to nrfx_gpiote.o(i.nrf_gpiote_event_clear) for nrf_gpiote_event_clear
    nrfx_gpiote.o(i.GPIOTE_IRQHandler) refers to nrfx_gpiote.o(i.nrf_gpio_ports_read) for nrf_gpio_ports_read
    nrfx_gpiote.o(i.GPIOTE_IRQHandler) refers to nrfx_gpiote.o(i.channel_handler_get) for channel_handler_get
    nrfx_gpiote.o(i.GPIOTE_IRQHandler) refers to nrfx_gpiote.o(i.nrf_bitmask_bit_is_set) for nrf_bitmask_bit_is_set
    nrfx_gpiote.o(i.GPIOTE_IRQHandler) refers to nrfx_gpiote.o(i.channel_port_get) for channel_port_get
    nrfx_gpiote.o(i.GPIOTE_IRQHandler) refers to nrfx_gpiote.o(i.nrf_bitmask_bit_set) for nrf_bitmask_bit_set
    nrfx_gpiote.o(i.GPIOTE_IRQHandler) refers to nrfx_gpiote.o(i.nrf_gpio_cfg_sense_set) for nrf_gpio_cfg_sense_set
    nrfx_gpiote.o(i.GPIOTE_IRQHandler) refers to nrfx_gpiote.o(.bss) for m_cb
    nrfx_gpiote.o(i.channel_free) refers to nrfx_gpiote.o(.bss) for m_cb
    nrfx_gpiote.o(i.channel_handler_get) refers to nrfx_gpiote.o(.bss) for m_cb
    nrfx_gpiote.o(i.channel_port_alloc) refers to nrfx_gpiote.o(.bss) for m_cb
    nrfx_gpiote.o(i.channel_port_get) refers to nrfx_gpiote.o(.bss) for m_cb
    nrfx_gpiote.o(i.nrf_gpio_cfg_default) refers to nrfx_gpiote.o(i.nrf_gpio_cfg) for nrf_gpio_cfg
    nrfx_gpiote.o(i.nrf_gpio_ports_read) refers to nrfx_gpiote.o(.constdata) for .constdata
    nrfx_gpiote.o(i.nrf_gpiote_event_clear) refers to nrfx_gpiote.o(i.nrf_gpiote_event_addr_get) for nrf_gpiote_event_addr_get
    nrfx_gpiote.o(i.nrf_gpiote_event_is_set) refers to nrfx_gpiote.o(i.nrf_gpiote_event_addr_get) for nrf_gpiote_event_addr_get
    nrfx_gpiote.o(i.nrfx_gpiote_clr_task_addr_get) refers to nrfx_gpiote.o(i.channel_port_get) for channel_port_get
    nrfx_gpiote.o(i.nrfx_gpiote_clr_task_addr_get) refers to nrfx_gpiote.o(i.nrf_gpiote_task_addr_get) for nrf_gpiote_task_addr_get
    nrfx_gpiote.o(i.nrfx_gpiote_clr_task_trigger) refers to nrfx_gpiote.o(i.channel_port_get) for channel_port_get
    nrfx_gpiote.o(i.nrfx_gpiote_in_event_addr_get) refers to nrfx_gpiote.o(i.pin_in_use_by_te) for pin_in_use_by_te
    nrfx_gpiote.o(i.nrfx_gpiote_in_event_addr_get) refers to nrfx_gpiote.o(i.channel_port_get) for channel_port_get
    nrfx_gpiote.o(i.nrfx_gpiote_in_event_addr_get) refers to nrfx_gpiote.o(i.nrf_gpiote_event_addr_get) for nrf_gpiote_event_addr_get
    nrfx_gpiote.o(i.nrfx_gpiote_in_event_disable) refers to nrfx_gpiote.o(i.pin_in_use_by_port) for pin_in_use_by_port
    nrfx_gpiote.o(i.nrfx_gpiote_in_event_disable) refers to nrfx_gpiote.o(i.nrf_gpio_cfg_sense_set) for nrf_gpio_cfg_sense_set
    nrfx_gpiote.o(i.nrfx_gpiote_in_event_disable) refers to nrfx_gpiote.o(i.pin_in_use_by_te) for pin_in_use_by_te
    nrfx_gpiote.o(i.nrfx_gpiote_in_event_disable) refers to nrfx_gpiote.o(i.channel_port_get) for channel_port_get
    nrfx_gpiote.o(i.nrfx_gpiote_in_event_enable) refers to nrfx_gpiote.o(i.pin_in_use_by_port) for pin_in_use_by_port
    nrfx_gpiote.o(i.nrfx_gpiote_in_event_enable) refers to nrfx_gpiote.o(i.channel_port_get) for channel_port_get
    nrfx_gpiote.o(i.nrfx_gpiote_in_event_enable) refers to nrfx_gpiote.o(i.nrf_gpio_pin_read) for nrf_gpio_pin_read
    nrfx_gpiote.o(i.nrfx_gpiote_in_event_enable) refers to nrfx_gpiote.o(i.nrf_gpio_cfg_sense_set) for nrf_gpio_cfg_sense_set
    nrfx_gpiote.o(i.nrfx_gpiote_in_event_enable) refers to nrfx_gpiote.o(i.pin_in_use_by_te) for pin_in_use_by_te
    nrfx_gpiote.o(i.nrfx_gpiote_in_event_enable) refers to nrfx_gpiote.o(i.nrf_gpiote_event_clear) for nrf_gpiote_event_clear
    nrfx_gpiote.o(i.nrfx_gpiote_in_event_enable) refers to nrfx_gpiote.o(i.channel_handler_get) for channel_handler_get
    nrfx_gpiote.o(i.nrfx_gpiote_in_event_enable) refers to nrfx_gpiote.o(i.nrf_gpiote_int_enable) for nrf_gpiote_int_enable
    nrfx_gpiote.o(i.nrfx_gpiote_in_event_enable) refers to nrfx_gpiote.o(.bss) for m_cb
    nrfx_gpiote.o(i.nrfx_gpiote_in_init) refers to nrfx_gpiote.o(i.pin_in_use_by_gpiote) for pin_in_use_by_gpiote
    nrfx_gpiote.o(i.nrfx_gpiote_in_init) refers to nrfx_gpiote.o(i.channel_port_alloc) for channel_port_alloc
    nrfx_gpiote.o(i.nrfx_gpiote_in_init) refers to nrfx_gpiote.o(i.nrf_gpio_cfg) for nrf_gpio_cfg
    nrfx_gpiote.o(i.nrfx_gpiote_in_init) refers to nrfx_gpiote.o(i.pin_configured_set) for pin_configured_set
    nrfx_gpiote.o(i.nrfx_gpiote_in_init) refers to nrfx_gpiote.o(.bss) for m_cb
    nrfx_gpiote.o(i.nrfx_gpiote_in_is_set) refers to nrfx_gpiote.o(i.nrf_gpio_pin_read) for nrf_gpio_pin_read
    nrfx_gpiote.o(i.nrfx_gpiote_in_uninit) refers to nrfx_gpiote.o(i.nrfx_gpiote_in_event_disable) for nrfx_gpiote_in_event_disable
    nrfx_gpiote.o(i.nrfx_gpiote_in_uninit) refers to nrfx_gpiote.o(i.pin_in_use_by_te) for pin_in_use_by_te
    nrfx_gpiote.o(i.nrfx_gpiote_in_uninit) refers to nrfx_gpiote.o(i.channel_port_get) for channel_port_get
    nrfx_gpiote.o(i.nrfx_gpiote_in_uninit) refers to nrfx_gpiote.o(i.nrf_gpiote_te_default) for nrf_gpiote_te_default
    nrfx_gpiote.o(i.nrfx_gpiote_in_uninit) refers to nrfx_gpiote.o(i.pin_configured_check) for pin_configured_check
    nrfx_gpiote.o(i.nrfx_gpiote_in_uninit) refers to nrfx_gpiote.o(i.nrf_gpio_cfg_default) for nrf_gpio_cfg_default
    nrfx_gpiote.o(i.nrfx_gpiote_in_uninit) refers to nrfx_gpiote.o(i.pin_configured_clear) for pin_configured_clear
    nrfx_gpiote.o(i.nrfx_gpiote_in_uninit) refers to nrfx_gpiote.o(i.channel_free) for channel_free
    nrfx_gpiote.o(i.nrfx_gpiote_in_uninit) refers to nrfx_gpiote.o(i.pin_in_use_clear) for pin_in_use_clear
    nrfx_gpiote.o(i.nrfx_gpiote_init) refers to nrfx_gpiote.o(i.pin_in_use_clear) for pin_in_use_clear
    nrfx_gpiote.o(i.nrfx_gpiote_init) refers to nrfx_gpiote.o(i.channel_free) for channel_free
    nrfx_gpiote.o(i.nrfx_gpiote_init) refers to nrfx_gpiote.o(i.nrf_gpiote_event_clear) for nrf_gpiote_event_clear
    nrfx_gpiote.o(i.nrfx_gpiote_init) refers to nrfx_gpiote.o(i.nrf_gpiote_int_enable) for nrf_gpiote_int_enable
    nrfx_gpiote.o(i.nrfx_gpiote_init) refers to nrfx_gpiote.o(.bss) for m_cb
    nrfx_gpiote.o(i.nrfx_gpiote_is_init) refers to nrfx_gpiote.o(.bss) for m_cb
    nrfx_gpiote.o(i.nrfx_gpiote_out_clear) refers to nrfx_gpiote.o(i.nrf_gpio_pin_clear) for nrf_gpio_pin_clear
    nrfx_gpiote.o(i.nrfx_gpiote_out_init) refers to nrfx_gpiote.o(i.channel_port_alloc) for channel_port_alloc
    nrfx_gpiote.o(i.nrfx_gpiote_out_init) refers to nrfx_gpiote.o(i.nrf_gpio_pin_set) for nrf_gpio_pin_set
    nrfx_gpiote.o(i.nrfx_gpiote_out_init) refers to nrfx_gpiote.o(i.nrf_gpio_pin_clear) for nrf_gpio_pin_clear
    nrfx_gpiote.o(i.nrfx_gpiote_out_init) refers to nrfx_gpiote.o(i.nrf_gpio_cfg) for nrf_gpio_cfg
    nrfx_gpiote.o(i.nrfx_gpiote_out_init) refers to nrfx_gpiote.o(i.pin_configured_set) for pin_configured_set
    nrfx_gpiote.o(i.nrfx_gpiote_out_init) refers to nrfx_gpiote.o(.bss) for m_cb
    nrfx_gpiote.o(i.nrfx_gpiote_out_set) refers to nrfx_gpiote.o(i.nrf_gpio_pin_set) for nrf_gpio_pin_set
    nrfx_gpiote.o(i.nrfx_gpiote_out_task_addr_get) refers to nrfx_gpiote.o(i.channel_port_get) for channel_port_get
    nrfx_gpiote.o(i.nrfx_gpiote_out_task_addr_get) refers to nrfx_gpiote.o(i.nrf_gpiote_task_addr_get) for nrf_gpiote_task_addr_get
    nrfx_gpiote.o(i.nrfx_gpiote_out_task_disable) refers to nrfx_gpiote.o(.bss) for m_cb
    nrfx_gpiote.o(i.nrfx_gpiote_out_task_enable) refers to nrfx_gpiote.o(.bss) for m_cb
    nrfx_gpiote.o(i.nrfx_gpiote_out_task_force) refers to nrfx_gpiote.o(.bss) for m_cb
    nrfx_gpiote.o(i.nrfx_gpiote_out_task_trigger) refers to nrfx_gpiote.o(i.channel_port_get) for channel_port_get
    nrfx_gpiote.o(i.nrfx_gpiote_out_uninit) refers to nrfx_gpiote.o(i.pin_in_use_by_te) for pin_in_use_by_te
    nrfx_gpiote.o(i.nrfx_gpiote_out_uninit) refers to nrfx_gpiote.o(i.channel_port_get) for channel_port_get
    nrfx_gpiote.o(i.nrfx_gpiote_out_uninit) refers to nrfx_gpiote.o(i.channel_free) for channel_free
    nrfx_gpiote.o(i.nrfx_gpiote_out_uninit) refers to nrfx_gpiote.o(i.nrf_gpiote_te_default) for nrf_gpiote_te_default
    nrfx_gpiote.o(i.nrfx_gpiote_out_uninit) refers to nrfx_gpiote.o(i.pin_in_use_clear) for pin_in_use_clear
    nrfx_gpiote.o(i.nrfx_gpiote_out_uninit) refers to nrfx_gpiote.o(i.pin_configured_check) for pin_configured_check
    nrfx_gpiote.o(i.nrfx_gpiote_out_uninit) refers to nrfx_gpiote.o(i.nrf_gpio_cfg_default) for nrf_gpio_cfg_default
    nrfx_gpiote.o(i.nrfx_gpiote_out_uninit) refers to nrfx_gpiote.o(i.pin_configured_clear) for pin_configured_clear
    nrfx_gpiote.o(i.nrfx_gpiote_set_task_addr_get) refers to nrfx_gpiote.o(i.channel_port_get) for channel_port_get
    nrfx_gpiote.o(i.nrfx_gpiote_set_task_addr_get) refers to nrfx_gpiote.o(i.nrf_gpiote_task_addr_get) for nrf_gpiote_task_addr_get
    nrfx_gpiote.o(i.nrfx_gpiote_set_task_trigger) refers to nrfx_gpiote.o(i.channel_port_get) for channel_port_get
    nrfx_gpiote.o(i.nrfx_gpiote_uninit) refers to nrfx_gpiote.o(i.nrfx_gpiote_out_uninit) for nrfx_gpiote_out_uninit
    nrfx_gpiote.o(i.nrfx_gpiote_uninit) refers to nrfx_gpiote.o(i.pin_in_use_by_gpiote) for pin_in_use_by_gpiote
    nrfx_gpiote.o(i.nrfx_gpiote_uninit) refers to nrfx_gpiote.o(i.nrfx_gpiote_in_uninit) for nrfx_gpiote_in_uninit
    nrfx_gpiote.o(i.nrfx_gpiote_uninit) refers to nrfx_gpiote.o(.bss) for m_cb
    nrfx_gpiote.o(i.pin_configured_check) refers to nrfx_gpiote.o(i.nrf_bitmask_bit_is_set) for nrf_bitmask_bit_is_set
    nrfx_gpiote.o(i.pin_configured_check) refers to nrfx_gpiote.o(.bss) for m_cb
    nrfx_gpiote.o(i.pin_configured_clear) refers to nrfx_gpiote.o(.bss) for m_cb
    nrfx_gpiote.o(i.pin_configured_set) refers to nrfx_gpiote.o(i.nrf_bitmask_bit_set) for nrf_bitmask_bit_set
    nrfx_gpiote.o(i.pin_configured_set) refers to nrfx_gpiote.o(.bss) for m_cb
    nrfx_gpiote.o(i.pin_in_use_by_gpiote) refers to nrfx_gpiote.o(.bss) for m_cb
    nrfx_gpiote.o(i.pin_in_use_by_port) refers to nrfx_gpiote.o(.bss) for m_cb
    nrfx_gpiote.o(i.pin_in_use_by_te) refers to nrfx_gpiote.o(.bss) for m_cb
    nrfx_gpiote.o(i.pin_in_use_clear) refers to nrfx_gpiote.o(.bss) for m_cb
    app_error.o(i.app_error_handler_bare) refers to app_error_weak.o(i.app_error_fault_handler) for app_error_fault_handler
    app_error.o(i.app_error_save_and_stop) refers to app_error.o(.bss) for m_error_data
    app_error_handler_keil.o(.emb_text) refers to app_error_weak.o(i.app_error_fault_handler) for app_error_fault_handler
    app_fifo.o(i.app_fifo_get) refers to app_fifo.o(i.fifo_length) for fifo_length
    app_fifo.o(i.app_fifo_get) refers to app_fifo.o(i.fifo_get) for fifo_get
    app_fifo.o(i.app_fifo_peek) refers to app_fifo.o(i.fifo_length) for fifo_length
    app_fifo.o(i.app_fifo_peek) refers to app_fifo.o(i.fifo_peek) for fifo_peek
    app_fifo.o(i.app_fifo_put) refers to app_fifo.o(i.fifo_length) for fifo_length
    app_fifo.o(i.app_fifo_put) refers to app_fifo.o(i.fifo_put) for fifo_put
    app_fifo.o(i.app_fifo_read) refers to app_fifo.o(i.fifo_length) for fifo_length
    app_fifo.o(i.app_fifo_read) refers to app_fifo.o(i.fifo_get) for fifo_get
    app_fifo.o(i.app_fifo_write) refers to app_fifo.o(i.fifo_length) for fifo_length
    app_fifo.o(i.app_fifo_write) refers to app_fifo.o(i.fifo_put) for fifo_put
    app_fifo.o(i.fifo_get) refers to app_fifo.o(i.fifo_peek) for fifo_peek
    app_uart_fifo.o(i.app_uart_close) refers to nrfx_uarte.o(i.nrfx_uarte_uninit) for nrfx_uarte_uninit
    app_uart_fifo.o(i.app_uart_close) refers to nrfx_uart.o(i.nrfx_uart_uninit) for nrfx_uart_uninit
    app_uart_fifo.o(i.app_uart_close) refers to app_uart_fifo.o(.data) for app_uart_inst
    app_uart_fifo.o(i.app_uart_close) refers to nrf_drv_uart.o(.data) for nrf_drv_uart_use_easy_dma
    app_uart_fifo.o(i.app_uart_flush) refers to app_fifo.o(i.app_fifo_flush) for app_fifo_flush
    app_uart_fifo.o(i.app_uart_flush) refers to app_uart_fifo.o(.bss) for m_rx_fifo
    app_uart_fifo.o(i.app_uart_get) refers to app_fifo.o(i.app_fifo_get) for app_fifo_get
    app_uart_fifo.o(i.app_uart_get) refers to app_uart_fifo.o(i.nrf_drv_uart_rx) for nrf_drv_uart_rx
    app_uart_fifo.o(i.app_uart_get) refers to app_error.o(i.app_error_handler_bare) for app_error_handler_bare
    app_uart_fifo.o(i.app_uart_get) refers to app_uart_fifo.o(.data) for m_rx_ovf
    app_uart_fifo.o(i.app_uart_get) refers to app_uart_fifo.o(.bss) for m_rx_fifo
    app_uart_fifo.o(i.app_uart_init) refers to app_fifo.o(i.app_fifo_init) for app_fifo_init
    app_uart_fifo.o(i.app_uart_init) refers to memcpya.o(.text) for __aeabi_memcpy4
    app_uart_fifo.o(i.app_uart_init) refers to nrf_drv_uart.o(i.nrf_drv_uart_init) for nrf_drv_uart_init
    app_uart_fifo.o(i.app_uart_init) refers to app_uart_fifo.o(i.nrf_drv_uart_rx) for nrf_drv_uart_rx
    app_uart_fifo.o(i.app_uart_init) refers to app_uart_fifo.o(.data) for m_event_handler
    app_uart_fifo.o(i.app_uart_init) refers to app_uart_fifo.o(.bss) for m_rx_fifo
    app_uart_fifo.o(i.app_uart_init) refers to app_uart_fifo.o(.constdata) for .constdata
    app_uart_fifo.o(i.app_uart_init) refers to app_uart_fifo.o(i.uart_event_handler) for uart_event_handler
    app_uart_fifo.o(i.app_uart_put) refers to app_fifo.o(i.app_fifo_put) for app_fifo_put
    app_uart_fifo.o(i.app_uart_put) refers to nrfx_uarte.o(i.nrfx_uarte_tx_in_progress) for nrfx_uarte_tx_in_progress
    app_uart_fifo.o(i.app_uart_put) refers to nrfx_uart.o(i.nrfx_uart_tx_in_progress) for nrfx_uart_tx_in_progress
    app_uart_fifo.o(i.app_uart_put) refers to app_fifo.o(i.app_fifo_get) for app_fifo_get
    app_uart_fifo.o(i.app_uart_put) refers to app_uart_fifo.o(i.nrf_drv_uart_tx) for nrf_drv_uart_tx
    app_uart_fifo.o(i.app_uart_put) refers to app_uart_fifo.o(.bss) for m_tx_fifo
    app_uart_fifo.o(i.app_uart_put) refers to app_uart_fifo.o(.data) for app_uart_inst
    app_uart_fifo.o(i.app_uart_put) refers to nrf_drv_uart.o(.data) for nrf_drv_uart_use_easy_dma
    app_uart_fifo.o(i.nrf_drv_uart_rx) refers to nrfx_uarte.o(i.nrfx_uarte_rx) for nrfx_uarte_rx
    app_uart_fifo.o(i.nrf_drv_uart_rx) refers to nrfx_uart.o(i.nrfx_uart_rx) for nrfx_uart_rx
    app_uart_fifo.o(i.nrf_drv_uart_rx) refers to nrf_drv_uart.o(.data) for nrf_drv_uart_use_easy_dma
    app_uart_fifo.o(i.nrf_drv_uart_tx) refers to nrfx_uarte.o(i.nrfx_uarte_tx) for nrfx_uarte_tx
    app_uart_fifo.o(i.nrf_drv_uart_tx) refers to nrfx_uart.o(i.nrfx_uart_tx) for nrfx_uart_tx
    app_uart_fifo.o(i.nrf_drv_uart_tx) refers to nrf_drv_uart.o(.data) for nrf_drv_uart_use_easy_dma
    app_uart_fifo.o(i.uart_event_handler) refers to app_fifo.o(i.app_fifo_put) for app_fifo_put
    app_uart_fifo.o(i.uart_event_handler) refers to app_uart_fifo.o(i.fifo_length) for fifo_length
    app_uart_fifo.o(i.uart_event_handler) refers to app_uart_fifo.o(i.nrf_drv_uart_rx) for nrf_drv_uart_rx
    app_uart_fifo.o(i.uart_event_handler) refers to app_fifo.o(i.app_fifo_get) for app_fifo_get
    app_uart_fifo.o(i.uart_event_handler) refers to app_uart_fifo.o(i.nrf_drv_uart_tx) for nrf_drv_uart_tx
    app_uart_fifo.o(i.uart_event_handler) refers to app_uart_fifo.o(.bss) for m_rx_fifo
    app_uart_fifo.o(i.uart_event_handler) refers to app_uart_fifo.o(.data) for m_event_handler
    app_util_platform.o(i.app_util_critical_region_enter) refers to app_util_platform.o(i.app_util_disable_irq) for app_util_disable_irq
    app_util_platform.o(i.app_util_critical_region_exit) refers to app_util_platform.o(i.app_util_enable_irq) for app_util_enable_irq
    app_util_platform.o(i.app_util_disable_irq) refers to app_util_platform.o(.data) for m_in_critical_region
    app_util_platform.o(i.app_util_enable_irq) refers to app_util_platform.o(.data) for m_in_critical_region
    nrf_assert.o(i.assert_nrf_callback) refers to app_error_weak.o(i.app_error_fault_handler) for app_error_fault_handler
    nrf_atomic.o(i.nrf_atomic_flag_clear) refers to nrf_atomic.o(i.nrf_atomic_u32_and) for nrf_atomic_u32_and
    nrf_atomic.o(i.nrf_atomic_flag_clear_fetch) refers to nrf_atomic.o(i.nrf_atomic_u32_fetch_and) for nrf_atomic_u32_fetch_and
    nrf_atomic.o(i.nrf_atomic_flag_set) refers to nrf_atomic.o(i.nrf_atomic_u32_or) for nrf_atomic_u32_or
    nrf_atomic.o(i.nrf_atomic_flag_set_fetch) refers to nrf_atomic.o(i.nrf_atomic_u32_fetch_or) for nrf_atomic_u32_fetch_or
    nrf_atomic.o(i.nrf_atomic_u32_add) refers to nrf_atomic.o(.emb_text) for __asm___12_nrf_atomic_c_85ca2469__nrf_atomic_internal_add
    nrf_atomic.o(i.nrf_atomic_u32_and) refers to nrf_atomic.o(.emb_text) for __asm___12_nrf_atomic_c_85ca2469__nrf_atomic_internal_and
    nrf_atomic.o(i.nrf_atomic_u32_cmp_exch) refers to nrf_atomic.o(.emb_text) for __asm___12_nrf_atomic_c_85ca2469__nrf_atomic_internal_cmp_exch
    nrf_atomic.o(i.nrf_atomic_u32_fetch_add) refers to nrf_atomic.o(.emb_text) for __asm___12_nrf_atomic_c_85ca2469__nrf_atomic_internal_add
    nrf_atomic.o(i.nrf_atomic_u32_fetch_and) refers to nrf_atomic.o(.emb_text) for __asm___12_nrf_atomic_c_85ca2469__nrf_atomic_internal_and
    nrf_atomic.o(i.nrf_atomic_u32_fetch_or) refers to nrf_atomic.o(.emb_text) for __asm___12_nrf_atomic_c_85ca2469__nrf_atomic_internal_orr
    nrf_atomic.o(i.nrf_atomic_u32_fetch_store) refers to nrf_atomic.o(.emb_text) for __asm___12_nrf_atomic_c_85ca2469__nrf_atomic_internal_mov
    nrf_atomic.o(i.nrf_atomic_u32_fetch_sub) refers to nrf_atomic.o(.emb_text) for __asm___12_nrf_atomic_c_85ca2469__nrf_atomic_internal_sub
    nrf_atomic.o(i.nrf_atomic_u32_fetch_sub_hs) refers to nrf_atomic.o(.emb_text) for __asm___12_nrf_atomic_c_85ca2469__nrf_atomic_internal_sub_hs
    nrf_atomic.o(i.nrf_atomic_u32_fetch_xor) refers to nrf_atomic.o(.emb_text) for __asm___12_nrf_atomic_c_85ca2469__nrf_atomic_internal_eor
    nrf_atomic.o(i.nrf_atomic_u32_or) refers to nrf_atomic.o(.emb_text) for __asm___12_nrf_atomic_c_85ca2469__nrf_atomic_internal_orr
    nrf_atomic.o(i.nrf_atomic_u32_store) refers to nrf_atomic.o(.emb_text) for __asm___12_nrf_atomic_c_85ca2469__nrf_atomic_internal_mov
    nrf_atomic.o(i.nrf_atomic_u32_sub) refers to nrf_atomic.o(.emb_text) for __asm___12_nrf_atomic_c_85ca2469__nrf_atomic_internal_sub
    nrf_atomic.o(i.nrf_atomic_u32_sub_hs) refers to nrf_atomic.o(.emb_text) for __asm___12_nrf_atomic_c_85ca2469__nrf_atomic_internal_sub_hs
    nrf_atomic.o(i.nrf_atomic_u32_xor) refers to nrf_atomic.o(.emb_text) for __asm___12_nrf_atomic_c_85ca2469__nrf_atomic_internal_eor
    nrf_balloc.o(i.nrf_balloc_alloc) refers to app_util_platform.o(i.app_util_critical_region_enter) for app_util_critical_region_enter
    nrf_balloc.o(i.nrf_balloc_alloc) refers to nrf_balloc.o(i.nrf_balloc_idx2block) for nrf_balloc_idx2block
    nrf_balloc.o(i.nrf_balloc_alloc) refers to app_util_platform.o(i.app_util_critical_region_exit) for app_util_critical_region_exit
    nrf_balloc.o(i.nrf_balloc_free) refers to app_util_platform.o(i.app_util_critical_region_enter) for app_util_critical_region_enter
    nrf_balloc.o(i.nrf_balloc_free) refers to nrf_balloc.o(i.nrf_balloc_block2idx) for nrf_balloc_block2idx
    nrf_balloc.o(i.nrf_balloc_free) refers to app_util_platform.o(i.app_util_critical_region_exit) for app_util_critical_region_exit
    nrf_fprintf.o(i.nrf_fprintf) refers to nrf_fprintf_format.o(i.nrf_fprintf_fmt) for nrf_fprintf_fmt
    nrf_fprintf_format.o(i.buffer_add) refers to nrf_fprintf.o(i.nrf_fprintf_buffer_flush) for nrf_fprintf_buffer_flush
    nrf_fprintf_format.o(i.int_print) refers to nrf_fprintf_format.o(i.buffer_add) for buffer_add
    nrf_fprintf_format.o(i.int_print) refers to nrf_fprintf_format.o(i.unsigned_print) for unsigned_print
    nrf_fprintf_format.o(i.nrf_fprintf_fmt) refers to nrf_fprintf_format.o(i.buffer_add) for buffer_add
    nrf_fprintf_format.o(i.nrf_fprintf_fmt) refers to nrf_fprintf_format.o(i.int_print) for int_print
    nrf_fprintf_format.o(i.nrf_fprintf_fmt) refers to nrf_fprintf_format.o(i.unsigned_print) for unsigned_print
    nrf_fprintf_format.o(i.nrf_fprintf_fmt) refers to nrf_fprintf_format.o(i.string_print) for string_print
    nrf_fprintf_format.o(i.nrf_fprintf_fmt) refers to nrf_fprintf.o(i.nrf_fprintf_buffer_flush) for nrf_fprintf_buffer_flush
    nrf_fprintf_format.o(i.string_print) refers to nrf_fprintf_format.o(i.buffer_add) for buffer_add
    nrf_fprintf_format.o(i.string_print) refers to strlen.o(.text) for strlen
    nrf_fprintf_format.o(i.unsigned_print) refers to nrf_fprintf_format.o(i.buffer_add) for buffer_add
    nrf_fprintf_format.o(i.unsigned_print) refers to nrf_fprintf_format.o(.constdata) for _aV2C
    nrf_memobj.o(i.memobj_op) refers to memcpya.o(.text) for __aeabi_memcpy
    nrf_memobj.o(i.nrf_memobj_alloc) refers to nrf_balloc.o(i.nrf_balloc_alloc) for nrf_balloc_alloc
    nrf_memobj.o(i.nrf_memobj_alloc) refers to nrf_memobj.o(i.nrf_memobj_free) for nrf_memobj_free
    nrf_memobj.o(i.nrf_memobj_free) refers to nrf_balloc.o(i.nrf_balloc_free) for nrf_balloc_free
    nrf_memobj.o(i.nrf_memobj_get) refers to nrf_atomic.o(i.nrf_atomic_u32_add) for nrf_atomic_u32_add
    nrf_memobj.o(i.nrf_memobj_pool_init) refers to nrf_balloc.o(i.nrf_balloc_init) for nrf_balloc_init
    nrf_memobj.o(i.nrf_memobj_put) refers to nrf_atomic.o(i.nrf_atomic_u32_sub) for nrf_atomic_u32_sub
    nrf_memobj.o(i.nrf_memobj_put) refers to nrf_memobj.o(i.nrf_memobj_free) for nrf_memobj_free
    nrf_memobj.o(i.nrf_memobj_read) refers to nrf_memobj.o(i.memobj_op) for memobj_op
    nrf_memobj.o(i.nrf_memobj_write) refers to nrf_memobj.o(i.memobj_op) for memobj_op
    nrf_ringbuf.o(i.nrf_ringbuf_alloc) refers to nrf_atomic.o(i.nrf_atomic_flag_set_fetch) for nrf_atomic_flag_set_fetch
    nrf_ringbuf.o(i.nrf_ringbuf_alloc) refers to nrf_atomic.o(i.nrf_atomic_flag_clear) for nrf_atomic_flag_clear
    nrf_ringbuf.o(i.nrf_ringbuf_cpy_get) refers to nrf_atomic.o(i.nrf_atomic_flag_set_fetch) for nrf_atomic_flag_set_fetch
    nrf_ringbuf.o(i.nrf_ringbuf_cpy_get) refers to memcpya.o(.text) for __aeabi_memcpy
    nrf_ringbuf.o(i.nrf_ringbuf_cpy_get) refers to nrf_atomic.o(i.nrf_atomic_flag_clear) for nrf_atomic_flag_clear
    nrf_ringbuf.o(i.nrf_ringbuf_cpy_put) refers to nrf_atomic.o(i.nrf_atomic_flag_set_fetch) for nrf_atomic_flag_set_fetch
    nrf_ringbuf.o(i.nrf_ringbuf_cpy_put) refers to memcpya.o(.text) for __aeabi_memcpy
    nrf_ringbuf.o(i.nrf_ringbuf_cpy_put) refers to nrf_atomic.o(i.nrf_atomic_flag_clear) for nrf_atomic_flag_clear
    nrf_ringbuf.o(i.nrf_ringbuf_free) refers to nrf_atomic.o(i.nrf_atomic_flag_clear) for nrf_atomic_flag_clear
    nrf_ringbuf.o(i.nrf_ringbuf_get) refers to nrf_atomic.o(i.nrf_atomic_flag_set_fetch) for nrf_atomic_flag_set_fetch
    nrf_ringbuf.o(i.nrf_ringbuf_get) refers to nrf_atomic.o(i.nrf_atomic_flag_clear) for nrf_atomic_flag_clear
    nrf_ringbuf.o(i.nrf_ringbuf_put) refers to nrf_atomic.o(i.nrf_atomic_flag_clear_fetch) for nrf_atomic_flag_clear_fetch
    nrf_strerror.o(i.nrf_strerror_find) refers to nrf_strerror.o(.constdata) for nrf_strerror_array
    nrf_strerror.o(i.nrf_strerror_get) refers to nrf_strerror.o(i.nrf_strerror_find) for nrf_strerror_find
    nrf_strerror.o(i.nrf_strerror_get) refers to nrf_strerror.o(.constdata) for m_unknown_str
    nrf_strerror.o(.constdata) refers to nrf_strerror.o(.conststring) for .conststring
    app_timer.o(i.RTC1_IRQHandler) refers to app_timer.o(i.timer_timeouts_check) for timer_timeouts_check
    app_timer.o(i.SWI1_EGU1_IRQHandler) refers to app_timer.o(i.timer_list_handler) for timer_list_handler
    app_timer.o(i.app_timer_cnt_diff_compute) refers to app_timer.o(i.ticks_diff_get) for ticks_diff_get
    app_timer.o(i.app_timer_cnt_get) refers to app_timer.o(i.rtc1_counter_get) for rtc1_counter_get
    app_timer.o(i.app_timer_create) refers to app_timer.o(.bss) for m_op_queue
    app_timer.o(i.app_timer_init) refers to app_timer.o(i.rtc1_stop) for rtc1_stop
    app_timer.o(i.app_timer_init) refers to app_timer.o(i.NVIC_ClearPendingIRQ) for NVIC_ClearPendingIRQ
    app_timer.o(i.app_timer_init) refers to app_timer.o(i.NVIC_SetPriority) for NVIC_SetPriority
    app_timer.o(i.app_timer_init) refers to app_timer.o(i.NVIC_EnableIRQ) for NVIC_EnableIRQ
    app_timer.o(i.app_timer_init) refers to app_timer.o(i.rtc1_init) for rtc1_init
    app_timer.o(i.app_timer_init) refers to app_timer.o(i.rtc1_counter_get) for rtc1_counter_get
    app_timer.o(i.app_timer_init) refers to app_timer.o(.bss) for m_op_queue
    app_timer.o(i.app_timer_init) refers to app_timer.o(.data) for mp_timer_id_head
    app_timer.o(i.app_timer_start) refers to app_timer.o(i.timer_start_op_schedule) for timer_start_op_schedule
    app_timer.o(i.app_timer_start) refers to app_timer.o(.bss) for m_op_queue
    app_timer.o(i.app_timer_stop) refers to app_timer.o(i.timer_stop_op_schedule) for timer_stop_op_schedule
    app_timer.o(i.app_timer_stop) refers to app_timer.o(.bss) for m_op_queue
    app_timer.o(i.app_timer_stop_all) refers to app_timer.o(i.timer_stop_op_schedule) for timer_stop_op_schedule
    app_timer.o(i.app_timer_stop_all) refers to app_timer.o(.bss) for m_op_queue
    app_timer.o(i.compare_reg_update) refers to app_timer.o(i.rtc1_counter_get) for rtc1_counter_get
    app_timer.o(i.compare_reg_update) refers to app_timer.o(i.ticks_diff_get) for ticks_diff_get
    app_timer.o(i.compare_reg_update) refers to app_timer.o(i.rtc1_start) for rtc1_start
    app_timer.o(i.compare_reg_update) refers to app_timer.o(i.rtc1_compare0_set) for rtc1_compare0_set
    app_timer.o(i.compare_reg_update) refers to app_timer.o(i.nrfx_coredep_delay_us) for nrfx_coredep_delay_us
    app_timer.o(i.compare_reg_update) refers to app_timer.o(i.timer_timeouts_check_sched) for timer_timeouts_check_sched
    app_timer.o(i.compare_reg_update) refers to app_timer.o(i.rtc1_stop) for rtc1_stop
    app_timer.o(i.compare_reg_update) refers to app_timer.o(.data) for mp_timer_id_head
    app_timer.o(i.elapsed_ticks_acquire) refers to app_timer.o(.data) for m_ticks_elapsed_q_read_ind
    app_timer.o(i.expired_timers_handler) refers to app_timer.o(.data) for mp_timer_id_head
    app_timer.o(i.list_insertions_handler) refers to app_timer.o(i.timer_list_remove) for timer_list_remove
    app_timer.o(i.list_insertions_handler) refers to app_timer.o(i.ticks_diff_get) for ticks_diff_get
    app_timer.o(i.list_insertions_handler) refers to app_timer.o(i.timer_list_insert) for timer_list_insert
    app_timer.o(i.list_insertions_handler) refers to app_timer.o(.data) for mp_timer_id_head
    app_timer.o(i.list_insertions_handler) refers to app_timer.o(.bss) for m_op_queue
    app_timer.o(i.nrfx_coredep_delay_us) refers to app_timer.o(.constdata) for delay_machine_code
    app_timer.o(i.rtc1_init) refers to app_timer.o(i.NVIC_SetPriority) for NVIC_SetPriority
    app_timer.o(i.rtc1_start) refers to app_timer.o(i.NVIC_ClearPendingIRQ) for NVIC_ClearPendingIRQ
    app_timer.o(i.rtc1_start) refers to app_timer.o(i.NVIC_EnableIRQ) for NVIC_EnableIRQ
    app_timer.o(i.rtc1_start) refers to app_timer.o(i.nrfx_coredep_delay_us) for nrfx_coredep_delay_us
    app_timer.o(i.rtc1_start) refers to app_timer.o(.data) for m_rtc1_running
    app_timer.o(i.rtc1_stop) refers to app_timer.o(i.nrfx_coredep_delay_us) for nrfx_coredep_delay_us
    app_timer.o(i.rtc1_stop) refers to app_timer.o(.data) for m_ticks_latest
    app_timer.o(i.timer_list_handler) refers to app_timer.o(i.elapsed_ticks_acquire) for elapsed_ticks_acquire
    app_timer.o(i.timer_list_handler) refers to app_timer.o(i.expired_timers_handler) for expired_timers_handler
    app_timer.o(i.timer_list_handler) refers to app_timer.o(i.list_insertions_handler) for list_insertions_handler
    app_timer.o(i.timer_list_handler) refers to app_timer.o(i.compare_reg_update) for compare_reg_update
    app_timer.o(i.timer_list_handler) refers to app_timer.o(.data) for m_ticks_latest
    app_timer.o(i.timer_list_handler_sched) refers to app_timer.o(i.NVIC_SetPendingIRQ) for NVIC_SetPendingIRQ
    app_timer.o(i.timer_list_insert) refers to app_timer.o(.data) for mp_timer_id_head
    app_timer.o(i.timer_list_remove) refers to app_timer.o(i.nrfx_coredep_delay_us) for nrfx_coredep_delay_us
    app_timer.o(i.timer_list_remove) refers to app_timer.o(.data) for mp_timer_id_head
    app_timer.o(i.timer_start_op_schedule) refers to app_util_platform.o(i.app_util_critical_region_enter) for app_util_critical_region_enter
    app_timer.o(i.timer_start_op_schedule) refers to app_timer.o(i.user_op_alloc) for user_op_alloc
    app_timer.o(i.timer_start_op_schedule) refers to app_timer.o(i.rtc1_counter_get) for rtc1_counter_get
    app_timer.o(i.timer_start_op_schedule) refers to app_timer.o(i.user_op_enque) for user_op_enque
    app_timer.o(i.timer_start_op_schedule) refers to app_util_platform.o(i.app_util_critical_region_exit) for app_util_critical_region_exit
    app_timer.o(i.timer_start_op_schedule) refers to app_timer.o(i.timer_list_handler_sched) for timer_list_handler_sched
    app_timer.o(i.timer_stop_op_schedule) refers to app_util_platform.o(i.app_util_critical_region_enter) for app_util_critical_region_enter
    app_timer.o(i.timer_stop_op_schedule) refers to app_timer.o(i.user_op_alloc) for user_op_alloc
    app_timer.o(i.timer_stop_op_schedule) refers to app_timer.o(i.user_op_enque) for user_op_enque
    app_timer.o(i.timer_stop_op_schedule) refers to app_util_platform.o(i.app_util_critical_region_exit) for app_util_critical_region_exit
    app_timer.o(i.timer_stop_op_schedule) refers to app_timer.o(i.timer_list_handler_sched) for timer_list_handler_sched
    app_timer.o(i.timer_timeouts_check) refers to app_timer.o(i.rtc1_counter_get) for rtc1_counter_get
    app_timer.o(i.timer_timeouts_check) refers to app_timer.o(i.ticks_diff_get) for ticks_diff_get
    app_timer.o(i.timer_timeouts_check) refers to app_timer.o(i.timeout_handler_exec) for timeout_handler_exec
    app_timer.o(i.timer_timeouts_check) refers to app_timer.o(i.timer_list_handler_sched) for timer_list_handler_sched
    app_timer.o(i.timer_timeouts_check) refers to app_timer.o(.data) for mp_timer_id_head
    app_timer.o(i.timer_timeouts_check_sched) refers to app_timer.o(i.NVIC_SetPendingIRQ) for NVIC_SetPendingIRQ
    app_timer.o(i.user_op_alloc) refers to app_timer.o(.bss) for m_op_queue
    app_timer.o(i.user_op_enque) refers to app_timer.o(.bss) for m_op_queue
    retarget.o(i.fgetc) refers to app_uart_fifo.o(i.app_uart_get) for app_uart_get
    retarget.o(i.fputc) refers to app_uart_fifo.o(i.app_uart_put) for app_uart_put
    nrf_esb.o(i.RADIO_IRQHandler) refers to nrf_esb.o(.data) for on_radio_end
    nrf_esb.o(i.SWI0_EGU0_IRQHandler) refers to nrf_esb.o(i.nrf_esb_get_clear_interrupts) for nrf_esb_get_clear_interrupts
    nrf_esb.o(i.SWI0_EGU0_IRQHandler) refers to nrf_esb.o(.data) for m_last_tx_attempts
    nrf_esb.o(i.TIMER3_IRQHandler) refers to nrf_esb.o(.data) for m_nrf_esb_mainstate
    nrf_esb.o(i.addr_conv) refers to nrf_esb.o(i.bytewise_bit_swap) for bytewise_bit_swap
    nrf_esb.o(i.apply_address_workarounds) refers to nrf_esb.o(.data) for m_esb_addr
    nrf_esb.o(i.clear_events_restart_rx) refers to nrf_esb.o(.data) for m_radio_shorts_common
    nrf_esb.o(i.clear_events_restart_rx) refers to nrf_esb.o(.bss) for m_config_local
    nrf_esb.o(i.initialize_fifos) refers to nrf_esb.o(i.reset_fifos) for reset_fifos
    nrf_esb.o(i.initialize_fifos) refers to nrf_esb.o(.bss) for m_tx_fifo_payload
    nrf_esb.o(i.nrf_esb_disable) refers to nrf_esb.o(i.reset_fifos) for reset_fifos
    nrf_esb.o(i.nrf_esb_disable) refers to memseta.o(.text) for __aeabi_memclr
    nrf_esb.o(i.nrf_esb_disable) refers to nrf_esb.o(i.NVIC_DisableIRQ) for NVIC_DisableIRQ
    nrf_esb.o(i.nrf_esb_disable) refers to nrf_esb.o(.data) for m_nrf_esb_mainstate
    nrf_esb.o(i.nrf_esb_disable) refers to nrf_esb.o(.bss) for m_rx_pipe_info
    nrf_esb.o(i.nrf_esb_enable_pipes) refers to nrf_esb.o(i.apply_address_workarounds) for apply_address_workarounds
    nrf_esb.o(i.nrf_esb_enable_pipes) refers to nrf_esb.o(.data) for m_nrf_esb_mainstate
    nrf_esb.o(i.nrf_esb_flush_rx) refers to nrf_esb.o(i.NVIC_DisableIRQ) for NVIC_DisableIRQ
    nrf_esb.o(i.nrf_esb_flush_rx) refers to memseta.o(.text) for __aeabi_memclr
    nrf_esb.o(i.nrf_esb_flush_rx) refers to nrf_esb.o(i.NVIC_EnableIRQ) for NVIC_EnableIRQ
    nrf_esb.o(i.nrf_esb_flush_rx) refers to nrf_esb.o(.data) for m_esb_initialized
    nrf_esb.o(i.nrf_esb_flush_rx) refers to nrf_esb.o(.bss) for m_rx_fifo
    nrf_esb.o(i.nrf_esb_flush_tx) refers to nrf_esb.o(i.NVIC_DisableIRQ) for NVIC_DisableIRQ
    nrf_esb.o(i.nrf_esb_flush_tx) refers to nrf_esb.o(i.NVIC_EnableIRQ) for NVIC_EnableIRQ
    nrf_esb.o(i.nrf_esb_flush_tx) refers to nrf_esb.o(.data) for m_esb_initialized
    nrf_esb.o(i.nrf_esb_flush_tx) refers to nrf_esb.o(.bss) for m_tx_fifo
    nrf_esb.o(i.nrf_esb_get_clear_interrupts) refers to nrf_esb.o(i.NVIC_DisableIRQ) for NVIC_DisableIRQ
    nrf_esb.o(i.nrf_esb_get_clear_interrupts) refers to nrf_esb.o(i.NVIC_EnableIRQ) for NVIC_EnableIRQ
    nrf_esb.o(i.nrf_esb_get_clear_interrupts) refers to nrf_esb.o(.data) for m_esb_initialized
    nrf_esb.o(i.nrf_esb_get_rf_channel) refers to nrf_esb.o(.data) for m_esb_addr
    nrf_esb.o(i.nrf_esb_init) refers to nrf_esb.o(i.nrf_esb_disable) for nrf_esb_disable
    nrf_esb.o(i.nrf_esb_init) refers to memcpya.o(.text) for __aeabi_memcpy4
    nrf_esb.o(i.nrf_esb_init) refers to memseta.o(.text) for __aeabi_memclr
    nrf_esb.o(i.nrf_esb_init) refers to nrf_esb.o(i.update_radio_parameters) for update_radio_parameters
    nrf_esb.o(i.nrf_esb_init) refers to nrf_esb.o(i.initialize_fifos) for initialize_fifos
    nrf_esb.o(i.nrf_esb_init) refers to nrf_esb.o(i.sys_timer_init) for sys_timer_init
    nrf_esb.o(i.nrf_esb_init) refers to nrf_esb.o(i.ppi_init) for ppi_init
    nrf_esb.o(i.nrf_esb_init) refers to nrf_esb.o(i.NVIC_SetPriority) for NVIC_SetPriority
    nrf_esb.o(i.nrf_esb_init) refers to nrf_esb.o(i.NVIC_EnableIRQ) for NVIC_EnableIRQ
    nrf_esb.o(i.nrf_esb_init) refers to nrf_esb.o(.data) for m_esb_initialized
    nrf_esb.o(i.nrf_esb_init) refers to nrf_esb.o(.bss) for m_config_local
    nrf_esb.o(i.nrf_esb_is_idle) refers to nrf_esb.o(.data) for m_nrf_esb_mainstate
    nrf_esb.o(i.nrf_esb_pop_tx) refers to nrf_esb.o(i.NVIC_DisableIRQ) for NVIC_DisableIRQ
    nrf_esb.o(i.nrf_esb_pop_tx) refers to nrf_esb.o(i.NVIC_EnableIRQ) for NVIC_EnableIRQ
    nrf_esb.o(i.nrf_esb_pop_tx) refers to nrf_esb.o(.data) for m_esb_initialized
    nrf_esb.o(i.nrf_esb_pop_tx) refers to nrf_esb.o(.bss) for m_tx_fifo
    nrf_esb.o(i.nrf_esb_read_rx_payload) refers to nrf_esb.o(i.NVIC_DisableIRQ) for NVIC_DisableIRQ
    nrf_esb.o(i.nrf_esb_read_rx_payload) refers to memcpya.o(.text) for __aeabi_memcpy
    nrf_esb.o(i.nrf_esb_read_rx_payload) refers to nrf_esb.o(i.NVIC_EnableIRQ) for NVIC_EnableIRQ
    nrf_esb.o(i.nrf_esb_read_rx_payload) refers to nrf_esb.o(.data) for m_esb_initialized
    nrf_esb.o(i.nrf_esb_read_rx_payload) refers to nrf_esb.o(.bss) for m_rx_fifo
    nrf_esb.o(i.nrf_esb_reuse_pid) refers to nrf_esb.o(.data) for m_nrf_esb_mainstate
    nrf_esb.o(i.nrf_esb_set_address_length) refers to nrf_esb.o(i.apply_address_workarounds) for apply_address_workarounds
    nrf_esb.o(i.nrf_esb_set_address_length) refers to nrf_esb.o(.data) for m_nrf_esb_mainstate
    nrf_esb.o(i.nrf_esb_set_address_length) refers to nrf_esb.o(.bss) for m_config_local
    nrf_esb.o(i.nrf_esb_set_base_address_0) refers to nrf_esb.o(i.addr_conv) for addr_conv
    nrf_esb.o(i.nrf_esb_set_base_address_0) refers to nrf_esb.o(i.update_radio_addresses) for update_radio_addresses
    nrf_esb.o(i.nrf_esb_set_base_address_0) refers to nrf_esb.o(i.apply_address_workarounds) for apply_address_workarounds
    nrf_esb.o(i.nrf_esb_set_base_address_0) refers to nrf_esb.o(.data) for m_nrf_esb_mainstate
    nrf_esb.o(i.nrf_esb_set_base_address_1) refers to nrf_esb.o(i.addr_conv) for addr_conv
    nrf_esb.o(i.nrf_esb_set_base_address_1) refers to nrf_esb.o(i.update_radio_addresses) for update_radio_addresses
    nrf_esb.o(i.nrf_esb_set_base_address_1) refers to nrf_esb.o(i.apply_address_workarounds) for apply_address_workarounds
    nrf_esb.o(i.nrf_esb_set_base_address_1) refers to nrf_esb.o(.data) for m_nrf_esb_mainstate
    nrf_esb.o(i.nrf_esb_set_bitrate) refers to nrf_esb.o(i.update_radio_bitrate) for update_radio_bitrate
    nrf_esb.o(i.nrf_esb_set_bitrate) refers to nrf_esb.o(.data) for m_nrf_esb_mainstate
    nrf_esb.o(i.nrf_esb_set_bitrate) refers to nrf_esb.o(.bss) for m_config_local
    nrf_esb.o(i.nrf_esb_set_prefixes) refers to memcpya.o(.text) for __aeabi_memcpy
    nrf_esb.o(i.nrf_esb_set_prefixes) refers to nrf_esb.o(i.update_radio_addresses) for update_radio_addresses
    nrf_esb.o(i.nrf_esb_set_prefixes) refers to nrf_esb.o(i.apply_address_workarounds) for apply_address_workarounds
    nrf_esb.o(i.nrf_esb_set_prefixes) refers to nrf_esb.o(.data) for m_nrf_esb_mainstate
    nrf_esb.o(i.nrf_esb_set_retransmit_count) refers to nrf_esb.o(.data) for m_nrf_esb_mainstate
    nrf_esb.o(i.nrf_esb_set_retransmit_count) refers to nrf_esb.o(.bss) for m_config_local
    nrf_esb.o(i.nrf_esb_set_retransmit_delay) refers to nrf_esb.o(.data) for m_nrf_esb_mainstate
    nrf_esb.o(i.nrf_esb_set_retransmit_delay) refers to nrf_esb.o(.bss) for m_config_local
    nrf_esb.o(i.nrf_esb_set_rf_channel) refers to nrf_esb.o(.data) for m_nrf_esb_mainstate
    nrf_esb.o(i.nrf_esb_set_tx_power) refers to nrf_esb.o(i.update_radio_tx_power) for update_radio_tx_power
    nrf_esb.o(i.nrf_esb_set_tx_power) refers to nrf_esb.o(.data) for m_nrf_esb_mainstate
    nrf_esb.o(i.nrf_esb_set_tx_power) refers to nrf_esb.o(.bss) for m_config_local
    nrf_esb.o(i.nrf_esb_skip_tx) refers to nrf_esb.o(i.NVIC_DisableIRQ) for NVIC_DisableIRQ
    nrf_esb.o(i.nrf_esb_skip_tx) refers to nrf_esb.o(i.NVIC_EnableIRQ) for NVIC_EnableIRQ
    nrf_esb.o(i.nrf_esb_skip_tx) refers to nrf_esb.o(.data) for m_esb_initialized
    nrf_esb.o(i.nrf_esb_skip_tx) refers to nrf_esb.o(.bss) for m_tx_fifo
    nrf_esb.o(i.nrf_esb_start_rx) refers to nrf_esb.o(i.NVIC_ClearPendingIRQ) for NVIC_ClearPendingIRQ
    nrf_esb.o(i.nrf_esb_start_rx) refers to nrf_esb.o(i.NVIC_EnableIRQ) for NVIC_EnableIRQ
    nrf_esb.o(i.nrf_esb_start_rx) refers to nrf_esb.o(.data) for m_nrf_esb_mainstate
    nrf_esb.o(i.nrf_esb_start_rx) refers to nrf_esb.o(i.on_radio_disabled_rx) for on_radio_disabled_rx
    nrf_esb.o(i.nrf_esb_start_rx) refers to nrf_esb.o(.bss) for m_rx_payload_buffer
    nrf_esb.o(i.nrf_esb_start_tx) refers to nrf_esb.o(i.start_tx_transaction) for start_tx_transaction
    nrf_esb.o(i.nrf_esb_start_tx) refers to nrf_esb.o(.data) for m_nrf_esb_mainstate
    nrf_esb.o(i.nrf_esb_start_tx) refers to nrf_esb.o(.bss) for m_tx_fifo
    nrf_esb.o(i.nrf_esb_stop_rx) refers to nrf_esb.o(.data) for m_nrf_esb_mainstate
    nrf_esb.o(i.nrf_esb_suspend) refers to nrf_esb.o(.data) for m_nrf_esb_mainstate
    nrf_esb.o(i.nrf_esb_update_prefix) refers to nrf_esb.o(i.update_radio_addresses) for update_radio_addresses
    nrf_esb.o(i.nrf_esb_update_prefix) refers to nrf_esb.o(i.apply_address_workarounds) for apply_address_workarounds
    nrf_esb.o(i.nrf_esb_update_prefix) refers to nrf_esb.o(.data) for m_nrf_esb_mainstate
    nrf_esb.o(i.nrf_esb_write_payload) refers to nrf_esb.o(i.NVIC_DisableIRQ) for NVIC_DisableIRQ
    nrf_esb.o(i.nrf_esb_write_payload) refers to memcpya.o(.text) for __aeabi_memcpy
    nrf_esb.o(i.nrf_esb_write_payload) refers to nrf_esb.o(i.NVIC_EnableIRQ) for NVIC_EnableIRQ
    nrf_esb.o(i.nrf_esb_write_payload) refers to nrf_esb.o(i.start_tx_transaction) for start_tx_transaction
    nrf_esb.o(i.nrf_esb_write_payload) refers to nrf_esb.o(.data) for m_esb_initialized
    nrf_esb.o(i.nrf_esb_write_payload) refers to nrf_esb.o(.bss) for m_config_local
    nrf_esb.o(i.on_radio_disabled_rx) refers to nrf_esb.o(i.clear_events_restart_rx) for clear_events_restart_rx
    nrf_esb.o(i.on_radio_disabled_rx) refers to memcpya.o(.text) for __aeabi_memcpy
    nrf_esb.o(i.on_radio_disabled_rx) refers to nrf_esb.o(i.rx_fifo_push_rfbuf) for rx_fifo_push_rfbuf
    nrf_esb.o(i.on_radio_disabled_rx) refers to nrf_esb.o(i.NVIC_SetPendingIRQ) for NVIC_SetPendingIRQ
    nrf_esb.o(i.on_radio_disabled_rx) refers to nrf_esb.o(.bss) for m_rx_fifo
    nrf_esb.o(i.on_radio_disabled_rx) refers to nrf_esb.o(.data) for m_radio_shorts_common
    nrf_esb.o(i.on_radio_disabled_rx) refers to nrf_esb.o(i.on_radio_disabled_rx_ack) for on_radio_disabled_rx_ack
    nrf_esb.o(i.on_radio_disabled_rx_ack) refers to nrf_esb.o(.data) for m_radio_shorts_common
    nrf_esb.o(i.on_radio_disabled_rx_ack) refers to nrf_esb.o(.bss) for m_config_local
    nrf_esb.o(i.on_radio_disabled_rx_ack) refers to nrf_esb.o(i.on_radio_disabled_rx) for on_radio_disabled_rx
    nrf_esb.o(i.on_radio_disabled_tx) refers to nrf_esb.o(.data) for m_radio_shorts_common
    nrf_esb.o(i.on_radio_disabled_tx) refers to nrf_esb.o(.bss) for m_config_local
    nrf_esb.o(i.on_radio_disabled_tx) refers to nrf_esb.o(i.on_radio_disabled_tx_wait_for_ack) for on_radio_disabled_tx_wait_for_ack
    nrf_esb.o(i.on_radio_disabled_tx_noack) refers to nrf_esb.o(i.nrf_esb_skip_tx) for nrf_esb_skip_tx
    nrf_esb.o(i.on_radio_disabled_tx_noack) refers to nrf_esb.o(i.NVIC_SetPendingIRQ) for NVIC_SetPendingIRQ
    nrf_esb.o(i.on_radio_disabled_tx_noack) refers to nrf_esb.o(i.start_tx_transaction) for start_tx_transaction
    nrf_esb.o(i.on_radio_disabled_tx_noack) refers to nrf_esb.o(.data) for m_interrupt_flags
    nrf_esb.o(i.on_radio_disabled_tx_noack) refers to nrf_esb.o(.bss) for m_tx_fifo
    nrf_esb.o(i.on_radio_disabled_tx_wait_for_ack) refers to nrf_esb.o(i.nrf_esb_skip_tx) for nrf_esb_skip_tx
    nrf_esb.o(i.on_radio_disabled_tx_wait_for_ack) refers to nrf_esb.o(i.rx_fifo_push_rfbuf) for rx_fifo_push_rfbuf
    nrf_esb.o(i.on_radio_disabled_tx_wait_for_ack) refers to nrf_esb.o(i.NVIC_SetPendingIRQ) for NVIC_SetPendingIRQ
    nrf_esb.o(i.on_radio_disabled_tx_wait_for_ack) refers to nrf_esb.o(i.start_tx_transaction) for start_tx_transaction
    nrf_esb.o(i.on_radio_disabled_tx_wait_for_ack) refers to nrf_esb.o(.data) for m_interrupt_flags
    nrf_esb.o(i.on_radio_disabled_tx_wait_for_ack) refers to nrf_esb.o(.bss) for m_config_local
    nrf_esb.o(i.on_radio_disabled_tx_wait_for_ack) refers to nrf_esb.o(i.on_radio_disabled_tx) for on_radio_disabled_tx
    nrf_esb.o(i.reset_fifos) refers to nrf_esb.o(.bss) for m_tx_fifo
    nrf_esb.o(i.rx_fifo_push_rfbuf) refers to memcpya.o(.text) for __aeabi_memcpy
    nrf_esb.o(i.rx_fifo_push_rfbuf) refers to nrf_esb.o(.bss) for m_rx_fifo
    nrf_esb.o(i.start_tx_transaction) refers to memcpya.o(.text) for __aeabi_memcpy
    nrf_esb.o(i.start_tx_transaction) refers to nrf_esb.o(i.NVIC_ClearPendingIRQ) for NVIC_ClearPendingIRQ
    nrf_esb.o(i.start_tx_transaction) refers to nrf_esb.o(i.NVIC_EnableIRQ) for NVIC_EnableIRQ
    nrf_esb.o(i.start_tx_transaction) refers to nrf_esb.o(.data) for m_last_tx_attempts
    nrf_esb.o(i.start_tx_transaction) refers to nrf_esb.o(.bss) for m_tx_fifo
    nrf_esb.o(i.start_tx_transaction) refers to nrf_esb.o(i.on_radio_disabled_tx) for on_radio_disabled_tx
    nrf_esb.o(i.start_tx_transaction) refers to nrf_esb.o(i.on_radio_disabled_tx_noack) for on_radio_disabled_tx_noack
    nrf_esb.o(i.update_radio_addresses) refers to nrf_esb.o(i.addr_conv) for addr_conv
    nrf_esb.o(i.update_radio_addresses) refers to nrf_esb.o(i.bytewise_bit_swap) for bytewise_bit_swap
    nrf_esb.o(i.update_radio_addresses) refers to nrf_esb.o(.data) for m_esb_addr
    nrf_esb.o(i.update_radio_bitrate) refers to nrf_esb.o(.bss) for m_config_local
    nrf_esb.o(i.update_radio_bitrate) refers to nrf_esb.o(.data) for m_wait_for_ack_timeout_us
    nrf_esb.o(i.update_radio_crc) refers to nrf_esb.o(.bss) for m_config_local
    nrf_esb.o(i.update_radio_parameters) refers to nrf_esb.o(i.update_radio_tx_power) for update_radio_tx_power
    nrf_esb.o(i.update_radio_parameters) refers to nrf_esb.o(i.update_radio_bitrate) for update_radio_bitrate
    nrf_esb.o(i.update_radio_parameters) refers to nrf_esb.o(i.update_radio_protocol) for update_radio_protocol
    nrf_esb.o(i.update_radio_parameters) refers to nrf_esb.o(i.update_radio_crc) for update_radio_crc
    nrf_esb.o(i.update_radio_parameters) refers to nrf_esb.o(.bss) for m_config_local
    nrf_esb.o(i.update_radio_parameters) refers to nrf_esb.o(.data) for update_rf_payload_format
    nrf_esb.o(i.update_radio_protocol) refers to nrf_esb.o(.bss) for m_config_local
    nrf_esb.o(i.update_radio_protocol) refers to nrf_esb.o(i.update_rf_payload_format_esb_dpl) for update_rf_payload_format_esb_dpl
    nrf_esb.o(i.update_radio_protocol) refers to nrf_esb.o(.data) for update_rf_payload_format
    nrf_esb.o(i.update_radio_protocol) refers to nrf_esb.o(i.update_rf_payload_format_esb) for update_rf_payload_format_esb
    nrf_esb.o(i.update_radio_tx_power) refers to nrf_esb.o(.bss) for m_config_local
    nrf_esb.o(i.update_rf_payload_format_esb) refers to nrf_esb.o(.data) for m_esb_addr
    nrf_esb.o(i.update_rf_payload_format_esb_dpl) refers to nrf_esb.o(.data) for m_esb_addr
    uartprocess.o(i.UART_Init) refers to memcpya.o(.text) for __aeabi_memcpy4
    uartprocess.o(i.UART_Init) refers to app_uart_fifo.o(i.app_uart_init) for app_uart_init
    uartprocess.o(i.UART_Init) refers to app_error.o(i.app_error_handler_bare) for app_error_handler_bare
    uartprocess.o(i.UART_Init) refers to uartprocess.o(.constdata) for .constdata
    uartprocess.o(i.UART_Init) refers to uartprocess.o(.bss) for rx_buf
    uartprocess.o(i.UART_Init) refers to uartprocess.o(i.uart_event_handle) for uart_event_handle
    uartprocess.o(i.uart_event_handle) refers to app_uart_fifo.o(i.app_uart_get) for app_uart_get
    uartprocess.o(i.uart_event_handle) refers to memcmp.o(.text) for memcmp
    uartprocess.o(i.uart_event_handle) refers to printf1.o(i.__0printf$1) for __2printf
    uartprocess.o(i.uart_event_handle) refers to app_error.o(i.app_error_handler_bare) for app_error_handler_bare
    uartprocess.o(i.uart_event_handle) refers to uartprocess.o(.bss) for data_array
    uartprocess.o(i.uart_event_handle) refers to uartprocess.o(.data) for index
    uartprocess.o(i.uart_event_handle) refers to uartprocess.o(.constdata) for delay_machine_code
    arm_startup_nrf52.o(RESET) refers to arm_startup_nrf52.o(STACK) for __initial_sp
    arm_startup_nrf52.o(RESET) refers to arm_startup_nrf52.o(.text) for Reset_Handler
    arm_startup_nrf52.o(RESET) refers to nrf_esb.o(i.RADIO_IRQHandler) for RADIO_IRQHandler
    arm_startup_nrf52.o(RESET) refers to nrfx_prs.o(i.UARTE0_UART0_IRQHandler) for UARTE0_UART0_IRQHandler
    arm_startup_nrf52.o(RESET) refers to nrfx_gpiote.o(i.GPIOTE_IRQHandler) for GPIOTE_IRQHandler
    arm_startup_nrf52.o(RESET) refers to app_timer.o(i.RTC1_IRQHandler) for RTC1_IRQHandler
    arm_startup_nrf52.o(RESET) refers to nrf_esb.o(i.SWI0_EGU0_IRQHandler) for SWI0_EGU0_IRQHandler
    arm_startup_nrf52.o(RESET) refers to app_timer.o(i.SWI1_EGU1_IRQHandler) for SWI1_EGU1_IRQHandler
    arm_startup_nrf52.o(RESET) refers to nrf_esb.o(i.TIMER3_IRQHandler) for TIMER3_IRQHandler
    arm_startup_nrf52.o(.text) refers to system_nrf52.o(i.SystemInit) for SystemInit
    arm_startup_nrf52.o(.text) refers to entry.o(.ARM.Collect$$$$00000000) for __main
    system_nrf52.o(i.SystemCoreClockUpdate) refers to system_nrf52.o(.data) for SystemCoreClock
    system_nrf52.o(i.SystemInit) refers to system_nrf52.o(i.errata_12) for errata_12
    system_nrf52.o(i.SystemInit) refers to system_nrf52.o(i.errata_16) for errata_16
    system_nrf52.o(i.SystemInit) refers to system_nrf52.o(i.errata_31) for errata_31
    system_nrf52.o(i.SystemInit) refers to system_nrf52.o(i.errata_32) for errata_32
    system_nrf52.o(i.SystemInit) refers to system_nrf52.o(i.errata_36) for errata_36
    system_nrf52.o(i.SystemInit) refers to system_nrf52.o(i.errata_37) for errata_37
    system_nrf52.o(i.SystemInit) refers to system_nrf52.o(i.errata_57) for errata_57
    system_nrf52.o(i.SystemInit) refers to system_nrf52.o(i.errata_66) for errata_66
    system_nrf52.o(i.SystemInit) refers to system_nrf52.o(i.errata_108) for errata_108
    system_nrf52.o(i.SystemInit) refers to system_nrf52.o(i.errata_136) for errata_136
    system_nrf52.o(i.SystemInit) refers to system_nrf52.o(i.errata_182) for errata_182
    system_nrf52.o(i.SystemInit) refers to system_nrf52.o(i.SystemCoreClockUpdate) for SystemCoreClockUpdate
    entry.o(.ARM.Collect$$$$00000000) refers (Special) to entry10a.o(.ARM.Collect$$$$0000000D) for __rt_final_cpp
    entry.o(.ARM.Collect$$$$00000000) refers (Special) to entry11a.o(.ARM.Collect$$$$0000000F) for __rt_final_exit
    entry.o(.ARM.Collect$$$$00000000) refers (Special) to entry7b.o(.ARM.Collect$$$$00000008) for _main_clock
    entry.o(.ARM.Collect$$$$00000000) refers (Special) to entry8b.o(.ARM.Collect$$$$0000000A) for _main_cpp_init
    entry.o(.ARM.Collect$$$$00000000) refers (Special) to entry9a.o(.ARM.Collect$$$$0000000B) for _main_init
    entry.o(.ARM.Collect$$$$00000000) refers (Special) to entry5.o(.ARM.Collect$$$$00000004) for _main_scatterload
    entry.o(.ARM.Collect$$$$00000000) refers (Special) to entry2.o(.ARM.Collect$$$$00000001) for _main_stk
    printfb.o(i.__0fprintf$bare) refers to printfb.o(i._printf_core) for _printf_core
    printfb.o(i.__0fprintf$bare) refers to retarget.o(i.fputc) for fputc
    printfb.o(i.__0printf$bare) refers to printfb.o(i._printf_core) for _printf_core
    printfb.o(i.__0printf$bare) refers to retarget.o(i.fputc) for fputc
    printfb.o(i.__0printf$bare) refers to retarget.o(.data) for __stdout
    printfb.o(i.__0snprintf$bare) refers to printfb.o(i._printf_core) for _printf_core
    printfb.o(i.__0snprintf$bare) refers to printfb.o(i._snputc) for _snputc
    printfb.o(i.__0sprintf$bare) refers to printfb.o(i._printf_core) for _printf_core
    printfb.o(i.__0sprintf$bare) refers to printfb.o(i._sputc) for _sputc
    printfb.o(i.__0vfprintf$bare) refers to printfb.o(i._printf_core) for _printf_core
    printfb.o(i.__0vfprintf$bare) refers to retarget.o(i.fputc) for fputc
    printfb.o(i.__0vprintf$bare) refers to printfb.o(i._printf_core) for _printf_core
    printfb.o(i.__0vprintf$bare) refers to retarget.o(i.fputc) for fputc
    printfb.o(i.__0vprintf$bare) refers to retarget.o(.data) for __stdout
    printfb.o(i.__0vsnprintf$bare) refers to printfb.o(i._printf_core) for _printf_core
    printfb.o(i.__0vsnprintf$bare) refers to printfb.o(i._snputc) for _snputc
    printfb.o(i.__0vsprintf$bare) refers to printfb.o(i._printf_core) for _printf_core
    printfb.o(i.__0vsprintf$bare) refers to printfb.o(i._sputc) for _sputc
    printf0.o(i.__0fprintf$0) refers to printf0.o(i._printf_core) for _printf_core
    printf0.o(i.__0fprintf$0) refers to retarget.o(i.fputc) for fputc
    printf0.o(i.__0printf$0) refers to printf0.o(i._printf_core) for _printf_core
    printf0.o(i.__0printf$0) refers to retarget.o(i.fputc) for fputc
    printf0.o(i.__0printf$0) refers to retarget.o(.data) for __stdout
    printf0.o(i.__0snprintf$0) refers to printf0.o(i._printf_core) for _printf_core
    printf0.o(i.__0snprintf$0) refers to printf0.o(i._snputc) for _snputc
    printf0.o(i.__0sprintf$0) refers to printf0.o(i._printf_core) for _printf_core
    printf0.o(i.__0sprintf$0) refers to printf0.o(i._sputc) for _sputc
    printf0.o(i.__0vfprintf$0) refers to printf0.o(i._printf_core) for _printf_core
    printf0.o(i.__0vfprintf$0) refers to retarget.o(i.fputc) for fputc
    printf0.o(i.__0vprintf$0) refers to printf0.o(i._printf_core) for _printf_core
    printf0.o(i.__0vprintf$0) refers to retarget.o(i.fputc) for fputc
    printf0.o(i.__0vprintf$0) refers to retarget.o(.data) for __stdout
    printf0.o(i.__0vsnprintf$0) refers to printf0.o(i._printf_core) for _printf_core
    printf0.o(i.__0vsnprintf$0) refers to printf0.o(i._snputc) for _snputc
    printf0.o(i.__0vsprintf$0) refers to printf0.o(i._printf_core) for _printf_core
    printf0.o(i.__0vsprintf$0) refers to printf0.o(i._sputc) for _sputc
    printf1.o(i.__0fprintf$1) refers to printf1.o(i._printf_core) for _printf_core
    printf1.o(i.__0fprintf$1) refers to retarget.o(i.fputc) for fputc
    printf1.o(i.__0printf$1) refers to printf1.o(i._printf_core) for _printf_core
    printf1.o(i.__0printf$1) refers to retarget.o(i.fputc) for fputc
    printf1.o(i.__0printf$1) refers to retarget.o(.data) for __stdout
    printf1.o(i.__0snprintf$1) refers to printf1.o(i._printf_core) for _printf_core
    printf1.o(i.__0snprintf$1) refers to printf1.o(i._snputc) for _snputc
    printf1.o(i.__0sprintf$1) refers to printf1.o(i._printf_core) for _printf_core
    printf1.o(i.__0sprintf$1) refers to printf1.o(i._sputc) for _sputc
    printf1.o(i.__0vfprintf$1) refers to printf1.o(i._printf_core) for _printf_core
    printf1.o(i.__0vfprintf$1) refers to retarget.o(i.fputc) for fputc
    printf1.o(i.__0vprintf$1) refers to printf1.o(i._printf_core) for _printf_core
    printf1.o(i.__0vprintf$1) refers to retarget.o(i.fputc) for fputc
    printf1.o(i.__0vprintf$1) refers to retarget.o(.data) for __stdout
    printf1.o(i.__0vsnprintf$1) refers to printf1.o(i._printf_core) for _printf_core
    printf1.o(i.__0vsnprintf$1) refers to printf1.o(i._snputc) for _snputc
    printf1.o(i.__0vsprintf$1) refers to printf1.o(i._printf_core) for _printf_core
    printf1.o(i.__0vsprintf$1) refers to printf1.o(i._sputc) for _sputc
    printf1.o(i._printf_core) refers to uidiv.o(.text) for __aeabi_uidivmod
    printf2.o(i.__0fprintf$2) refers to printf2.o(i._printf_core) for _printf_core
    printf2.o(i.__0fprintf$2) refers to retarget.o(i.fputc) for fputc
    printf2.o(i.__0printf$2) refers to printf2.o(i._printf_core) for _printf_core
    printf2.o(i.__0printf$2) refers to retarget.o(i.fputc) for fputc
    printf2.o(i.__0printf$2) refers to retarget.o(.data) for __stdout
    printf2.o(i.__0snprintf$2) refers to printf2.o(i._printf_core) for _printf_core
    printf2.o(i.__0snprintf$2) refers to printf2.o(i._snputc) for _snputc
    printf2.o(i.__0sprintf$2) refers to printf2.o(i._printf_core) for _printf_core
    printf2.o(i.__0sprintf$2) refers to printf2.o(i._sputc) for _sputc
    printf2.o(i.__0vfprintf$2) refers to printf2.o(i._printf_core) for _printf_core
    printf2.o(i.__0vfprintf$2) refers to retarget.o(i.fputc) for fputc
    printf2.o(i.__0vprintf$2) refers to printf2.o(i._printf_core) for _printf_core
    printf2.o(i.__0vprintf$2) refers to retarget.o(i.fputc) for fputc
    printf2.o(i.__0vprintf$2) refers to retarget.o(.data) for __stdout
    printf2.o(i.__0vsnprintf$2) refers to printf2.o(i._printf_core) for _printf_core
    printf2.o(i.__0vsnprintf$2) refers to printf2.o(i._snputc) for _snputc
    printf2.o(i.__0vsprintf$2) refers to printf2.o(i._printf_core) for _printf_core
    printf2.o(i.__0vsprintf$2) refers to printf2.o(i._sputc) for _sputc
    printf3.o(i.__0fprintf$3) refers to printf3.o(i._printf_core) for _printf_core
    printf3.o(i.__0fprintf$3) refers to retarget.o(i.fputc) for fputc
    printf3.o(i.__0printf$3) refers to printf3.o(i._printf_core) for _printf_core
    printf3.o(i.__0printf$3) refers to retarget.o(i.fputc) for fputc
    printf3.o(i.__0printf$3) refers to retarget.o(.data) for __stdout
    printf3.o(i.__0snprintf$3) refers to printf3.o(i._printf_core) for _printf_core
    printf3.o(i.__0snprintf$3) refers to printf3.o(i._snputc) for _snputc
    printf3.o(i.__0sprintf$3) refers to printf3.o(i._printf_core) for _printf_core
    printf3.o(i.__0sprintf$3) refers to printf3.o(i._sputc) for _sputc
    printf3.o(i.__0vfprintf$3) refers to printf3.o(i._printf_core) for _printf_core
    printf3.o(i.__0vfprintf$3) refers to retarget.o(i.fputc) for fputc
    printf3.o(i.__0vprintf$3) refers to printf3.o(i._printf_core) for _printf_core
    printf3.o(i.__0vprintf$3) refers to retarget.o(i.fputc) for fputc
    printf3.o(i.__0vprintf$3) refers to retarget.o(.data) for __stdout
    printf3.o(i.__0vsnprintf$3) refers to printf3.o(i._printf_core) for _printf_core
    printf3.o(i.__0vsnprintf$3) refers to printf3.o(i._snputc) for _snputc
    printf3.o(i.__0vsprintf$3) refers to printf3.o(i._printf_core) for _printf_core
    printf3.o(i.__0vsprintf$3) refers to printf3.o(i._sputc) for _sputc
    printf3.o(i._printf_core) refers to uidiv.o(.text) for __aeabi_uidivmod
    printf4.o(i.__0fprintf$4) refers to printf4.o(i._printf_core) for _printf_core
    printf4.o(i.__0fprintf$4) refers to retarget.o(i.fputc) for fputc
    printf4.o(i.__0printf$4) refers to printf4.o(i._printf_core) for _printf_core
    printf4.o(i.__0printf$4) refers to retarget.o(i.fputc) for fputc
    printf4.o(i.__0printf$4) refers to retarget.o(.data) for __stdout
    printf4.o(i.__0snprintf$4) refers to printf4.o(i._printf_core) for _printf_core
    printf4.o(i.__0snprintf$4) refers to printf4.o(i._snputc) for _snputc
    printf4.o(i.__0sprintf$4) refers to printf4.o(i._printf_core) for _printf_core
    printf4.o(i.__0sprintf$4) refers to printf4.o(i._sputc) for _sputc
    printf4.o(i.__0vfprintf$4) refers to printf4.o(i._printf_core) for _printf_core
    printf4.o(i.__0vfprintf$4) refers to retarget.o(i.fputc) for fputc
    printf4.o(i.__0vprintf$4) refers to printf4.o(i._printf_core) for _printf_core
    printf4.o(i.__0vprintf$4) refers to retarget.o(i.fputc) for fputc
    printf4.o(i.__0vprintf$4) refers to retarget.o(.data) for __stdout
    printf4.o(i.__0vsnprintf$4) refers to printf4.o(i._printf_core) for _printf_core
    printf4.o(i.__0vsnprintf$4) refers to printf4.o(i._snputc) for _snputc
    printf4.o(i.__0vsprintf$4) refers to printf4.o(i._printf_core) for _printf_core
    printf4.o(i.__0vsprintf$4) refers to printf4.o(i._sputc) for _sputc
    printf4.o(i._printf_core) refers to uldiv.o(.text) for __aeabi_uldivmod
    printf5.o(i.__0fprintf$5) refers to printf5.o(i._printf_core) for _printf_core
    printf5.o(i.__0fprintf$5) refers to retarget.o(i.fputc) for fputc
    printf5.o(i.__0printf$5) refers to printf5.o(i._printf_core) for _printf_core
    printf5.o(i.__0printf$5) refers to retarget.o(i.fputc) for fputc
    printf5.o(i.__0printf$5) refers to retarget.o(.data) for __stdout
    printf5.o(i.__0snprintf$5) refers to printf5.o(i._printf_core) for _printf_core
    printf5.o(i.__0snprintf$5) refers to printf5.o(i._snputc) for _snputc
    printf5.o(i.__0sprintf$5) refers to printf5.o(i._printf_core) for _printf_core
    printf5.o(i.__0sprintf$5) refers to printf5.o(i._sputc) for _sputc
    printf5.o(i.__0vfprintf$5) refers to printf5.o(i._printf_core) for _printf_core
    printf5.o(i.__0vfprintf$5) refers to retarget.o(i.fputc) for fputc
    printf5.o(i.__0vprintf$5) refers to printf5.o(i._printf_core) for _printf_core
    printf5.o(i.__0vprintf$5) refers to retarget.o(i.fputc) for fputc
    printf5.o(i.__0vprintf$5) refers to retarget.o(.data) for __stdout
    printf5.o(i.__0vsnprintf$5) refers to printf5.o(i._printf_core) for _printf_core
    printf5.o(i.__0vsnprintf$5) refers to printf5.o(i._snputc) for _snputc
    printf5.o(i.__0vsprintf$5) refers to printf5.o(i._printf_core) for _printf_core
    printf5.o(i.__0vsprintf$5) refers to printf5.o(i._sputc) for _sputc
    printf5.o(i._printf_core) refers to uldiv.o(.text) for __aeabi_uldivmod
    printf6.o(i.__0fprintf$6) refers to printf6.o(i._printf_core) for _printf_core
    printf6.o(i.__0fprintf$6) refers to retarget.o(i.fputc) for fputc
    printf6.o(i.__0printf$6) refers to printf6.o(i._printf_core) for _printf_core
    printf6.o(i.__0printf$6) refers to retarget.o(i.fputc) for fputc
    printf6.o(i.__0printf$6) refers to retarget.o(.data) for __stdout
    printf6.o(i.__0snprintf$6) refers to printf6.o(i._printf_core) for _printf_core
    printf6.o(i.__0snprintf$6) refers to printf6.o(i._snputc) for _snputc
    printf6.o(i.__0sprintf$6) refers to printf6.o(i._printf_core) for _printf_core
    printf6.o(i.__0sprintf$6) refers to printf6.o(i._sputc) for _sputc
    printf6.o(i.__0vfprintf$6) refers to printf6.o(i._printf_core) for _printf_core
    printf6.o(i.__0vfprintf$6) refers to retarget.o(i.fputc) for fputc
    printf6.o(i.__0vprintf$6) refers to printf6.o(i._printf_core) for _printf_core
    printf6.o(i.__0vprintf$6) refers to retarget.o(i.fputc) for fputc
    printf6.o(i.__0vprintf$6) refers to retarget.o(.data) for __stdout
    printf6.o(i.__0vsnprintf$6) refers to printf6.o(i._printf_core) for _printf_core
    printf6.o(i.__0vsnprintf$6) refers to printf6.o(i._snputc) for _snputc
    printf6.o(i.__0vsprintf$6) refers to printf6.o(i._printf_core) for _printf_core
    printf6.o(i.__0vsprintf$6) refers to printf6.o(i._sputc) for _sputc
    printf6.o(i._printf_core) refers to printf6.o(i._printf_pre_padding) for _printf_pre_padding
    printf6.o(i._printf_core) refers to uidiv.o(.text) for __aeabi_uidivmod
    printf6.o(i._printf_core) refers to printf6.o(i._printf_post_padding) for _printf_post_padding
    printf7.o(i.__0fprintf$7) refers to printf7.o(i._printf_core) for _printf_core
    printf7.o(i.__0fprintf$7) refers to retarget.o(i.fputc) for fputc
    printf7.o(i.__0printf$7) refers to printf7.o(i._printf_core) for _printf_core
    printf7.o(i.__0printf$7) refers to retarget.o(i.fputc) for fputc
    printf7.o(i.__0printf$7) refers to retarget.o(.data) for __stdout
    printf7.o(i.__0snprintf$7) refers to printf7.o(i._printf_core) for _printf_core
    printf7.o(i.__0snprintf$7) refers to printf7.o(i._snputc) for _snputc
    printf7.o(i.__0sprintf$7) refers to printf7.o(i._printf_core) for _printf_core
    printf7.o(i.__0sprintf$7) refers to printf7.o(i._sputc) for _sputc
    printf7.o(i.__0vfprintf$7) refers to printf7.o(i._printf_core) for _printf_core
    printf7.o(i.__0vfprintf$7) refers to retarget.o(i.fputc) for fputc
    printf7.o(i.__0vprintf$7) refers to printf7.o(i._printf_core) for _printf_core
    printf7.o(i.__0vprintf$7) refers to retarget.o(i.fputc) for fputc
    printf7.o(i.__0vprintf$7) refers to retarget.o(.data) for __stdout
    printf7.o(i.__0vsnprintf$7) refers to printf7.o(i._printf_core) for _printf_core
    printf7.o(i.__0vsnprintf$7) refers to printf7.o(i._snputc) for _snputc
    printf7.o(i.__0vsprintf$7) refers to printf7.o(i._printf_core) for _printf_core
    printf7.o(i.__0vsprintf$7) refers to printf7.o(i._sputc) for _sputc
    printf7.o(i._printf_core) refers to printf7.o(i._printf_pre_padding) for _printf_pre_padding
    printf7.o(i._printf_core) refers to uldiv.o(.text) for __aeabi_uldivmod
    printf7.o(i._printf_core) refers to printf7.o(i._printf_post_padding) for _printf_post_padding
    printf8.o(i.__0fprintf$8) refers to printf8.o(i._printf_core) for _printf_core
    printf8.o(i.__0fprintf$8) refers to retarget.o(i.fputc) for fputc
    printf8.o(i.__0printf$8) refers to printf8.o(i._printf_core) for _printf_core
    printf8.o(i.__0printf$8) refers to retarget.o(i.fputc) for fputc
    printf8.o(i.__0printf$8) refers to retarget.o(.data) for __stdout
    printf8.o(i.__0snprintf$8) refers to printf8.o(i._printf_core) for _printf_core
    printf8.o(i.__0snprintf$8) refers to printf8.o(i._snputc) for _snputc
    printf8.o(i.__0sprintf$8) refers to printf8.o(i._printf_core) for _printf_core
    printf8.o(i.__0sprintf$8) refers to printf8.o(i._sputc) for _sputc
    printf8.o(i.__0vfprintf$8) refers to printf8.o(i._printf_core) for _printf_core
    printf8.o(i.__0vfprintf$8) refers to retarget.o(i.fputc) for fputc
    printf8.o(i.__0vprintf$8) refers to printf8.o(i._printf_core) for _printf_core
    printf8.o(i.__0vprintf$8) refers to retarget.o(i.fputc) for fputc
    printf8.o(i.__0vprintf$8) refers to retarget.o(.data) for __stdout
    printf8.o(i.__0vsnprintf$8) refers to printf8.o(i._printf_core) for _printf_core
    printf8.o(i.__0vsnprintf$8) refers to printf8.o(i._snputc) for _snputc
    printf8.o(i.__0vsprintf$8) refers to printf8.o(i._printf_core) for _printf_core
    printf8.o(i.__0vsprintf$8) refers to printf8.o(i._sputc) for _sputc
    printf8.o(i._printf_core) refers to printf8.o(i._printf_pre_padding) for _printf_pre_padding
    printf8.o(i._printf_core) refers to uldiv.o(.text) for __aeabi_uldivmod
    printf8.o(i._printf_core) refers to printf8.o(i._printf_post_padding) for _printf_post_padding
    printfa.o(i.__0fprintf) refers (Special) to iusefp.o(.text) for __I$use$fp
    printfa.o(i.__0fprintf) refers to printfa.o(i._printf_core) for _printf_core
    printfa.o(i.__0fprintf) refers to retarget.o(i.fputc) for fputc
    printfa.o(i.__0printf) refers (Special) to iusefp.o(.text) for __I$use$fp
    printfa.o(i.__0printf) refers to printfa.o(i._printf_core) for _printf_core
    printfa.o(i.__0printf) refers to retarget.o(i.fputc) for fputc
    printfa.o(i.__0printf) refers to retarget.o(.data) for __stdout
    printfa.o(i.__0snprintf) refers (Special) to iusefp.o(.text) for __I$use$fp
    printfa.o(i.__0snprintf) refers to printfa.o(i._printf_core) for _printf_core
    printfa.o(i.__0snprintf) refers to printfa.o(i._snputc) for _snputc
    printfa.o(i.__0sprintf) refers (Special) to iusefp.o(.text) for __I$use$fp
    printfa.o(i.__0sprintf) refers to printfa.o(i._printf_core) for _printf_core
    printfa.o(i.__0sprintf) refers to printfa.o(i._sputc) for _sputc
    printfa.o(i.__0vfprintf) refers (Special) to iusefp.o(.text) for __I$use$fp
    printfa.o(i.__0vfprintf) refers to printfa.o(i._printf_core) for _printf_core
    printfa.o(i.__0vfprintf) refers to retarget.o(i.fputc) for fputc
    printfa.o(i.__0vprintf) refers (Special) to iusefp.o(.text) for __I$use$fp
    printfa.o(i.__0vprintf) refers to printfa.o(i._printf_core) for _printf_core
    printfa.o(i.__0vprintf) refers to retarget.o(i.fputc) for fputc
    printfa.o(i.__0vprintf) refers to retarget.o(.data) for __stdout
    printfa.o(i.__0vsnprintf) refers (Special) to iusefp.o(.text) for __I$use$fp
    printfa.o(i.__0vsnprintf) refers to printfa.o(i._printf_core) for _printf_core
    printfa.o(i.__0vsnprintf) refers to printfa.o(i._snputc) for _snputc
    printfa.o(i.__0vsprintf) refers (Special) to iusefp.o(.text) for __I$use$fp
    printfa.o(i.__0vsprintf) refers to printfa.o(i._printf_core) for _printf_core
    printfa.o(i.__0vsprintf) refers to printfa.o(i._sputc) for _sputc
    printfa.o(i._fp_digits) refers (Special) to iusefp.o(.text) for __I$use$fp
    printfa.o(i._fp_digits) refers to dmul.o(.text) for __aeabi_dmul
    printfa.o(i._fp_digits) refers to ddiv.o(.text) for __aeabi_ddiv
    printfa.o(i._fp_digits) refers to cdrcmple.o(.text) for __aeabi_cdrcmple
    printfa.o(i._fp_digits) refers to dadd.o(.text) for __aeabi_dadd
    printfa.o(i._fp_digits) refers to dfixul.o(.text) for __aeabi_d2ulz
    printfa.o(i._fp_digits) refers to uldiv.o(.text) for __aeabi_uldivmod
    printfa.o(i._printf_core) refers (Special) to iusefp.o(.text) for __I$use$fp
    printfa.o(i._printf_core) refers to printfa.o(i._printf_pre_padding) for _printf_pre_padding
    printfa.o(i._printf_core) refers to uldiv.o(.text) for __aeabi_uldivmod
    printfa.o(i._printf_core) refers to printfa.o(i._printf_post_padding) for _printf_post_padding
    printfa.o(i._printf_core) refers to printfa.o(i._fp_digits) for _fp_digits
    printfa.o(i._printf_core) refers to uidiv.o(.text) for __aeabi_uidivmod
    printfa.o(i._printf_post_padding) refers (Special) to iusefp.o(.text) for __I$use$fp
    printfa.o(i._printf_pre_padding) refers (Special) to iusefp.o(.text) for __I$use$fp
    printfa.o(i._snputc) refers (Special) to iusefp.o(.text) for __I$use$fp
    printfa.o(i._sputc) refers (Special) to iusefp.o(.text) for __I$use$fp
    entry2.o(.ARM.Collect$$$$00000001) refers to entry2.o(.ARM.Collect$$$$00002712) for __lit__00000000
    entry2.o(.ARM.Collect$$$$00002712) refers to arm_startup_nrf52.o(STACK) for __initial_sp
    entry2.o(__vectab_stack_and_reset_area) refers to arm_startup_nrf52.o(STACK) for __initial_sp
    entry2.o(__vectab_stack_and_reset_area) refers to entry.o(.ARM.Collect$$$$00000000) for __main
    entry5.o(.ARM.Collect$$$$00000004) refers to init.o(.text) for __scatterload
    entry9a.o(.ARM.Collect$$$$0000000B) refers to host.o(i.main) for main
    entry9b.o(.ARM.Collect$$$$0000000C) refers to host.o(i.main) for main
    uldiv.o(.text) refers to llushr.o(.text) for __aeabi_llsr
    uldiv.o(.text) refers to llshl.o(.text) for __aeabi_llsl
    dadd.o(.text) refers to llshl.o(.text) for __aeabi_llsl
    dadd.o(.text) refers to llsshr.o(.text) for __aeabi_lasr
    dadd.o(.text) refers to depilogue.o(.text) for _double_epilogue
    dmul.o(.text) refers to depilogue.o(.text) for _double_epilogue
    ddiv.o(.text) refers to depilogue.o(.text) for _double_round
    dfixul.o(.text) refers to llushr.o(.text) for __aeabi_llsr
    dfixul.o(.text) refers to llshl.o(.text) for __aeabi_llsl
    init.o(.text) refers to entry5.o(.ARM.Collect$$$$00000004) for __main_after_scatterload
    depilogue.o(.text) refers to llshl.o(.text) for __aeabi_llsl
    depilogue.o(.text) refers to llushr.o(.text) for __aeabi_llsr


==============================================================================

Removing Unused input sections from the image.

    Removing gpioprocess.o(.rev16_text), (4 bytes).
    Removing gpioprocess.o(.revsh_text), (4 bytes).
    Removing gpioprocess.o(.rrx_text), (6 bytes).
    Removing host.o(.rev16_text), (4 bytes).
    Removing host.o(.revsh_text), (4 bytes).
    Removing host.o(.rrx_text), (6 bytes).
    Removing esbprocess.o(.rev16_text), (4 bytes).
    Removing esbprocess.o(.revsh_text), (4 bytes).
    Removing esbprocess.o(.rrx_text), (6 bytes).
    Removing boards.o(.rev16_text), (4 bytes).
    Removing boards.o(.revsh_text), (4 bytes).
    Removing boards.o(.rrx_text), (6 bytes).
    Removing boards.o(i.bsp_board_button_idx_to_pin), (12 bytes).
    Removing boards.o(i.bsp_board_button_state_get), (48 bytes).
    Removing boards.o(i.bsp_board_buttons_init), (44 bytes).
    Removing boards.o(i.bsp_board_init), (26 bytes).
    Removing boards.o(i.bsp_board_led_idx_to_pin), (12 bytes).
    Removing boards.o(i.bsp_board_led_invert), (48 bytes).
    Removing boards.o(i.bsp_board_led_off), (20 bytes).
    Removing boards.o(i.bsp_board_led_on), (20 bytes).
    Removing boards.o(i.bsp_board_led_state_get), (48 bytes).
    Removing boards.o(i.bsp_board_leds_init), (48 bytes).
    Removing boards.o(i.bsp_board_leds_off), (20 bytes).
    Removing boards.o(i.bsp_board_leds_on), (20 bytes).
    Removing boards.o(i.bsp_board_pin_to_button_idx), (36 bytes).
    Removing boards.o(i.bsp_board_pin_to_led_idx), (36 bytes).
    Removing boards.o(i.nrf_gpio_cfg), (40 bytes).
    Removing boards.o(i.nrf_gpio_pin_write), (58 bytes).
    Removing boards.o(.constdata), (8 bytes).
    Removing nrf_drv_uart.o(.rev16_text), (4 bytes).
    Removing nrf_drv_uart.o(.revsh_text), (4 bytes).
    Removing nrf_drv_uart.o(.rrx_text), (6 bytes).
    Removing nrfx_prs.o(.rev16_text), (4 bytes).
    Removing nrfx_prs.o(.revsh_text), (4 bytes).
    Removing nrfx_prs.o(.rrx_text), (6 bytes).
    Removing nrfx_prs.o(i.nrfx_prs_release), (22 bytes).
    Removing nrfx_prs.o(.constdata), (17 bytes).
    Removing nrfx_uart.o(.rev16_text), (4 bytes).
    Removing nrfx_uart.o(.revsh_text), (4 bytes).
    Removing nrfx_uart.o(.rrx_text), (6 bytes).
    Removing nrfx_uart.o(i.interrupts_disable), (52 bytes).
    Removing nrfx_uart.o(i.nrf_gpio_cfg_default), (24 bytes).
    Removing nrfx_uart.o(i.nrfx_uart_errorsrc_get), (22 bytes).
    Removing nrfx_uart.o(i.nrfx_uart_rx_abort), (24 bytes).
    Removing nrfx_uart.o(i.nrfx_uart_rx_disable), (40 bytes).
    Removing nrfx_uart.o(i.nrfx_uart_rx_enable), (60 bytes).
    Removing nrfx_uart.o(i.nrfx_uart_rx_ready), (16 bytes).
    Removing nrfx_uart.o(i.nrfx_uart_tx_abort), (52 bytes).
    Removing nrfx_uart.o(i.nrfx_uart_uninit), (68 bytes).
    Removing nrfx_uart.o(i.pins_to_default), (120 bytes).
    Removing nrfx_uarte.o(.rev16_text), (4 bytes).
    Removing nrfx_uarte.o(.revsh_text), (4 bytes).
    Removing nrfx_uarte.o(.rrx_text), (6 bytes).
    Removing nrfx_uarte.o(i.interrupts_disable), (52 bytes).
    Removing nrfx_uarte.o(i.nrf_gpio_cfg_default), (24 bytes).
    Removing nrfx_uarte.o(i.nrfx_uarte_errorsrc_get), (22 bytes).
    Removing nrfx_uarte.o(i.nrfx_uarte_rx_abort), (44 bytes).
    Removing nrfx_uarte.o(i.nrfx_uarte_rx_ready), (16 bytes).
    Removing nrfx_uarte.o(i.nrfx_uarte_tx_abort), (60 bytes).
    Removing nrfx_uarte.o(i.nrfx_uarte_uninit), (64 bytes).
    Removing nrfx_uarte.o(i.pins_to_default), (126 bytes).
    Removing nrfx_gpiote.o(.rev16_text), (4 bytes).
    Removing nrfx_gpiote.o(.revsh_text), (4 bytes).
    Removing nrfx_gpiote.o(.rrx_text), (6 bytes).
    Removing nrfx_gpiote.o(i.nrf_gpio_cfg_default), (24 bytes).
    Removing nrfx_gpiote.o(i.nrf_gpio_pin_clear), (22 bytes).
    Removing nrfx_gpiote.o(i.nrf_gpio_pin_set), (22 bytes).
    Removing nrfx_gpiote.o(i.nrf_gpiote_task_addr_get), (12 bytes).
    Removing nrfx_gpiote.o(i.nrf_gpiote_te_default), (16 bytes).
    Removing nrfx_gpiote.o(i.nrfx_gpiote_clr_task_addr_get), (24 bytes).
    Removing nrfx_gpiote.o(i.nrfx_gpiote_clr_task_trigger), (32 bytes).
    Removing nrfx_gpiote.o(i.nrfx_gpiote_in_event_addr_get), (38 bytes).
    Removing nrfx_gpiote.o(i.nrfx_gpiote_in_event_disable), (84 bytes).
    Removing nrfx_gpiote.o(i.nrfx_gpiote_in_is_set), (20 bytes).
    Removing nrfx_gpiote.o(i.nrfx_gpiote_in_uninit), (72 bytes).
    Removing nrfx_gpiote.o(i.nrfx_gpiote_is_init), (20 bytes).
    Removing nrfx_gpiote.o(i.nrfx_gpiote_out_clear), (12 bytes).
    Removing nrfx_gpiote.o(i.nrfx_gpiote_out_init), (208 bytes).
    Removing nrfx_gpiote.o(i.nrfx_gpiote_out_set), (12 bytes).
    Removing nrfx_gpiote.o(i.nrfx_gpiote_out_task_addr_get), (22 bytes).
    Removing nrfx_gpiote.o(i.nrfx_gpiote_out_task_disable), (36 bytes).
    Removing nrfx_gpiote.o(i.nrfx_gpiote_out_task_enable), (44 bytes).
    Removing nrfx_gpiote.o(i.nrfx_gpiote_out_task_force), (48 bytes).
    Removing nrfx_gpiote.o(i.nrfx_gpiote_out_task_trigger), (32 bytes).
    Removing nrfx_gpiote.o(i.nrfx_gpiote_out_toggle), (38 bytes).
    Removing nrfx_gpiote.o(i.nrfx_gpiote_out_uninit), (66 bytes).
    Removing nrfx_gpiote.o(i.nrfx_gpiote_set_task_addr_get), (24 bytes).
    Removing nrfx_gpiote.o(i.nrfx_gpiote_set_task_trigger), (32 bytes).
    Removing nrfx_gpiote.o(i.nrfx_gpiote_uninit), (68 bytes).
    Removing nrfx_gpiote.o(i.pin_configured_check), (28 bytes).
    Removing nrfx_gpiote.o(i.pin_configured_clear), (32 bytes).
    Removing app_error.o(.rev16_text), (4 bytes).
    Removing app_error.o(.revsh_text), (4 bytes).
    Removing app_error.o(.rrx_text), (6 bytes).
    Removing app_error.o(i.app_error_save_and_stop), (136 bytes).
    Removing app_error.o(.bss), (32 bytes).
    Removing app_error_handler_keil.o(.rev16_text), (4 bytes).
    Removing app_error_handler_keil.o(.revsh_text), (4 bytes).
    Removing app_error_handler_keil.o(.rrx_text), (6 bytes).
    Removing app_error_handler_keil.o(.emb_text), (26 bytes).
    Removing app_error_weak.o(.rev16_text), (4 bytes).
    Removing app_error_weak.o(.revsh_text), (4 bytes).
    Removing app_error_weak.o(.rrx_text), (6 bytes).
    Removing app_fifo.o(.rev16_text), (4 bytes).
    Removing app_fifo.o(.revsh_text), (4 bytes).
    Removing app_fifo.o(.rrx_text), (6 bytes).
    Removing app_fifo.o(i.app_fifo_flush), (10 bytes).
    Removing app_fifo.o(i.app_fifo_peek), (36 bytes).
    Removing app_fifo.o(i.app_fifo_read), (102 bytes).
    Removing app_fifo.o(i.app_fifo_write), (106 bytes).
    Removing app_uart_fifo.o(.rev16_text), (4 bytes).
    Removing app_uart_fifo.o(.revsh_text), (4 bytes).
    Removing app_uart_fifo.o(.rrx_text), (6 bytes).
    Removing app_uart_fifo.o(i.app_uart_close), (52 bytes).
    Removing app_uart_fifo.o(i.app_uart_flush), (52 bytes).
    Removing app_util_platform.o(.rev16_text), (4 bytes).
    Removing app_util_platform.o(.revsh_text), (4 bytes).
    Removing app_util_platform.o(.rrx_text), (6 bytes).
    Removing app_util_platform.o(i.current_int_priority_get), (60 bytes).
    Removing app_util_platform.o(i.privilege_level_get), (34 bytes).
    Removing nrf_assert.o(.rev16_text), (4 bytes).
    Removing nrf_assert.o(.revsh_text), (4 bytes).
    Removing nrf_assert.o(.rrx_text), (6 bytes).
    Removing nrf_assert.o(i.assert_nrf_callback), (26 bytes).
    Removing nrf_atomic.o(.rev16_text), (4 bytes).
    Removing nrf_atomic.o(.revsh_text), (4 bytes).
    Removing nrf_atomic.o(.rrx_text), (6 bytes).
    Removing nrf_atomic.o(.emb_text), (226 bytes).
    Removing nrf_atomic.o(i.nrf_atomic_flag_clear), (14 bytes).
    Removing nrf_atomic.o(i.nrf_atomic_flag_clear_fetch), (14 bytes).
    Removing nrf_atomic.o(i.nrf_atomic_flag_set), (14 bytes).
    Removing nrf_atomic.o(i.nrf_atomic_flag_set_fetch), (14 bytes).
    Removing nrf_atomic.o(i.nrf_atomic_u32_add), (22 bytes).
    Removing nrf_atomic.o(i.nrf_atomic_u32_and), (22 bytes).
    Removing nrf_atomic.o(i.nrf_atomic_u32_cmp_exch), (20 bytes).
    Removing nrf_atomic.o(i.nrf_atomic_u32_fetch_add), (22 bytes).
    Removing nrf_atomic.o(i.nrf_atomic_u32_fetch_and), (22 bytes).
    Removing nrf_atomic.o(i.nrf_atomic_u32_fetch_or), (22 bytes).
    Removing nrf_atomic.o(i.nrf_atomic_u32_fetch_store), (22 bytes).
    Removing nrf_atomic.o(i.nrf_atomic_u32_fetch_sub), (22 bytes).
    Removing nrf_atomic.o(i.nrf_atomic_u32_fetch_sub_hs), (22 bytes).
    Removing nrf_atomic.o(i.nrf_atomic_u32_fetch_xor), (22 bytes).
    Removing nrf_atomic.o(i.nrf_atomic_u32_or), (22 bytes).
    Removing nrf_atomic.o(i.nrf_atomic_u32_store), (22 bytes).
    Removing nrf_atomic.o(i.nrf_atomic_u32_sub), (22 bytes).
    Removing nrf_atomic.o(i.nrf_atomic_u32_sub_hs), (22 bytes).
    Removing nrf_atomic.o(i.nrf_atomic_u32_xor), (22 bytes).
    Removing nrf_balloc.o(.rev16_text), (4 bytes).
    Removing nrf_balloc.o(.revsh_text), (4 bytes).
    Removing nrf_balloc.o(.rrx_text), (6 bytes).
    Removing nrf_balloc.o(i.nrf_balloc_alloc), (76 bytes).
    Removing nrf_balloc.o(i.nrf_balloc_block2idx), (16 bytes).
    Removing nrf_balloc.o(i.nrf_balloc_free), (42 bytes).
    Removing nrf_balloc.o(i.nrf_balloc_idx2block), (12 bytes).
    Removing nrf_balloc.o(i.nrf_balloc_init), (60 bytes).
    Removing nrf_fprintf.o(.rev16_text), (4 bytes).
    Removing nrf_fprintf.o(.revsh_text), (4 bytes).
    Removing nrf_fprintf.o(.rrx_text), (6 bytes).
    Removing nrf_fprintf.o(i.nrf_fprintf), (42 bytes).
    Removing nrf_fprintf.o(i.nrf_fprintf_buffer_flush), (28 bytes).
    Removing nrf_fprintf_format.o(.rev16_text), (4 bytes).
    Removing nrf_fprintf_format.o(.revsh_text), (4 bytes).
    Removing nrf_fprintf_format.o(.rrx_text), (6 bytes).
    Removing nrf_fprintf_format.o(i.buffer_add), (32 bytes).
    Removing nrf_fprintf_format.o(i.int_print), (190 bytes).
    Removing nrf_fprintf_format.o(i.nrf_fprintf_fmt), (496 bytes).
    Removing nrf_fprintf_format.o(i.string_print), (116 bytes).
    Removing nrf_fprintf_format.o(i.unsigned_print), (184 bytes).
    Removing nrf_fprintf_format.o(.constdata), (16 bytes).
    Removing nrf_memobj.o(.rev16_text), (4 bytes).
    Removing nrf_memobj.o(.revsh_text), (4 bytes).
    Removing nrf_memobj.o(.rrx_text), (6 bytes).
    Removing nrf_memobj.o(i.memobj_op), (202 bytes).
    Removing nrf_memobj.o(i.nrf_memobj_alloc), (122 bytes).
    Removing nrf_memobj.o(i.nrf_memobj_free), (64 bytes).
    Removing nrf_memobj.o(i.nrf_memobj_get), (16 bytes).
    Removing nrf_memobj.o(i.nrf_memobj_pool_init), (12 bytes).
    Removing nrf_memobj.o(i.nrf_memobj_put), (30 bytes).
    Removing nrf_memobj.o(i.nrf_memobj_read), (34 bytes).
    Removing nrf_memobj.o(i.nrf_memobj_write), (34 bytes).
    Removing nrf_ringbuf.o(.rev16_text), (4 bytes).
    Removing nrf_ringbuf.o(.revsh_text), (4 bytes).
    Removing nrf_ringbuf.o(.rrx_text), (6 bytes).
    Removing nrf_ringbuf.o(i.nrf_ringbuf_alloc), (150 bytes).
    Removing nrf_ringbuf.o(i.nrf_ringbuf_cpy_get), (152 bytes).
    Removing nrf_ringbuf.o(i.nrf_ringbuf_cpy_put), (138 bytes).
    Removing nrf_ringbuf.o(i.nrf_ringbuf_free), (54 bytes).
    Removing nrf_ringbuf.o(i.nrf_ringbuf_get), (146 bytes).
    Removing nrf_ringbuf.o(i.nrf_ringbuf_init), (28 bytes).
    Removing nrf_ringbuf.o(i.nrf_ringbuf_put), (64 bytes).
    Removing nrf_strerror.o(.rev16_text), (4 bytes).
    Removing nrf_strerror.o(.revsh_text), (4 bytes).
    Removing nrf_strerror.o(.rrx_text), (6 bytes).
    Removing nrf_strerror.o(i.nrf_strerror_find), (64 bytes).
    Removing nrf_strerror.o(i.nrf_strerror_get), (28 bytes).
    Removing nrf_strerror.o(.constdata), (300 bytes).
    Removing nrf_strerror.o(.conststring), (957 bytes).
    Removing app_timer.o(.rev16_text), (4 bytes).
    Removing app_timer.o(.revsh_text), (4 bytes).
    Removing app_timer.o(.rrx_text), (6 bytes).
    Removing app_timer.o(i.app_timer_cnt_diff_compute), (16 bytes).
    Removing app_timer.o(i.app_timer_cnt_get), (8 bytes).
    Removing app_timer.o(i.app_timer_pause), (12 bytes).
    Removing app_timer.o(i.app_timer_resume), (12 bytes).
    Removing app_timer.o(i.app_timer_stop), (48 bytes).
    Removing app_timer.o(i.app_timer_stop_all), (32 bytes).
    Removing app_timer.o(i.timer_stop_op_schedule), (56 bytes).
    Removing retarget.o(.rev16_text), (4 bytes).
    Removing retarget.o(.revsh_text), (4 bytes).
    Removing retarget.o(.rrx_text), (6 bytes).
    Removing retarget.o(i.fgetc), (22 bytes).
    Removing nrf_log_frontend.o(.rev16_text), (4 bytes).
    Removing nrf_log_frontend.o(.revsh_text), (4 bytes).
    Removing nrf_log_frontend.o(.rrx_text), (6 bytes).
    Removing nrf_log_str_formatter.o(.rev16_text), (4 bytes).
    Removing nrf_log_str_formatter.o(.revsh_text), (4 bytes).
    Removing nrf_log_str_formatter.o(.rrx_text), (6 bytes).
    Removing nrf_esb.o(.rev16_text), (4 bytes).
    Removing nrf_esb.o(.revsh_text), (4 bytes).
    Removing nrf_esb.o(.rrx_text), (6 bytes).
    Removing nrf_esb.o(i.nrf_esb_enable_pipes), (52 bytes).
    Removing nrf_esb.o(i.nrf_esb_flush_rx), (64 bytes).
    Removing nrf_esb.o(i.nrf_esb_flush_tx), (52 bytes).
    Removing nrf_esb.o(i.nrf_esb_get_rf_channel), (28 bytes).
    Removing nrf_esb.o(i.nrf_esb_is_idle), (20 bytes).
    Removing nrf_esb.o(i.nrf_esb_pop_tx), (84 bytes).
    Removing nrf_esb.o(i.nrf_esb_reuse_pid), (64 bytes).
    Removing nrf_esb.o(i.nrf_esb_set_address_length), (248 bytes).
    Removing nrf_esb.o(i.nrf_esb_set_bitrate), (44 bytes).
    Removing nrf_esb.o(i.nrf_esb_set_retransmit_count), (32 bytes).
    Removing nrf_esb.o(i.nrf_esb_set_retransmit_delay), (44 bytes).
    Removing nrf_esb.o(i.nrf_esb_set_tx_power), (48 bytes).
    Removing nrf_esb.o(i.nrf_esb_suspend), (40 bytes).
    Removing nrf_esb.o(i.nrf_esb_update_prefix), (136 bytes).
    Removing uartprocess.o(.rev16_text), (4 bytes).
    Removing uartprocess.o(.revsh_text), (4 bytes).
    Removing uartprocess.o(.rrx_text), (6 bytes).
    Removing arm_startup_nrf52.o(HEAP), (8192 bytes).
    Removing system_nrf52.o(.rev16_text), (4 bytes).
    Removing system_nrf52.o(.revsh_text), (4 bytes).
    Removing system_nrf52.o(.rrx_text), (6 bytes).
    Removing dadd.o(.text), (334 bytes).
    Removing dmul.o(.text), (228 bytes).
    Removing ddiv.o(.text), (222 bytes).
    Removing dfixul.o(.text), (48 bytes).
    Removing cdrcmple.o(.text), (48 bytes).
    Removing depilogue.o(.text), (186 bytes).

247 unused section(s) (total 18584 bytes) removed from the image.

==============================================================================

Image Symbol Table

    Local Symbols

    Symbol Name                              Value     Ov Type        Size  Object(Section)

    RESET                                    0x00000000   Section      512  arm_startup_nrf52.o(RESET)
    ../clib/microlib/division.c              0x00000000   Number         0  uldiv.o ABSOLUTE
    ../clib/microlib/division.c              0x00000000   Number         0  uidiv.o ABSOLUTE
    ../clib/microlib/init/entry.s            0x00000000   Number         0  entry.o ABSOLUTE
    ../clib/microlib/init/entry.s            0x00000000   Number         0  entry9a.o ABSOLUTE
    ../clib/microlib/init/entry.s            0x00000000   Number         0  entry10a.o ABSOLUTE
    ../clib/microlib/init/entry.s            0x00000000   Number         0  entry10b.o ABSOLUTE
    ../clib/microlib/init/entry.s            0x00000000   Number         0  entry8b.o ABSOLUTE
    ../clib/microlib/init/entry.s            0x00000000   Number         0  entry11a.o ABSOLUTE
    ../clib/microlib/init/entry.s            0x00000000   Number         0  entry9b.o ABSOLUTE
    ../clib/microlib/init/entry.s            0x00000000   Number         0  entry2.o ABSOLUTE
    ../clib/microlib/init/entry.s            0x00000000   Number         0  entry5.o ABSOLUTE
    ../clib/microlib/init/entry.s            0x00000000   Number         0  entry7a.o ABSOLUTE
    ../clib/microlib/init/entry.s            0x00000000   Number         0  entry7b.o ABSOLUTE
    ../clib/microlib/init/entry.s            0x00000000   Number         0  entry8a.o ABSOLUTE
    ../clib/microlib/init/entry.s            0x00000000   Number         0  entry11b.o ABSOLUTE
    ../clib/microlib/longlong.c              0x00000000   Number         0  llsshr.o ABSOLUTE
    ../clib/microlib/longlong.c              0x00000000   Number         0  llushr.o ABSOLUTE
    ../clib/microlib/longlong.c              0x00000000   Number         0  llshl.o ABSOLUTE
    ../clib/microlib/printf/printf.c         0x00000000   Number         0  printf1.o ABSOLUTE
    ../clib/microlib/printf/printf.c         0x00000000   Number         0  printf0.o ABSOLUTE
    ../clib/microlib/printf/printf.c         0x00000000   Number         0  printfb.o ABSOLUTE
    ../clib/microlib/printf/printf.c         0x00000000   Number         0  printfa.o ABSOLUTE
    ../clib/microlib/printf/printf.c         0x00000000   Number         0  printf8.o ABSOLUTE
    ../clib/microlib/printf/printf.c         0x00000000   Number         0  printf7.o ABSOLUTE
    ../clib/microlib/printf/printf.c         0x00000000   Number         0  printf6.o ABSOLUTE
    ../clib/microlib/printf/printf.c         0x00000000   Number         0  printf4.o ABSOLUTE
    ../clib/microlib/printf/printf.c         0x00000000   Number         0  printf5.o ABSOLUTE
    ../clib/microlib/printf/printf.c         0x00000000   Number         0  printf3.o ABSOLUTE
    ../clib/microlib/printf/printf.c         0x00000000   Number         0  printf2.o ABSOLUTE
    ../clib/microlib/printf/stubs.s          0x00000000   Number         0  stubs.o ABSOLUTE
    ../clib/microlib/string/memcmp.c         0x00000000   Number         0  memcmp.o ABSOLUTE
    ../clib/microlib/string/memcpy.c         0x00000000   Number         0  memcpya.o ABSOLUTE
    ../clib/microlib/string/memcpy.c         0x00000000   Number         0  memcpyb.o ABSOLUTE
    ../clib/microlib/string/memset.c         0x00000000   Number         0  memseta.o ABSOLUTE
    ../clib/microlib/string/strlen.c         0x00000000   Number         0  strlen.o ABSOLUTE
    ../clib/microlib/stubs.s                 0x00000000   Number         0  iusefp.o ABSOLUTE
    ../fplib/microlib/fpadd.c                0x00000000   Number         0  dadd.o ABSOLUTE
    ../fplib/microlib/fpdiv.c                0x00000000   Number         0  ddiv.o ABSOLUTE
    ../fplib/microlib/fpepilogue.c           0x00000000   Number         0  depilogue.o ABSOLUTE
    ../fplib/microlib/fpfix.c                0x00000000   Number         0  dfixul.o ABSOLUTE
    ../fplib/microlib/fpmul.c                0x00000000   Number         0  dmul.o ABSOLUTE
    ..\..\..\..\..\..\components\boards\boards.c 0x00000000   Number         0  boards.o ABSOLUTE
    ..\..\..\..\..\..\components\libraries\atomic\nrf_atomic.c 0x00000000   Number         0  nrf_atomic.o ABSOLUTE
    ..\..\..\..\..\..\components\libraries\balloc\nrf_balloc.c 0x00000000   Number         0  nrf_balloc.o ABSOLUTE
    ..\..\..\..\..\..\components\libraries\fifo\app_fifo.c 0x00000000   Number         0  app_fifo.o ABSOLUTE
    ..\..\..\..\..\..\components\libraries\log\src\nrf_log_frontend.c 0x00000000   Number         0  nrf_log_frontend.o ABSOLUTE
    ..\..\..\..\..\..\components\libraries\log\src\nrf_log_str_formatter.c 0x00000000   Number         0  nrf_log_str_formatter.o ABSOLUTE
    ..\..\..\..\..\..\components\libraries\memobj\nrf_memobj.c 0x00000000   Number         0  nrf_memobj.o ABSOLUTE
    ..\..\..\..\..\..\components\libraries\ringbuf\nrf_ringbuf.c 0x00000000   Number         0  nrf_ringbuf.o ABSOLUTE
    ..\..\..\..\..\..\components\libraries\strerror\nrf_strerror.c 0x00000000   Number         0  nrf_strerror.o ABSOLUTE
    ..\..\..\..\..\..\components\libraries\timer\app_timer.c 0x00000000   Number         0  app_timer.o ABSOLUTE
    ..\..\..\..\..\..\components\libraries\uart\app_uart_fifo.c 0x00000000   Number         0  app_uart_fifo.o ABSOLUTE
    ..\..\..\..\..\..\components\libraries\uart\retarget.c 0x00000000   Number         0  retarget.o ABSOLUTE
    ..\..\..\..\..\..\components\libraries\util\app_error.c 0x00000000   Number         0  app_error.o ABSOLUTE
    ..\..\..\..\..\..\components\libraries\util\app_error_handler_keil.c 0x00000000   Number         0  app_error_handler_keil.o ABSOLUTE
    ..\..\..\..\..\..\components\libraries\util\app_error_weak.c 0x00000000   Number         0  app_error_weak.o ABSOLUTE
    ..\..\..\..\..\..\components\libraries\util\app_util_platform.c 0x00000000   Number         0  app_util_platform.o ABSOLUTE
    ..\..\..\..\..\..\components\libraries\util\nrf_assert.c 0x00000000   Number         0  nrf_assert.o ABSOLUTE
    ..\..\..\..\..\..\components\proprietary_rf\esb\nrf_esb.c 0x00000000   Number         0  nrf_esb.o ABSOLUTE
    ..\..\..\..\..\..\external\fprintf\nrf_fprintf.c 0x00000000   Number         0  nrf_fprintf.o ABSOLUTE
    ..\..\..\..\..\..\external\fprintf\nrf_fprintf_format.c 0x00000000   Number         0  nrf_fprintf_format.o ABSOLUTE
    ..\..\..\..\..\..\integration\nrfx\legacy\nrf_drv_uart.c 0x00000000   Number         0  nrf_drv_uart.o ABSOLUTE
    ..\..\..\..\..\..\modules\nrfx\drivers\src\nrfx_gpiote.c 0x00000000   Number         0  nrfx_gpiote.o ABSOLUTE
    ..\..\..\..\..\..\modules\nrfx\drivers\src\nrfx_uart.c 0x00000000   Number         0  nrfx_uart.o ABSOLUTE
    ..\..\..\..\..\..\modules\nrfx\drivers\src\nrfx_uarte.c 0x00000000   Number         0  nrfx_uarte.o ABSOLUTE
    ..\..\..\..\..\..\modules\nrfx\drivers\src\prs\nrfx_prs.c 0x00000000   Number         0  nrfx_prs.o ABSOLUTE
    ..\..\..\Driver\EsbProcess.c             0x00000000   Number         0  esbprocess.o ABSOLUTE
    ..\..\..\Driver\GpioProcess.c            0x00000000   Number         0  gpioprocess.o ABSOLUTE
    ..\..\..\Driver\UartProcess.c            0x00000000   Number         0  uartprocess.o ABSOLUTE
    ..\..\..\Host.c                          0x00000000   Number         0  host.o ABSOLUTE
    ..\\..\\..\\..\\..\\..\\components\\boards\\boards.c 0x00000000   Number         0  boards.o ABSOLUTE
    ..\\..\\..\\..\\..\\..\\components\\libraries\\atomic\\nrf_atomic.c 0x00000000   Number         0  nrf_atomic.o ABSOLUTE
    ..\\..\\..\\..\\..\\..\\components\\libraries\\balloc\\nrf_balloc.c 0x00000000   Number         0  nrf_balloc.o ABSOLUTE
    ..\\..\\..\\..\\..\\..\\components\\libraries\\fifo\\app_fifo.c 0x00000000   Number         0  app_fifo.o ABSOLUTE
    ..\\..\\..\\..\\..\\..\\components\\libraries\\log\\src\\nrf_log_frontend.c 0x00000000   Number         0  nrf_log_frontend.o ABSOLUTE
    ..\\..\\..\\..\\..\\..\\components\\libraries\\log\\src\\nrf_log_str_formatter.c 0x00000000   Number         0  nrf_log_str_formatter.o ABSOLUTE
    ..\\..\\..\\..\\..\\..\\components\\libraries\\memobj\\nrf_memobj.c 0x00000000   Number         0  nrf_memobj.o ABSOLUTE
    ..\\..\\..\\..\\..\\..\\components\\libraries\\ringbuf\\nrf_ringbuf.c 0x00000000   Number         0  nrf_ringbuf.o ABSOLUTE
    ..\\..\\..\\..\\..\\..\\components\\libraries\\strerror\\nrf_strerror.c 0x00000000   Number         0  nrf_strerror.o ABSOLUTE
    ..\\..\\..\\..\\..\\..\\components\\libraries\\timer\\app_timer.c 0x00000000   Number         0  app_timer.o ABSOLUTE
    ..\\..\\..\\..\\..\\..\\components\\libraries\\uart\\app_uart_fifo.c 0x00000000   Number         0  app_uart_fifo.o ABSOLUTE
    ..\\..\\..\\..\\..\\..\\components\\libraries\\uart\\retarget.c 0x00000000   Number         0  retarget.o ABSOLUTE
    ..\\..\\..\\..\\..\\..\\components\\libraries\\util\\app_error.c 0x00000000   Number         0  app_error.o ABSOLUTE
    ..\\..\\..\\..\\..\\..\\components\\libraries\\util\\app_error_handler_keil.c 0x00000000   Number         0  app_error_handler_keil.o ABSOLUTE
    ..\\..\\..\\..\\..\\..\\components\\libraries\\util\\app_error_weak.c 0x00000000   Number         0  app_error_weak.o ABSOLUTE
    ..\\..\\..\\..\\..\\..\\components\\libraries\\util\\app_util_platform.c 0x00000000   Number         0  app_util_platform.o ABSOLUTE
    ..\\..\\..\\..\\..\\..\\components\\libraries\\util\\nrf_assert.c 0x00000000   Number         0  nrf_assert.o ABSOLUTE
    ..\\..\\..\\..\\..\\..\\components\\proprietary_rf\\esb\\nrf_esb.c 0x00000000   Number         0  nrf_esb.o ABSOLUTE
    ..\\..\\..\\..\\..\\..\\external\\fprintf\\nrf_fprintf.c 0x00000000   Number         0  nrf_fprintf.o ABSOLUTE
    ..\\..\\..\\..\\..\\..\\external\\fprintf\\nrf_fprintf_format.c 0x00000000   Number         0  nrf_fprintf_format.o ABSOLUTE
    ..\\..\\..\\..\\..\\..\\integration\\nrfx\\legacy\\nrf_drv_uart.c 0x00000000   Number         0  nrf_drv_uart.o ABSOLUTE
    ..\\..\\..\\..\\..\\..\\modules\\nrfx\\drivers\\src\\nrfx_gpiote.c 0x00000000   Number         0  nrfx_gpiote.o ABSOLUTE
    ..\\..\\..\\..\\..\\..\\modules\\nrfx\\drivers\\src\\nrfx_uart.c 0x00000000   Number         0  nrfx_uart.o ABSOLUTE
    ..\\..\\..\\..\\..\\..\\modules\\nrfx\\drivers\\src\\nrfx_uarte.c 0x00000000   Number         0  nrfx_uarte.o ABSOLUTE
    ..\\..\\..\\..\\..\\..\\modules\\nrfx\\drivers\\src\\prs\\nrfx_prs.c 0x00000000   Number         0  nrfx_prs.o ABSOLUTE
    ..\\..\\..\\Driver\\EsbProcess.c         0x00000000   Number         0  esbprocess.o ABSOLUTE
    ..\\..\\..\\Driver\\GpioProcess.c        0x00000000   Number         0  gpioprocess.o ABSOLUTE
    ..\\..\\..\\Driver\\UartProcess.c        0x00000000   Number         0  uartprocess.o ABSOLUTE
    ..\\..\\..\\Host.c                       0x00000000   Number         0  host.o ABSOLUTE
    RTE\Device\nRF52832_xxAA\arm_startup_nrf52.s 0x00000000   Number         0  arm_startup_nrf52.o ABSOLUTE
    RTE\Device\nRF52832_xxAA\system_nrf52.c  0x00000000   Number         0  system_nrf52.o ABSOLUTE
    RTE\\Device\\nRF52832_xxAA\\system_nrf52.c 0x00000000   Number         0  system_nrf52.o ABSOLUTE
    cdrcmple.s                               0x00000000   Number         0  cdrcmple.o ABSOLUTE
    dc.s                                     0x00000000   Number         0  dc.o ABSOLUTE
    handlers.s                               0x00000000   Number         0  handlers.o ABSOLUTE
    init.s                                   0x00000000   Number         0  init.o ABSOLUTE
    .ARM.Collect$$$$00000000                 0x00000200   Section        0  entry.o(.ARM.Collect$$$$00000000)
    .ARM.Collect$$$$00000001                 0x00000200   Section        4  entry2.o(.ARM.Collect$$$$00000001)
    .ARM.Collect$$$$00000004                 0x00000204   Section        4  entry5.o(.ARM.Collect$$$$00000004)
    .ARM.Collect$$$$00000008                 0x00000208   Section        0  entry7b.o(.ARM.Collect$$$$00000008)
    .ARM.Collect$$$$0000000A                 0x00000208   Section        0  entry8b.o(.ARM.Collect$$$$0000000A)
    .ARM.Collect$$$$0000000B                 0x00000208   Section        8  entry9a.o(.ARM.Collect$$$$0000000B)
    .ARM.Collect$$$$0000000D                 0x00000210   Section        0  entry10a.o(.ARM.Collect$$$$0000000D)
    .ARM.Collect$$$$0000000F                 0x00000210   Section        0  entry11a.o(.ARM.Collect$$$$0000000F)
    .ARM.Collect$$$$00002712                 0x00000210   Section        4  entry2.o(.ARM.Collect$$$$00002712)
    __lit__00000000                          0x00000210   Data           4  entry2.o(.ARM.Collect$$$$00002712)
    .text                                    0x00000214   Section       36  arm_startup_nrf52.o(.text)
    $v0                                      0x00000214   Number         0  arm_startup_nrf52.o(.text)
    .text                                    0x00000238   Section        0  memcpya.o(.text)
    .text                                    0x0000025c   Section        0  memseta.o(.text)
    .text                                    0x00000280   Section        0  memcmp.o(.text)
    .text                                    0x0000029a   Section        0  uidiv.o(.text)
    .text                                    0x000002c8   Section       36  init.o(.text)
    i.Action_Key1                            0x000002ec   Section        0  host.o(i.Action_Key1)
    i.GPIOTE_IRQHandler                      0x0000030c   Section        0  nrfx_gpiote.o(i.GPIOTE_IRQHandler)
    i.NVIC_ClearPendingIRQ                   0x00000528   Section        0  app_timer.o(i.NVIC_ClearPendingIRQ)
    NVIC_ClearPendingIRQ                     0x00000529   Thumb Code    18  app_timer.o(i.NVIC_ClearPendingIRQ)
    i.NVIC_ClearPendingIRQ                   0x00000540   Section        0  nrf_esb.o(i.NVIC_ClearPendingIRQ)
    NVIC_ClearPendingIRQ                     0x00000541   Thumb Code    18  nrf_esb.o(i.NVIC_ClearPendingIRQ)
    i.NVIC_DisableIRQ                        0x00000558   Section        0  nrf_esb.o(i.NVIC_DisableIRQ)
    NVIC_DisableIRQ                          0x00000559   Thumb Code    18  nrf_esb.o(i.NVIC_DisableIRQ)
    i.NVIC_EnableIRQ                         0x00000570   Section        0  app_timer.o(i.NVIC_EnableIRQ)
    NVIC_EnableIRQ                           0x00000571   Thumb Code    22  app_timer.o(i.NVIC_EnableIRQ)
    i.NVIC_EnableIRQ                         0x00000586   Section        0  nrf_esb.o(i.NVIC_EnableIRQ)
    NVIC_EnableIRQ                           0x00000587   Thumb Code    22  nrf_esb.o(i.NVIC_EnableIRQ)
    i.NVIC_SetPendingIRQ                     0x0000059c   Section        0  app_timer.o(i.NVIC_SetPendingIRQ)
    NVIC_SetPendingIRQ                       0x0000059d   Thumb Code    18  app_timer.o(i.NVIC_SetPendingIRQ)
    i.NVIC_SetPendingIRQ                     0x000005b4   Section        0  nrf_esb.o(i.NVIC_SetPendingIRQ)
    NVIC_SetPendingIRQ                       0x000005b5   Thumb Code    18  nrf_esb.o(i.NVIC_SetPendingIRQ)
    i.NVIC_SetPriority                       0x000005cc   Section        0  app_timer.o(i.NVIC_SetPriority)
    NVIC_SetPriority                         0x000005cd   Thumb Code    32  app_timer.o(i.NVIC_SetPriority)
    i.NVIC_SetPriority                       0x000005f4   Section        0  nrf_esb.o(i.NVIC_SetPriority)
    NVIC_SetPriority                         0x000005f5   Thumb Code    32  nrf_esb.o(i.NVIC_SetPriority)
    i.PacketSend                             0x0000061c   Section        0  host.o(i.PacketSend)
    i.Pin_Trigger_handler_1                  0x00000654   Section        0  gpioprocess.o(i.Pin_Trigger_handler_1)
    i.Pin_Trigger_handler_2                  0x000006ac   Section        0  gpioprocess.o(i.Pin_Trigger_handler_2)
    i.RADIO_IRQHandler                       0x0000071c   Section        0  nrf_esb.o(i.RADIO_IRQHandler)
    i.RTC1_IRQHandler                        0x00000794   Section        0  app_timer.o(i.RTC1_IRQHandler)
    i.SWI0_EGU0_IRQHandler                   0x000007c8   Section        0  nrf_esb.o(i.SWI0_EGU0_IRQHandler)
    i.SWI1_EGU1_IRQHandler                   0x0000082c   Section        0  app_timer.o(i.SWI1_EGU1_IRQHandler)
    i.SystemCoreClockUpdate                  0x00000834   Section        0  system_nrf52.o(i.SystemCoreClockUpdate)
    i.SystemInit                             0x00000844   Section        0  system_nrf52.o(i.SystemInit)
    i.TIMER3_IRQHandler                      0x00000adc   Section        0  nrf_esb.o(i.TIMER3_IRQHandler)
    i.Timer_1S                               0x00000b04   Section        0  host.o(i.Timer_1S)
    i.UARTE0_UART0_IRQHandler                0x00000b3c   Section        0  nrfx_prs.o(i.UARTE0_UART0_IRQHandler)
    i.UART_Init                              0x00000b4c   Section        0  uartprocess.o(i.UART_Init)
    i.__0printf$1                            0x00000ba8   Section        0  printf1.o(i.__0printf$1)
    i.__scatterload_copy                     0x00000bc8   Section       14  handlers.o(i.__scatterload_copy)
    i.__scatterload_null                     0x00000bd6   Section        2  handlers.o(i.__scatterload_null)
    i.__scatterload_zeroinit                 0x00000bd8   Section       14  handlers.o(i.__scatterload_zeroinit)
    i._printf_core                           0x00000be8   Section        0  printf1.o(i._printf_core)
    _printf_core                             0x00000be9   Thumb Code   336  printf1.o(i._printf_core)
    i.addr_conv                              0x00000d3c   Section        0  nrf_esb.o(i.addr_conv)
    addr_conv                                0x00000d3d   Thumb Code    14  nrf_esb.o(i.addr_conv)
    i.app_error_fault_handler                0x00000d4c   Section        0  app_error_weak.o(i.app_error_fault_handler)
    i.app_error_handler_bare                 0x00000da8   Section        0  app_error.o(i.app_error_handler_bare)
    i.app_fifo_get                           0x00000dc4   Section        0  app_fifo.o(i.app_fifo_get)
    i.app_fifo_init                          0x00000de2   Section        0  app_fifo.o(i.app_fifo_init)
    i.app_fifo_put                           0x00000e06   Section        0  app_fifo.o(i.app_fifo_put)
    i.app_timer_create                       0x00000e28   Section        0  app_timer.o(i.app_timer_create)
    i.app_timer_init                         0x00000e64   Section        0  app_timer.o(i.app_timer_init)
    i.app_timer_start                        0x00000ec0   Section        0  app_timer.o(i.app_timer_start)
    i.app_uart_get                           0x00000f14   Section        0  app_uart_fifo.o(i.app_uart_get)
    i.app_uart_init                          0x00000f68   Section        0  app_uart_fifo.o(i.app_uart_init)
    i.app_uart_put                           0x00001044   Section        0  app_uart_fifo.o(i.app_uart_put)
    i.app_util_critical_region_enter         0x000010b0   Section        0  app_util_platform.o(i.app_util_critical_region_enter)
    i.app_util_critical_region_exit          0x000010ba   Section        0  app_util_platform.o(i.app_util_critical_region_exit)
    i.app_util_disable_irq                   0x000010c4   Section        0  app_util_platform.o(i.app_util_disable_irq)
    i.app_util_enable_irq                    0x000010d8   Section        0  app_util_platform.o(i.app_util_enable_irq)
    i.apply_address_workarounds              0x000010f0   Section        0  nrf_esb.o(i.apply_address_workarounds)
    apply_address_workarounds                0x000010f1   Thumb Code   290  nrf_esb.o(i.apply_address_workarounds)
    i.apply_config                           0x0000122c   Section        0  nrfx_uart.o(i.apply_config)
    apply_config                             0x0000122d   Thumb Code   124  nrfx_uart.o(i.apply_config)
    i.apply_config                           0x000012a8   Section        0  nrfx_uarte.o(i.apply_config)
    apply_config                             0x000012a9   Thumb Code   124  nrfx_uarte.o(i.apply_config)
    i.bytewise_bit_swap                      0x00001324   Section        0  nrf_esb.o(i.bytewise_bit_swap)
    bytewise_bit_swap                        0x00001325   Thumb Code    12  nrf_esb.o(i.bytewise_bit_swap)
    i.channel_free                           0x00001330   Section        0  nrfx_gpiote.o(i.channel_free)
    channel_free                             0x00001331   Thumb Code    26  nrfx_gpiote.o(i.channel_free)
    i.channel_handler_get                    0x00001350   Section        0  nrfx_gpiote.o(i.channel_handler_get)
    channel_handler_get                      0x00001351   Thumb Code    10  nrfx_gpiote.o(i.channel_handler_get)
    i.channel_port_alloc                     0x00001360   Section        0  nrfx_gpiote.o(i.channel_port_alloc)
    channel_port_alloc                       0x00001361   Thumb Code   122  nrfx_gpiote.o(i.channel_port_alloc)
    i.channel_port_get                       0x000013e0   Section        0  nrfx_gpiote.o(i.channel_port_get)
    channel_port_get                         0x000013e1   Thumb Code     8  nrfx_gpiote.o(i.channel_port_get)
    i.clear_events_restart_rx                0x000013ec   Section        0  nrf_esb.o(i.clear_events_restart_rx)
    clear_events_restart_rx                  0x000013ed   Thumb Code    78  nrf_esb.o(i.clear_events_restart_rx)
    i.clocks_start                           0x00001458   Section        0  host.o(i.clocks_start)
    i.compare_reg_update                     0x00001474   Section        0  app_timer.o(i.compare_reg_update)
    compare_reg_update                       0x00001475   Thumb Code   132  app_timer.o(i.compare_reg_update)
    i.elapsed_ticks_acquire                  0x00001504   Section        0  app_timer.o(i.elapsed_ticks_acquire)
    elapsed_ticks_acquire                    0x00001505   Thumb Code    82  app_timer.o(i.elapsed_ticks_acquire)
    i.errata_108                             0x00001568   Section        0  system_nrf52.o(i.errata_108)
    errata_108                               0x00001569   Thumb Code    78  system_nrf52.o(i.errata_108)
    i.errata_12                              0x000015bc   Section        0  system_nrf52.o(i.errata_12)
    errata_12                                0x000015bd   Thumb Code    78  system_nrf52.o(i.errata_12)
    i.errata_136                             0x00001610   Section        0  system_nrf52.o(i.errata_136)
    errata_136                               0x00001611   Thumb Code    78  system_nrf52.o(i.errata_136)
    i.errata_16                              0x00001664   Section        0  system_nrf52.o(i.errata_16)
    errata_16                                0x00001665   Thumb Code    42  system_nrf52.o(i.errata_16)
    i.errata_182                             0x00001694   Section        0  system_nrf52.o(i.errata_182)
    errata_182                               0x00001695   Thumb Code    26  system_nrf52.o(i.errata_182)
    i.errata_31                              0x000016b4   Section        0  system_nrf52.o(i.errata_31)
    errata_31                                0x000016b5   Thumb Code    78  system_nrf52.o(i.errata_31)
    i.errata_32                              0x00001708   Section        0  system_nrf52.o(i.errata_32)
    errata_32                                0x00001709   Thumb Code    42  system_nrf52.o(i.errata_32)
    i.errata_36                              0x00001738   Section        0  system_nrf52.o(i.errata_36)
    errata_36                                0x00001739   Thumb Code    78  system_nrf52.o(i.errata_36)
    i.errata_37                              0x0000178c   Section        0  system_nrf52.o(i.errata_37)
    errata_37                                0x0000178d   Thumb Code    42  system_nrf52.o(i.errata_37)
    i.errata_57                              0x000017bc   Section        0  system_nrf52.o(i.errata_57)
    errata_57                                0x000017bd   Thumb Code    42  system_nrf52.o(i.errata_57)
    i.errata_66                              0x000017ec   Section        0  system_nrf52.o(i.errata_66)
    errata_66                                0x000017ed   Thumb Code    42  system_nrf52.o(i.errata_66)
    i.esb_init                               0x0000181c   Section        0  esbprocess.o(i.esb_init)
    i.esb_packet_received                    0x000018f4   Section        0  host.o(i.esb_packet_received)
    i.esb_packet_send                        0x00001978   Section        0  esbprocess.o(i.esb_packet_send)
    i.expired_timers_handler                 0x000019f4   Section        0  app_timer.o(i.expired_timers_handler)
    expired_timers_handler                   0x000019f5   Thumb Code    84  app_timer.o(i.expired_timers_handler)
    i.fifo_get                               0x00001a4c   Section        0  app_fifo.o(i.fifo_get)
    fifo_get                                 0x00001a4d   Thumb Code    24  app_fifo.o(i.fifo_get)
    i.fifo_length                            0x00001a64   Section        0  app_fifo.o(i.fifo_length)
    fifo_length                              0x00001a65   Thumb Code    10  app_fifo.o(i.fifo_length)
    i.fifo_length                            0x00001a6e   Section        0  app_uart_fifo.o(i.fifo_length)
    fifo_length                              0x00001a6f   Thumb Code    10  app_uart_fifo.o(i.fifo_length)
    i.fifo_peek                              0x00001a78   Section        0  app_fifo.o(i.fifo_peek)
    fifo_peek                                0x00001a79   Thumb Code    18  app_fifo.o(i.fifo_peek)
    i.fifo_put                               0x00001a8a   Section        0  app_fifo.o(i.fifo_put)
    fifo_put                                 0x00001a8b   Thumb Code    18  app_fifo.o(i.fifo_put)
    i.fputc                                  0x00001a9c   Section        0  retarget.o(i.fputc)
    i.gpio_init                              0x00001aac   Section        0  gpioprocess.o(i.gpio_init)
    i.initialize_fifos                       0x00001b5c   Section        0  nrf_esb.o(i.initialize_fifos)
    initialize_fifos                         0x00001b5d   Thumb Code    56  nrf_esb.o(i.initialize_fifos)
    i.interrupts_enable                      0x00001ba4   Section        0  nrfx_uart.o(i.interrupts_enable)
    interrupts_enable                        0x00001ba5   Thumb Code   124  nrfx_uart.o(i.interrupts_enable)
    i.interrupts_enable                      0x00001c2c   Section        0  nrfx_uarte.o(i.interrupts_enable)
    interrupts_enable                        0x00001c2d   Thumb Code   144  nrfx_uarte.o(i.interrupts_enable)
    i.list_insertions_handler                0x00001cc8   Section        0  app_timer.o(i.list_insertions_handler)
    list_insertions_handler                  0x00001cc9   Thumb Code   294  app_timer.o(i.list_insertions_handler)
    i.main                                   0x00001e04   Section        0  host.o(i.main)
    i.nrf_bitmask_bit_is_set                 0x00001e64   Section        0  nrfx_gpiote.o(i.nrf_bitmask_bit_is_set)
    nrf_bitmask_bit_is_set                   0x00001e65   Thumb Code    22  nrfx_gpiote.o(i.nrf_bitmask_bit_is_set)
    i.nrf_bitmask_bit_set                    0x00001e7a   Section        0  nrfx_gpiote.o(i.nrf_bitmask_bit_set)
    nrf_bitmask_bit_set                      0x00001e7b   Thumb Code    22  nrfx_gpiote.o(i.nrf_bitmask_bit_set)
    i.nrf_drv_uart_init                      0x00001e90   Section        0  nrf_drv_uart.o(i.nrf_drv_uart_init)
    i.nrf_drv_uart_rx                        0x00001f1c   Section        0  app_uart_fifo.o(i.nrf_drv_uart_rx)
    nrf_drv_uart_rx                          0x00001f1d   Thumb Code    62  app_uart_fifo.o(i.nrf_drv_uart_rx)
    i.nrf_drv_uart_tx                        0x00001f60   Section        0  app_uart_fifo.o(i.nrf_drv_uart_tx)
    nrf_drv_uart_tx                          0x00001f61   Thumb Code    62  app_uart_fifo.o(i.nrf_drv_uart_tx)
    i.nrf_esb_disable                        0x00001fa4   Section        0  nrf_esb.o(i.nrf_esb_disable)
    i.nrf_esb_event_handler                  0x00001ff4   Section        0  esbprocess.o(i.nrf_esb_event_handler)
    i.nrf_esb_get_clear_interrupts           0x00002078   Section        0  nrf_esb.o(i.nrf_esb_get_clear_interrupts)
    nrf_esb_get_clear_interrupts             0x00002079   Thumb Code    56  nrf_esb.o(i.nrf_esb_get_clear_interrupts)
    i.nrf_esb_init                           0x000020b8   Section        0  nrf_esb.o(i.nrf_esb_init)
    i.nrf_esb_read_rx_payload                0x000021b0   Section        0  nrf_esb.o(i.nrf_esb_read_rx_payload)
    i.nrf_esb_set_base_address_0             0x0000225c   Section        0  nrf_esb.o(i.nrf_esb_set_base_address_0)
    i.nrf_esb_set_base_address_1             0x000022d8   Section        0  nrf_esb.o(i.nrf_esb_set_base_address_1)
    i.nrf_esb_set_prefixes                   0x00002398   Section        0  nrf_esb.o(i.nrf_esb_set_prefixes)
    i.nrf_esb_set_rf_channel                 0x00002454   Section        0  nrf_esb.o(i.nrf_esb_set_rf_channel)
    i.nrf_esb_skip_tx                        0x00002480   Section        0  nrf_esb.o(i.nrf_esb_skip_tx)
    i.nrf_esb_start_rx                       0x000024d4   Section        0  nrf_esb.o(i.nrf_esb_start_rx)
    i.nrf_esb_start_tx                       0x0000257c   Section        0  nrf_esb.o(i.nrf_esb_start_tx)
    i.nrf_esb_stop_rx                        0x000025a8   Section        0  nrf_esb.o(i.nrf_esb_stop_rx)
    i.nrf_esb_write_payload                  0x00002604   Section        0  nrf_esb.o(i.nrf_esb_write_payload)
    i.nrf_gpio_cfg                           0x000026f4   Section        0  nrfx_uart.o(i.nrf_gpio_cfg)
    nrf_gpio_cfg                             0x000026f5   Thumb Code    40  nrfx_uart.o(i.nrf_gpio_cfg)
    i.nrf_gpio_cfg                           0x0000271c   Section        0  nrfx_uarte.o(i.nrf_gpio_cfg)
    nrf_gpio_cfg                             0x0000271d   Thumb Code    40  nrfx_uarte.o(i.nrf_gpio_cfg)
    i.nrf_gpio_cfg                           0x00002744   Section        0  nrfx_gpiote.o(i.nrf_gpio_cfg)
    nrf_gpio_cfg                             0x00002745   Thumb Code    40  nrfx_gpiote.o(i.nrf_gpio_cfg)
    i.nrf_gpio_cfg_input                     0x0000276c   Section        0  nrfx_uart.o(i.nrf_gpio_cfg_input)
    nrf_gpio_cfg_input                       0x0000276d   Thumb Code    26  nrfx_uart.o(i.nrf_gpio_cfg_input)
    i.nrf_gpio_cfg_input                     0x00002786   Section        0  nrfx_uarte.o(i.nrf_gpio_cfg_input)
    nrf_gpio_cfg_input                       0x00002787   Thumb Code    26  nrfx_uarte.o(i.nrf_gpio_cfg_input)
    i.nrf_gpio_cfg_output                    0x000027a0   Section        0  gpioprocess.o(i.nrf_gpio_cfg_output)
    nrf_gpio_cfg_output                      0x000027a1   Thumb Code    48  gpioprocess.o(i.nrf_gpio_cfg_output)
    i.nrf_gpio_cfg_output                    0x000027d0   Section        0  nrfx_uart.o(i.nrf_gpio_cfg_output)
    nrf_gpio_cfg_output                      0x000027d1   Thumb Code    24  nrfx_uart.o(i.nrf_gpio_cfg_output)
    i.nrf_gpio_cfg_output                    0x000027e8   Section        0  nrfx_uarte.o(i.nrf_gpio_cfg_output)
    nrf_gpio_cfg_output                      0x000027e9   Thumb Code    24  nrfx_uarte.o(i.nrf_gpio_cfg_output)
    i.nrf_gpio_cfg_sense_set                 0x00002800   Section        0  nrfx_gpiote.o(i.nrf_gpio_cfg_sense_set)
    nrf_gpio_cfg_sense_set                   0x00002801   Thumb Code    50  nrfx_gpiote.o(i.nrf_gpio_cfg_sense_set)
    i.nrf_gpio_pin_clear                     0x00002832   Section        0  gpioprocess.o(i.nrf_gpio_pin_clear)
    nrf_gpio_pin_clear                       0x00002833   Thumb Code    22  gpioprocess.o(i.nrf_gpio_pin_clear)
    i.nrf_gpio_pin_read                      0x00002848   Section        0  nrfx_gpiote.o(i.nrf_gpio_pin_read)
    nrf_gpio_pin_read                        0x00002849   Thumb Code    24  nrfx_gpiote.o(i.nrf_gpio_pin_read)
    i.nrf_gpio_pin_set                       0x00002860   Section        0  nrfx_uart.o(i.nrf_gpio_pin_set)
    nrf_gpio_pin_set                         0x00002861   Thumb Code    22  nrfx_uart.o(i.nrf_gpio_pin_set)
    i.nrf_gpio_pin_set                       0x00002876   Section        0  nrfx_uarte.o(i.nrf_gpio_pin_set)
    nrf_gpio_pin_set                         0x00002877   Thumb Code    22  nrfx_uarte.o(i.nrf_gpio_pin_set)
    i.nrf_gpio_ports_read                    0x0000288c   Section        0  nrfx_gpiote.o(i.nrf_gpio_ports_read)
    nrf_gpio_ports_read                      0x0000288d   Thumb Code    36  nrfx_gpiote.o(i.nrf_gpio_ports_read)
    i.nrf_gpiote_event_addr_get              0x000028b4   Section        0  nrfx_gpiote.o(i.nrf_gpiote_event_addr_get)
    nrf_gpiote_event_addr_get                0x000028b5   Thumb Code     8  nrfx_gpiote.o(i.nrf_gpiote_event_addr_get)
    i.nrf_gpiote_event_clear                 0x000028c0   Section        0  nrfx_gpiote.o(i.nrf_gpiote_event_clear)
    nrf_gpiote_event_clear                   0x000028c1   Thumb Code    28  nrfx_gpiote.o(i.nrf_gpiote_event_clear)
    i.nrf_gpiote_event_is_set                0x000028dc   Section        0  nrfx_gpiote.o(i.nrf_gpiote_event_is_set)
    nrf_gpiote_event_is_set                  0x000028dd   Thumb Code    22  nrfx_gpiote.o(i.nrf_gpiote_event_is_set)
    i.nrf_gpiote_int_enable                  0x000028f4   Section        0  nrfx_gpiote.o(i.nrf_gpiote_int_enable)
    nrf_gpiote_int_enable                    0x000028f5   Thumb Code     6  nrfx_gpiote.o(i.nrf_gpiote_int_enable)
    i.nrf_uart_errorsrc_get_and_clear        0x00002900   Section        0  nrfx_uart.o(i.nrf_uart_errorsrc_get_and_clear)
    nrf_uart_errorsrc_get_and_clear          0x00002901   Thumb Code    12  nrfx_uart.o(i.nrf_uart_errorsrc_get_and_clear)
    i.nrf_uart_event_check                   0x0000290c   Section        0  nrfx_uart.o(i.nrf_uart_event_check)
    nrf_uart_event_check                     0x0000290d   Thumb Code    14  nrfx_uart.o(i.nrf_uart_event_check)
    i.nrf_uart_event_clear                   0x0000291a   Section        0  nrfx_uart.o(i.nrf_uart_event_clear)
    nrf_uart_event_clear                     0x0000291b   Thumb Code    14  nrfx_uart.o(i.nrf_uart_event_clear)
    i.nrf_uart_hwfc_pins_set                 0x00002928   Section        0  nrfx_uart.o(i.nrf_uart_hwfc_pins_set)
    nrf_uart_hwfc_pins_set                   0x00002929   Thumb Code    10  nrfx_uart.o(i.nrf_uart_hwfc_pins_set)
    i.nrf_uart_int_disable                   0x00002932   Section        0  nrfx_uart.o(i.nrf_uart_int_disable)
    nrf_uart_int_disable                     0x00002933   Thumb Code     6  nrfx_uart.o(i.nrf_uart_int_disable)
    i.nrf_uart_int_enable                    0x00002938   Section        0  nrfx_uart.o(i.nrf_uart_int_enable)
    nrf_uart_int_enable                      0x00002939   Thumb Code     6  nrfx_uart.o(i.nrf_uart_int_enable)
    i.nrf_uart_int_enable_check              0x0000293e   Section        0  nrfx_uart.o(i.nrf_uart_int_enable_check)
    nrf_uart_int_enable_check                0x0000293f   Thumb Code    18  nrfx_uart.o(i.nrf_uart_int_enable_check)
    i.nrf_uart_task_trigger                  0x00002950   Section        0  nrfx_uart.o(i.nrf_uart_task_trigger)
    nrf_uart_task_trigger                    0x00002951   Thumb Code     6  nrfx_uart.o(i.nrf_uart_task_trigger)
    i.nrf_uart_txrx_pins_set                 0x00002956   Section        0  nrfx_uart.o(i.nrf_uart_txrx_pins_set)
    nrf_uart_txrx_pins_set                   0x00002957   Thumb Code    10  nrfx_uart.o(i.nrf_uart_txrx_pins_set)
    i.nrf_uarte_errorsrc_get_and_clear       0x00002960   Section        0  nrfx_uarte.o(i.nrf_uarte_errorsrc_get_and_clear)
    nrf_uarte_errorsrc_get_and_clear         0x00002961   Thumb Code    12  nrfx_uarte.o(i.nrf_uarte_errorsrc_get_and_clear)
    i.nrf_uarte_event_check                  0x0000296c   Section        0  nrfx_uarte.o(i.nrf_uarte_event_check)
    nrf_uarte_event_check                    0x0000296d   Thumb Code    14  nrfx_uarte.o(i.nrf_uarte_event_check)
    i.nrf_uarte_event_clear                  0x0000297a   Section        0  nrfx_uarte.o(i.nrf_uarte_event_clear)
    nrf_uarte_event_clear                    0x0000297b   Thumb Code    14  nrfx_uarte.o(i.nrf_uarte_event_clear)
    i.nrf_uarte_hwfc_pins_set                0x00002988   Section        0  nrfx_uarte.o(i.nrf_uarte_hwfc_pins_set)
    nrf_uarte_hwfc_pins_set                  0x00002989   Thumb Code    12  nrfx_uarte.o(i.nrf_uarte_hwfc_pins_set)
    i.nrf_uarte_int_disable                  0x00002994   Section        0  nrfx_uarte.o(i.nrf_uarte_int_disable)
    nrf_uarte_int_disable                    0x00002995   Thumb Code     6  nrfx_uarte.o(i.nrf_uarte_int_disable)
    i.nrf_uarte_int_enable                   0x0000299a   Section        0  nrfx_uarte.o(i.nrf_uarte_int_enable)
    nrf_uarte_int_enable                     0x0000299b   Thumb Code     6  nrfx_uarte.o(i.nrf_uarte_int_enable)
    i.nrf_uarte_rx_amount_get                0x000029a0   Section        0  nrfx_uarte.o(i.nrf_uarte_rx_amount_get)
    nrf_uarte_rx_amount_get                  0x000029a1   Thumb Code    10  nrfx_uarte.o(i.nrf_uarte_rx_amount_get)
    i.nrf_uarte_shorts_disable               0x000029aa   Section        0  nrfx_uarte.o(i.nrf_uarte_shorts_disable)
    nrf_uarte_shorts_disable                 0x000029ab   Thumb Code    12  nrfx_uarte.o(i.nrf_uarte_shorts_disable)
    i.nrf_uarte_task_trigger                 0x000029b6   Section        0  nrfx_uarte.o(i.nrf_uarte_task_trigger)
    nrf_uarte_task_trigger                   0x000029b7   Thumb Code     6  nrfx_uarte.o(i.nrf_uarte_task_trigger)
    i.nrf_uarte_txrx_pins_set                0x000029bc   Section        0  nrfx_uarte.o(i.nrf_uarte_txrx_pins_set)
    nrf_uarte_txrx_pins_set                  0x000029bd   Thumb Code    14  nrfx_uarte.o(i.nrf_uarte_txrx_pins_set)
    i.nrfx_coredep_delay_us                  0x000029cc   Section        0  app_timer.o(i.nrfx_coredep_delay_us)
    nrfx_coredep_delay_us                    0x000029cd   Thumb Code    20  app_timer.o(i.nrfx_coredep_delay_us)
    i.nrfx_get_irq_number                    0x000029e4   Section        0  nrfx_uart.o(i.nrfx_get_irq_number)
    nrfx_get_irq_number                      0x000029e5   Thumb Code     8  nrfx_uart.o(i.nrfx_get_irq_number)
    i.nrfx_get_irq_number                    0x000029ec   Section        0  nrfx_uarte.o(i.nrfx_get_irq_number)
    nrfx_get_irq_number                      0x000029ed   Thumb Code     8  nrfx_uarte.o(i.nrfx_get_irq_number)
    i.nrfx_gpiote_in_event_enable            0x000029f4   Section        0  nrfx_gpiote.o(i.nrfx_gpiote_in_event_enable)
    i.nrfx_gpiote_in_init                    0x00002aa0   Section        0  nrfx_gpiote.o(i.nrfx_gpiote_in_init)
    i.nrfx_gpiote_init                       0x00002b94   Section        0  nrfx_gpiote.o(i.nrfx_gpiote_init)
    i.nrfx_is_in_ram                         0x00002c44   Section        0  nrfx_uarte.o(i.nrfx_is_in_ram)
    nrfx_is_in_ram                           0x00002c45   Thumb Code    20  nrfx_uarte.o(i.nrfx_is_in_ram)
    i.nrfx_prs_acquire                       0x00002c58   Section        0  nrfx_prs.o(i.nrfx_prs_acquire)
    i.nrfx_uart_0_irq_handler                0x00002ca0   Section        0  nrfx_uart.o(i.nrfx_uart_0_irq_handler)
    i.nrfx_uart_init                         0x00002cb4   Section        0  nrfx_uart.o(i.nrfx_uart_init)
    i.nrfx_uart_rx                           0x00002d3c   Section        0  nrfx_uart.o(i.nrfx_uart_rx)
    i.nrfx_uart_tx                           0x00002e60   Section        0  nrfx_uart.o(i.nrfx_uart_tx)
    i.nrfx_uart_tx_in_progress               0x00002eec   Section        0  nrfx_uart.o(i.nrfx_uart_tx_in_progress)
    i.nrfx_uarte_0_irq_handler               0x00002f10   Section        0  nrfx_uarte.o(i.nrfx_uarte_0_irq_handler)
    i.nrfx_uarte_init                        0x00002f24   Section        0  nrfx_uarte.o(i.nrfx_uarte_init)
    i.nrfx_uarte_rx                          0x00002fa4   Section        0  nrfx_uarte.o(i.nrfx_uarte_rx)
    i.nrfx_uarte_tx                          0x000030dc   Section        0  nrfx_uarte.o(i.nrfx_uarte_tx)
    i.nrfx_uarte_tx_in_progress              0x00003184   Section        0  nrfx_uarte.o(i.nrfx_uarte_tx_in_progress)
    i.on_radio_disabled_rx                   0x000031a4   Section        0  nrf_esb.o(i.on_radio_disabled_rx)
    on_radio_disabled_rx                     0x000031a5   Thumb Code   408  nrf_esb.o(i.on_radio_disabled_rx)
    i.on_radio_disabled_rx_ack               0x0000337c   Section        0  nrf_esb.o(i.on_radio_disabled_rx_ack)
    on_radio_disabled_rx_ack                 0x0000337d   Thumb Code    44  nrf_esb.o(i.on_radio_disabled_rx_ack)
    i.on_radio_disabled_tx                   0x000033cc   Section        0  nrf_esb.o(i.on_radio_disabled_tx)
    on_radio_disabled_tx                     0x000033cd   Thumb Code   102  nrf_esb.o(i.on_radio_disabled_tx)
    i.on_radio_disabled_tx_noack             0x00003470   Section        0  nrf_esb.o(i.on_radio_disabled_tx_noack)
    on_radio_disabled_tx_noack               0x00003471   Thumb Code    50  nrf_esb.o(i.on_radio_disabled_tx_noack)
    i.on_radio_disabled_tx_wait_for_ack      0x000034b0   Section        0  nrf_esb.o(i.on_radio_disabled_tx_wait_for_ack)
    on_radio_disabled_tx_wait_for_ack        0x000034b1   Thumb Code   290  nrf_esb.o(i.on_radio_disabled_tx_wait_for_ack)
    i.pin_configured_set                     0x00003620   Section        0  nrfx_gpiote.o(i.pin_configured_set)
    pin_configured_set                       0x00003621   Thumb Code    14  nrfx_gpiote.o(i.pin_configured_set)
    i.pin_in_use_by_gpiote                   0x00003634   Section        0  nrfx_gpiote.o(i.pin_in_use_by_gpiote)
    pin_in_use_by_gpiote                     0x00003635   Thumb Code    22  nrfx_gpiote.o(i.pin_in_use_by_gpiote)
    i.pin_in_use_by_port                     0x00003650   Section        0  nrfx_gpiote.o(i.pin_in_use_by_port)
    pin_in_use_by_port                       0x00003651   Thumb Code    18  nrfx_gpiote.o(i.pin_in_use_by_port)
    i.pin_in_use_by_te                       0x00003668   Section        0  nrfx_gpiote.o(i.pin_in_use_by_te)
    pin_in_use_by_te                         0x00003669   Thumb Code    26  nrfx_gpiote.o(i.pin_in_use_by_te)
    i.pin_in_use_clear                       0x00003688   Section        0  nrfx_gpiote.o(i.pin_in_use_clear)
    pin_in_use_clear                         0x00003689   Thumb Code     8  nrfx_gpiote.o(i.pin_in_use_clear)
    i.ppi_init                               0x00003694   Section        0  nrf_esb.o(i.ppi_init)
    ppi_init                                 0x00003695   Thumb Code    58  nrf_esb.o(i.ppi_init)
    i.prs_box_get                            0x000036e4   Section        0  nrfx_prs.o(i.prs_box_get)
    prs_box_get                              0x000036e5   Thumb Code    16  nrfx_prs.o(i.prs_box_get)
    i.reset_fifos                            0x000036fc   Section        0  nrf_esb.o(i.reset_fifos)
    reset_fifos                              0x000036fd   Thumb Code    20  nrf_esb.o(i.reset_fifos)
    i.rtc1_compare0_set                      0x00003718   Section        0  app_timer.o(i.rtc1_compare0_set)
    rtc1_compare0_set                        0x00003719   Thumb Code     6  app_timer.o(i.rtc1_compare0_set)
    i.rtc1_counter_get                       0x00003724   Section        0  app_timer.o(i.rtc1_counter_get)
    rtc1_counter_get                         0x00003725   Thumb Code     6  app_timer.o(i.rtc1_counter_get)
    i.rtc1_init                              0x00003730   Section        0  app_timer.o(i.rtc1_init)
    rtc1_init                                0x00003731   Thumb Code    18  app_timer.o(i.rtc1_init)
    i.rtc1_start                             0x00003748   Section        0  app_timer.o(i.rtc1_start)
    rtc1_start                               0x00003749   Thumb Code    48  app_timer.o(i.rtc1_start)
    i.rtc1_stop                              0x00003784   Section        0  app_timer.o(i.rtc1_stop)
    rtc1_stop                                0x00003785   Thumb Code    68  app_timer.o(i.rtc1_stop)
    i.rx_byte                                0x000037dc   Section        0  nrfx_uart.o(i.rx_byte)
    rx_byte                                  0x000037dd   Thumb Code    62  nrfx_uart.o(i.rx_byte)
    i.rx_done_event                          0x0000381a   Section        0  nrfx_uart.o(i.rx_done_event)
    rx_done_event                            0x0000381b   Thumb Code    28  nrfx_uart.o(i.rx_done_event)
    i.rx_done_event                          0x00003836   Section        0  nrfx_uarte.o(i.rx_done_event)
    rx_done_event                            0x00003837   Thumb Code    28  nrfx_uarte.o(i.rx_done_event)
    i.rx_enable                              0x00003852   Section        0  nrfx_uart.o(i.rx_enable)
    rx_enable                                0x00003853   Thumb Code    34  nrfx_uart.o(i.rx_enable)
    i.rx_fifo_push_rfbuf                     0x00003874   Section        0  nrf_esb.o(i.rx_fifo_push_rfbuf)
    rx_fifo_push_rfbuf                       0x00003875   Thumb Code   216  nrf_esb.o(i.rx_fifo_push_rfbuf)
    i.start_tx_transaction                   0x0000395c   Section        0  nrf_esb.o(i.start_tx_transaction)
    start_tx_transaction                     0x0000395d   Thumb Code   372  nrf_esb.o(i.start_tx_transaction)
    i.sys_timer_init                         0x00003b10   Section        0  nrf_esb.o(i.sys_timer_init)
    sys_timer_init                           0x00003b11   Thumb Code    24  nrf_esb.o(i.sys_timer_init)
    i.ticks_diff_get                         0x00003b30   Section        0  app_timer.o(i.ticks_diff_get)
    ticks_diff_get                           0x00003b31   Thumb Code    10  app_timer.o(i.ticks_diff_get)
    i.timeout_handler_exec                   0x00003b3a   Section        0  app_timer.o(i.timeout_handler_exec)
    timeout_handler_exec                     0x00003b3b   Thumb Code    12  app_timer.o(i.timeout_handler_exec)
    i.timer_list_handler                     0x00003b48   Section        0  app_timer.o(i.timer_list_handler)
    timer_list_handler                       0x00003b49   Thumb Code    68  app_timer.o(i.timer_list_handler)
    i.timer_list_handler_sched               0x00003b98   Section        0  app_timer.o(i.timer_list_handler_sched)
    timer_list_handler_sched                 0x00003b99   Thumb Code    10  app_timer.o(i.timer_list_handler_sched)
    i.timer_list_insert                      0x00003ba4   Section        0  app_timer.o(i.timer_list_insert)
    timer_list_insert                        0x00003ba5   Thumb Code    98  app_timer.o(i.timer_list_insert)
    i.timer_list_remove                      0x00003c0c   Section        0  app_timer.o(i.timer_list_remove)
    timer_list_remove                        0x00003c0d   Thumb Code   118  app_timer.o(i.timer_list_remove)
    i.timer_start_op_schedule                0x00003c94   Section        0  app_timer.o(i.timer_start_op_schedule)
    timer_start_op_schedule                  0x00003c95   Thumb Code    88  app_timer.o(i.timer_start_op_schedule)
    i.timer_timeouts_check                   0x00003cec   Section        0  app_timer.o(i.timer_timeouts_check)
    timer_timeouts_check                     0x00003ced   Thumb Code   130  app_timer.o(i.timer_timeouts_check)
    i.timer_timeouts_check_sched             0x00003d84   Section        0  app_timer.o(i.timer_timeouts_check_sched)
    timer_timeouts_check_sched               0x00003d85   Thumb Code    10  app_timer.o(i.timer_timeouts_check_sched)
    i.timers_init                            0x00003d90   Section        0  host.o(i.timers_init)
    timers_init                              0x00003d91   Thumb Code    64  host.o(i.timers_init)
    i.timers_start                           0x00003dd8   Section        0  host.o(i.timers_start)
    timers_start                             0x00003dd9   Thumb Code    38  host.o(i.timers_start)
    i.tx_blocking                            0x00003e04   Section        0  nrfx_uart.o(i.tx_blocking)
    tx_blocking                              0x00003e05   Thumb Code    54  nrfx_uart.o(i.tx_blocking)
    i.tx_byte                                0x00003e3a   Section        0  nrfx_uart.o(i.tx_byte)
    tx_byte                                  0x00003e3b   Thumb Code    38  nrfx_uart.o(i.tx_byte)
    i.tx_done_event                          0x00003e60   Section        0  nrfx_uart.o(i.tx_done_event)
    tx_done_event                            0x00003e61   Thumb Code    32  nrfx_uart.o(i.tx_done_event)
    i.tx_done_event                          0x00003e80   Section        0  nrfx_uarte.o(i.tx_done_event)
    tx_done_event                            0x00003e81   Thumb Code    32  nrfx_uarte.o(i.tx_done_event)
    i.uart_event_handle                      0x00003ea0   Section        0  uartprocess.o(i.uart_event_handle)
    i.uart_event_handler                     0x00004034   Section        0  app_uart_fifo.o(i.uart_event_handler)
    uart_event_handler                       0x00004035   Thumb Code   184  app_uart_fifo.o(i.uart_event_handler)
    i.uart_evt_handler                       0x00004108   Section        0  nrf_drv_uart.o(i.uart_evt_handler)
    uart_evt_handler                         0x00004109   Thumb Code    46  nrf_drv_uart.o(i.uart_evt_handler)
    i.uart_irq_handler                       0x00004140   Section        0  nrfx_uart.o(i.uart_irq_handler)
    uart_irq_handler                         0x00004141   Thumb Code   332  nrfx_uart.o(i.uart_irq_handler)
    i.uarte_evt_handler                      0x0000428c   Section        0  nrf_drv_uart.o(i.uarte_evt_handler)
    uarte_evt_handler                        0x0000428d   Thumb Code    46  nrf_drv_uart.o(i.uarte_evt_handler)
    i.uarte_irq_handler                      0x000042c4   Section        0  nrfx_uarte.o(i.uarte_irq_handler)
    uarte_irq_handler                        0x000042c5   Thumb Code   260  nrfx_uarte.o(i.uarte_irq_handler)
    i.update_radio_addresses                 0x000043c8   Section        0  nrf_esb.o(i.update_radio_addresses)
    update_radio_addresses                   0x000043c9   Thumb Code    76  nrf_esb.o(i.update_radio_addresses)
    i.update_radio_bitrate                   0x0000441c   Section        0  nrf_esb.o(i.update_radio_bitrate)
    update_radio_bitrate                     0x0000441d   Thumb Code    64  nrf_esb.o(i.update_radio_bitrate)
    i.update_radio_crc                       0x00004468   Section        0  nrf_esb.o(i.update_radio_crc)
    update_radio_crc                         0x00004469   Thumb Code    68  nrf_esb.o(i.update_radio_crc)
    i.update_radio_parameters                0x000044b8   Section        0  nrf_esb.o(i.update_radio_parameters)
    update_radio_parameters                  0x000044b9   Thumb Code    56  nrf_esb.o(i.update_radio_parameters)
    i.update_radio_protocol                  0x000044f8   Section        0  nrf_esb.o(i.update_radio_protocol)
    update_radio_protocol                    0x000044f9   Thumb Code    36  nrf_esb.o(i.update_radio_protocol)
    i.update_radio_tx_power                  0x0000452c   Section        0  nrf_esb.o(i.update_radio_tx_power)
    update_radio_tx_power                    0x0000452d   Thumb Code    10  nrf_esb.o(i.update_radio_tx_power)
    i.update_rf_payload_format_esb           0x00004540   Section        0  nrf_esb.o(i.update_rf_payload_format_esb)
    update_rf_payload_format_esb             0x00004541   Thumb Code    34  nrf_esb.o(i.update_rf_payload_format_esb)
    i.update_rf_payload_format_esb_dpl       0x00004570   Section        0  nrf_esb.o(i.update_rf_payload_format_esb_dpl)
    update_rf_payload_format_esb_dpl         0x00004571   Thumb Code    32  nrf_esb.o(i.update_rf_payload_format_esb_dpl)
    i.user_op_alloc                          0x0000459c   Section        0  app_timer.o(i.user_op_alloc)
    user_op_alloc                            0x0000459d   Thumb Code    56  app_timer.o(i.user_op_alloc)
    i.user_op_enque                          0x000045d8   Section        0  app_timer.o(i.user_op_enque)
    user_op_enque                            0x000045d9   Thumb Code     6  app_timer.o(i.user_op_enque)
    .constdata                               0x000045e4   Section        3  gpioprocess.o(.constdata)
    .constdata                               0x000045e8   Section        4  host.o(.constdata)
    Timer_1S_timer_id                        0x000045e8   Data           4  host.o(.constdata)
    .constdata                               0x000045ec   Section       46  nrfx_uart.o(.constdata)
    __func__                                 0x000045ec   Data          15  nrfx_uart.o(.constdata)
    irq_handlers                             0x000045fc   Data           4  nrfx_uart.o(.constdata)
    __func__                                 0x00004600   Data          13  nrfx_uart.o(.constdata)
    __func__                                 0x0000460d   Data          13  nrfx_uart.o(.constdata)
    .constdata                               0x0000461c   Section       48  nrfx_uarte.o(.constdata)
    __func__                                 0x0000461c   Data          16  nrfx_uarte.o(.constdata)
    irq_handlers                             0x0000462c   Data           4  nrfx_uarte.o(.constdata)
    __func__                                 0x00004630   Data          14  nrfx_uarte.o(.constdata)
    __func__                                 0x0000463e   Data          14  nrfx_uarte.o(.constdata)
    .constdata                               0x0000464c   Section       62  nrfx_gpiote.o(.constdata)
    __func__                                 0x00004650   Data          17  nrfx_gpiote.o(.constdata)
    __func__                                 0x00004661   Data          21  nrfx_gpiote.o(.constdata)
    __func__                                 0x00004676   Data          20  nrfx_gpiote.o(.constdata)
    .constdata                               0x0000468c   Section       32  app_uart_fifo.o(.constdata)
    .constdata                               0x000046b0   Section        6  app_timer.o(.constdata)
    delay_machine_code                       0x000046b0   Data           6  app_timer.o(.constdata)
    .constdata                               0x000046c0   Section       32  uartprocess.o(.constdata)
    delay_machine_code                       0x000046c0   Data           6  uartprocess.o(.constdata)
    .ARM.__AT_0x1000120C                     0x1000120c   Section        4  gpioprocess.o(.ARM.__AT_0x1000120C)
    __tagsym$$used                           0x1000120c   Number         0  gpioprocess.o(.ARM.__AT_0x1000120C)
    .data                                    0x20000000   Section        1  gpioprocess.o(.data)
    .data                                    0x20000004   Section        6  host.o(.data)
    .data                                    0x2000000c   Section       52  esbprocess.o(.data)
    .data                                    0x20000040   Section        9  nrf_drv_uart.o(.data)
    m_handlers                               0x20000040   Data           4  nrf_drv_uart.o(.data)
    m_contexts                               0x20000044   Data           4  nrf_drv_uart.o(.data)
    .data                                    0x2000004c   Section        8  nrfx_prs.o(.data)
    m_prs_box_4                              0x2000004c   Data           8  nrfx_prs.o(.data)
    .data                                    0x20000054   Section       27  app_uart_fifo.o(.data)
    app_uart_inst                            0x20000054   Data          20  app_uart_fifo.o(.data)
    m_event_handler                          0x20000068   Data           4  app_uart_fifo.o(.data)
    tx_buffer                                0x2000006c   Data           1  app_uart_fifo.o(.data)
    rx_buffer                                0x2000006d   Data           1  app_uart_fifo.o(.data)
    m_rx_ovf                                 0x2000006e   Data           1  app_uart_fifo.o(.data)
    .data                                    0x20000070   Section        4  app_util_platform.o(.data)
    m_in_critical_region                     0x20000070   Data           4  app_util_platform.o(.data)
    .data                                    0x20000074   Section       20  app_timer.o(.data)
    mp_timer_id_head                         0x20000074   Data           4  app_timer.o(.data)
    m_ticks_latest                           0x20000078   Data           4  app_timer.o(.data)
    m_ticks_elapsed                          0x2000007c   Data           8  app_timer.o(.data)
    m_ticks_elapsed_q_read_ind               0x20000084   Data           1  app_timer.o(.data)
    m_ticks_elapsed_q_write_ind              0x20000085   Data           1  app_timer.o(.data)
    m_rtc1_running                           0x20000086   Data           1  app_timer.o(.data)
    m_rtc1_reset                             0x20000087   Data           1  app_timer.o(.data)
    .data                                    0x20000088   Section        8  retarget.o(.data)
    .data                                    0x20000090   Section       72  nrf_esb.o(.data)
    m_esb_initialized                        0x20000090   Data           1  nrf_esb.o(.data)
    m_nrf_esb_mainstate                      0x20000091   Data           1  nrf_esb.o(.data)
    mp_current_payload                       0x20000094   Data           4  nrf_esb.o(.data)
    m_event_handler                          0x20000098   Data           4  nrf_esb.o(.data)
    m_esb_addr                               0x2000009c   Data          20  nrf_esb.o(.data)
    m_interrupt_flags                        0x200000b0   Data           4  nrf_esb.o(.data)
    m_pids                                   0x200000b4   Data           8  nrf_esb.o(.data)
    m_retransmits_remaining                  0x200000bc   Data           4  nrf_esb.o(.data)
    m_last_tx_attempts                       0x200000c0   Data           4  nrf_esb.o(.data)
    m_wait_for_ack_timeout_us                0x200000c4   Data           4  nrf_esb.o(.data)
    m_radio_shorts_common                    0x200000c8   Data           4  nrf_esb.o(.data)
    on_radio_disabled                        0x200000cc   Data           4  nrf_esb.o(.data)
    on_radio_end                             0x200000d0   Data           4  nrf_esb.o(.data)
    update_rf_payload_format                 0x200000d4   Data           4  nrf_esb.o(.data)
    .data                                    0x200000d8   Section        1  uartprocess.o(.data)
    index                                    0x200000d8   Data           1  uartprocess.o(.data)
    .data                                    0x200000dc   Section        4  system_nrf52.o(.data)
    __tagsym$$used                           0x200000dc   Number         0  system_nrf52.o(.data)
    .bss                                     0x200000e0   Section       32  host.o(.bss)
    Timer_1S_timer_id_data                   0x200000e0   Data          32  host.o(.bss)
    .bss                                     0x20000100   Section      510  esbprocess.o(.bss)
    .bss                                     0x20000300   Section       44  nrfx_uart.o(.bss)
    m_cb                                     0x20000300   Data          44  nrfx_uart.o(.bss)
    .bss                                     0x2000032c   Section       36  nrfx_uarte.o(.bss)
    m_cb                                     0x2000032c   Data          36  nrfx_uarte.o(.bss)
    .bss                                     0x20000350   Section       76  nrfx_gpiote.o(.bss)
    m_cb                                     0x20000350   Data          76  nrfx_gpiote.o(.bss)
    .bss                                     0x2000039c   Section       32  app_uart_fifo.o(.bss)
    m_rx_fifo                                0x2000039c   Data          16  app_uart_fifo.o(.bss)
    m_tx_fifo                                0x200003ac   Data          16  app_uart_fifo.o(.bss)
    .bss                                     0x200003bc   Section      268  app_timer.o(.bss)
    m_op_queue                               0x200003bc   Data         268  app_timer.o(.bss)
    .bss                                     0x200004c8   Section     4728  nrf_esb.o(.bss)
    m_config_local                           0x200004c8   Data          24  nrf_esb.o(.bss)
    m_tx_fifo_payload                        0x200004e0   Data        2040  nrf_esb.o(.bss)
    m_tx_fifo                                0x20000cd8   Data          44  nrf_esb.o(.bss)
    m_rx_fifo_payload                        0x20000d04   Data        2040  nrf_esb.o(.bss)
    m_rx_fifo                                0x200014fc   Data          44  nrf_esb.o(.bss)
    m_tx_payload_buffer                      0x20001528   Data         252  nrf_esb.o(.bss)
    m_rx_payload_buffer                      0x20001624   Data         252  nrf_esb.o(.bss)
    m_rx_pipe_info                           0x20001720   Data          32  nrf_esb.o(.bss)
    .bss                                     0x20001740   Section     2064  uartprocess.o(.bss)
    data_array                               0x20001740   Data          16  uartprocess.o(.bss)
    rx_buf                                   0x20001750   Data        1024  uartprocess.o(.bss)
    tx_buf                                   0x20001b50   Data        1024  uartprocess.o(.bss)
    STACK                                    0x20001f50   Section     8192  arm_startup_nrf52.o(STACK)

    Global Symbols

    Symbol Name                              Value     Ov Type        Size  Object(Section)

    BuildAttributes$$THM_ISAv4$E$P$D$K$B$S$7EM$VFPi3$EXTD16$VFPS$VFMA$PE$A:L22UL41UL21$X:L11$S22US41US21$IEEE1$IW$USESV6$~STKCKD$USESV7$~SHL$OSPACE$ROPI$EBA8$MICROLIB$REQ8$EABIv2 0x00000000   Number         0  anon$$obj.o ABSOLUTE
    __ARM_use_no_argv                        0x00000000   Number         0  host.o ABSOLUTE
    __Vectors                                0x00000000   Data           4  arm_startup_nrf52.o(RESET)
    _printf_a                                0x00000000   Number         0  stubs.o ABSOLUTE
    _printf_c                                0x00000000   Number         0  stubs.o ABSOLUTE
    _printf_charcount                        0x00000000   Number         0  stubs.o ABSOLUTE
    _printf_d                                0x00000000   Number         0  stubs.o ABSOLUTE
    _printf_e                                0x00000000   Number         0  stubs.o ABSOLUTE
    _printf_f                                0x00000000   Number         0  stubs.o ABSOLUTE
    _printf_flags                            0x00000000   Number         0  stubs.o ABSOLUTE
    _printf_fp_dec                           0x00000000   Number         0  stubs.o ABSOLUTE
    _printf_fp_hex                           0x00000000   Number         0  stubs.o ABSOLUTE
    _printf_g                                0x00000000   Number         0  stubs.o ABSOLUTE
    _printf_i                                0x00000000   Number         0  stubs.o ABSOLUTE
    _printf_int_dec                          0x00000000   Number         0  stubs.o ABSOLUTE
    _printf_l                                0x00000000   Number         0  stubs.o ABSOLUTE
    _printf_lc                               0x00000000   Number         0  stubs.o ABSOLUTE
    _printf_ll                               0x00000000   Number         0  stubs.o ABSOLUTE
    _printf_lld                              0x00000000   Number         0  stubs.o ABSOLUTE
    _printf_lli                              0x00000000   Number         0  stubs.o ABSOLUTE
    _printf_llo                              0x00000000   Number         0  stubs.o ABSOLUTE
    _printf_llu                              0x00000000   Number         0  stubs.o ABSOLUTE
    _printf_llx                              0x00000000   Number         0  stubs.o ABSOLUTE
    _printf_longlong_dec                     0x00000000   Number         0  stubs.o ABSOLUTE
    _printf_longlong_hex                     0x00000000   Number         0  stubs.o ABSOLUTE
    _printf_longlong_oct                     0x00000000   Number         0  stubs.o ABSOLUTE
    _printf_ls                               0x00000000   Number         0  stubs.o ABSOLUTE
    _printf_mbtowc                           0x00000000   Number         0  stubs.o ABSOLUTE
    _printf_n                                0x00000000   Number         0  stubs.o ABSOLUTE
    _printf_o                                0x00000000   Number         0  stubs.o ABSOLUTE
    _printf_p                                0x00000000   Number         0  stubs.o ABSOLUTE
    _printf_percent                          0x00000000   Number         0  stubs.o ABSOLUTE
    _printf_pre_padding                      0x00000000   Number         0  stubs.o ABSOLUTE
    _printf_return_value                     0x00000000   Number         0  stubs.o ABSOLUTE
    _printf_s                                0x00000000   Number         0  stubs.o ABSOLUTE
    _printf_sizespec                         0x00000000   Number         0  stubs.o ABSOLUTE
    _printf_str                              0x00000000   Number         0  stubs.o ABSOLUTE
    _printf_truncate_signed                  0x00000000   Number         0  stubs.o ABSOLUTE
    _printf_truncate_unsigned                0x00000000   Number         0  stubs.o ABSOLUTE
    _printf_u                                0x00000000   Number         0  stubs.o ABSOLUTE
    _printf_wc                               0x00000000   Number         0  stubs.o ABSOLUTE
    _printf_wctomb                           0x00000000   Number         0  stubs.o ABSOLUTE
    _printf_widthprec                        0x00000000   Number         0  stubs.o ABSOLUTE
    _printf_x                                0x00000000   Number         0  stubs.o ABSOLUTE
    __cpp_initialize__aeabi_                  - Undefined Weak Reference
    __cxa_finalize                            - Undefined Weak Reference
    __decompress                              - Undefined Weak Reference
    _clock_init                               - Undefined Weak Reference
    _microlib_exit                            - Undefined Weak Reference
    __Vectors_End                            0x00000200   Data           0  arm_startup_nrf52.o(RESET)
    __Vectors_Size                           0x00000200   Number         0  arm_startup_nrf52.o ABSOLUTE
    __main                                   0x00000201   Thumb Code     0  entry.o(.ARM.Collect$$$$00000000)
    _main_stk                                0x00000201   Thumb Code     0  entry2.o(.ARM.Collect$$$$00000001)
    _main_scatterload                        0x00000205   Thumb Code     0  entry5.o(.ARM.Collect$$$$00000004)
    __main_after_scatterload                 0x00000209   Thumb Code     0  entry5.o(.ARM.Collect$$$$00000004)
    _main_clock                              0x00000209   Thumb Code     0  entry7b.o(.ARM.Collect$$$$00000008)
    _main_cpp_init                           0x00000209   Thumb Code     0  entry8b.o(.ARM.Collect$$$$0000000A)
    _main_init                               0x00000209   Thumb Code     0  entry9a.o(.ARM.Collect$$$$0000000B)
    __rt_final_cpp                           0x00000211   Thumb Code     0  entry10a.o(.ARM.Collect$$$$0000000D)
    __rt_final_exit                          0x00000211   Thumb Code     0  entry11a.o(.ARM.Collect$$$$0000000F)
    Reset_Handler                            0x00000215   Thumb Code     8  arm_startup_nrf52.o(.text)
    NMI_Handler                              0x0000021d   Thumb Code     2  arm_startup_nrf52.o(.text)
    HardFault_Handler                        0x0000021f   Thumb Code     2  arm_startup_nrf52.o(.text)
    MemoryManagement_Handler                 0x00000221   Thumb Code     2  arm_startup_nrf52.o(.text)
    BusFault_Handler                         0x00000223   Thumb Code     2  arm_startup_nrf52.o(.text)
    UsageFault_Handler                       0x00000225   Thumb Code     2  arm_startup_nrf52.o(.text)
    SVC_Handler                              0x00000227   Thumb Code     2  arm_startup_nrf52.o(.text)
    DebugMon_Handler                         0x00000229   Thumb Code     2  arm_startup_nrf52.o(.text)
    PendSV_Handler                           0x0000022b   Thumb Code     2  arm_startup_nrf52.o(.text)
    SysTick_Handler                          0x0000022d   Thumb Code     2  arm_startup_nrf52.o(.text)
    CCM_AAR_IRQHandler                       0x0000022f   Thumb Code     0  arm_startup_nrf52.o(.text)
    COMP_LPCOMP_IRQHandler                   0x0000022f   Thumb Code     0  arm_startup_nrf52.o(.text)
    ECB_IRQHandler                           0x0000022f   Thumb Code     0  arm_startup_nrf52.o(.text)
    FPU_IRQHandler                           0x0000022f   Thumb Code     0  arm_startup_nrf52.o(.text)
    I2S_IRQHandler                           0x0000022f   Thumb Code     0  arm_startup_nrf52.o(.text)
    MWU_IRQHandler                           0x0000022f   Thumb Code     0  arm_startup_nrf52.o(.text)
    NFCT_IRQHandler                          0x0000022f   Thumb Code     0  arm_startup_nrf52.o(.text)
    PDM_IRQHandler                           0x0000022f   Thumb Code     0  arm_startup_nrf52.o(.text)
    POWER_CLOCK_IRQHandler                   0x0000022f   Thumb Code     0  arm_startup_nrf52.o(.text)
    PWM0_IRQHandler                          0x0000022f   Thumb Code     0  arm_startup_nrf52.o(.text)
    PWM1_IRQHandler                          0x0000022f   Thumb Code     0  arm_startup_nrf52.o(.text)
    PWM2_IRQHandler                          0x0000022f   Thumb Code     0  arm_startup_nrf52.o(.text)
    QDEC_IRQHandler                          0x0000022f   Thumb Code     0  arm_startup_nrf52.o(.text)
    RNG_IRQHandler                           0x0000022f   Thumb Code     0  arm_startup_nrf52.o(.text)
    RTC0_IRQHandler                          0x0000022f   Thumb Code     0  arm_startup_nrf52.o(.text)
    RTC2_IRQHandler                          0x0000022f   Thumb Code     0  arm_startup_nrf52.o(.text)
    SAADC_IRQHandler                         0x0000022f   Thumb Code     0  arm_startup_nrf52.o(.text)
    SPIM0_SPIS0_TWIM0_TWIS0_SPI0_TWI0_IRQHandler 0x0000022f   Thumb Code     0  arm_startup_nrf52.o(.text)
    SPIM1_SPIS1_TWIM1_TWIS1_SPI1_TWI1_IRQHandler 0x0000022f   Thumb Code     0  arm_startup_nrf52.o(.text)
    SPIM2_SPIS2_SPI2_IRQHandler              0x0000022f   Thumb Code     0  arm_startup_nrf52.o(.text)
    SWI2_EGU2_IRQHandler                     0x0000022f   Thumb Code     0  arm_startup_nrf52.o(.text)
    SWI3_EGU3_IRQHandler                     0x0000022f   Thumb Code     0  arm_startup_nrf52.o(.text)
    SWI4_EGU4_IRQHandler                     0x0000022f   Thumb Code     0  arm_startup_nrf52.o(.text)
    SWI5_EGU5_IRQHandler                     0x0000022f   Thumb Code     0  arm_startup_nrf52.o(.text)
    TEMP_IRQHandler                          0x0000022f   Thumb Code     0  arm_startup_nrf52.o(.text)
    TIMER0_IRQHandler                        0x0000022f   Thumb Code     0  arm_startup_nrf52.o(.text)
    TIMER1_IRQHandler                        0x0000022f   Thumb Code     0  arm_startup_nrf52.o(.text)
    TIMER2_IRQHandler                        0x0000022f   Thumb Code     0  arm_startup_nrf52.o(.text)
    TIMER4_IRQHandler                        0x0000022f   Thumb Code     0  arm_startup_nrf52.o(.text)
    WDT_IRQHandler                           0x0000022f   Thumb Code     0  arm_startup_nrf52.o(.text)
    __aeabi_memcpy                           0x00000239   Thumb Code    36  memcpya.o(.text)
    __aeabi_memcpy4                          0x00000239   Thumb Code     0  memcpya.o(.text)
    __aeabi_memcpy8                          0x00000239   Thumb Code     0  memcpya.o(.text)
    __aeabi_memset                           0x0000025d   Thumb Code    14  memseta.o(.text)
    __aeabi_memset4                          0x0000025d   Thumb Code     0  memseta.o(.text)
    __aeabi_memset8                          0x0000025d   Thumb Code     0  memseta.o(.text)
    __aeabi_memclr                           0x0000026b   Thumb Code     4  memseta.o(.text)
    __aeabi_memclr4                          0x0000026b   Thumb Code     0  memseta.o(.text)
    __aeabi_memclr8                          0x0000026b   Thumb Code     0  memseta.o(.text)
    _memset$wrapper                          0x0000026f   Thumb Code    18  memseta.o(.text)
    memcmp                                   0x00000281   Thumb Code    26  memcmp.o(.text)
    __aeabi_uidiv                            0x0000029b   Thumb Code     0  uidiv.o(.text)
    __aeabi_uidivmod                         0x0000029b   Thumb Code    44  uidiv.o(.text)
    __scatterload                            0x000002c9   Thumb Code    28  init.o(.text)
    __scatterload_rt2                        0x000002c9   Thumb Code     0  init.o(.text)
    Action_Key1                              0x000002ed   Thumb Code    30  host.o(i.Action_Key1)
    GPIOTE_IRQHandler                        0x0000030d   Thumb Code   528  nrfx_gpiote.o(i.GPIOTE_IRQHandler)
    PacketSend                               0x0000061d   Thumb Code    56  host.o(i.PacketSend)
    Pin_Trigger_handler_1                    0x00000655   Thumb Code    66  gpioprocess.o(i.Pin_Trigger_handler_1)
    Pin_Trigger_handler_2                    0x000006ad   Thumb Code    38  gpioprocess.o(i.Pin_Trigger_handler_2)
    RADIO_IRQHandler                         0x0000071d   Thumb Code   102  nrf_esb.o(i.RADIO_IRQHandler)
    RTC1_IRQHandler                          0x00000795   Thumb Code    44  app_timer.o(i.RTC1_IRQHandler)
    SWI0_EGU0_IRQHandler                     0x000007c9   Thumb Code    92  nrf_esb.o(i.SWI0_EGU0_IRQHandler)
    SWI1_EGU1_IRQHandler                     0x0000082d   Thumb Code     8  app_timer.o(i.SWI1_EGU1_IRQHandler)
    SystemCoreClockUpdate                    0x00000835   Thumb Code     8  system_nrf52.o(i.SystemCoreClockUpdate)
    SystemInit                               0x00000845   Thumb Code   596  system_nrf52.o(i.SystemInit)
    TIMER3_IRQHandler                        0x00000add   Thumb Code    28  nrf_esb.o(i.TIMER3_IRQHandler)
    Timer_1S                                 0x00000b05   Thumb Code    48  host.o(i.Timer_1S)
    UARTE0_UART0_IRQHandler                  0x00000b3d   Thumb Code    10  nrfx_prs.o(i.UARTE0_UART0_IRQHandler)
    UART_Init                                0x00000b4d   Thumb Code    74  uartprocess.o(i.UART_Init)
    __0printf$1                              0x00000ba9   Thumb Code    22  printf1.o(i.__0printf$1)
    __1printf$1                              0x00000ba9   Thumb Code     0  printf1.o(i.__0printf$1)
    __2printf                                0x00000ba9   Thumb Code     0  printf1.o(i.__0printf$1)
    __scatterload_copy                       0x00000bc9   Thumb Code    14  handlers.o(i.__scatterload_copy)
    __scatterload_null                       0x00000bd7   Thumb Code     2  handlers.o(i.__scatterload_null)
    __scatterload_zeroinit                   0x00000bd9   Thumb Code    14  handlers.o(i.__scatterload_zeroinit)
    app_error_fault_handler                  0x00000d4d   Thumb Code    82  app_error_weak.o(i.app_error_fault_handler)
    app_error_handler_bare                   0x00000da9   Thumb Code    28  app_error.o(i.app_error_handler_bare)
    app_fifo_get                             0x00000dc5   Thumb Code    30  app_fifo.o(i.app_fifo_get)
    app_fifo_init                            0x00000de3   Thumb Code    36  app_fifo.o(i.app_fifo_init)
    app_fifo_put                             0x00000e07   Thumb Code    34  app_fifo.o(i.app_fifo_put)
    app_timer_create                         0x00000e29   Thumb Code    56  app_timer.o(i.app_timer_create)
    app_timer_init                           0x00000e65   Thumb Code    70  app_timer.o(i.app_timer_init)
    app_timer_start                          0x00000ec1   Thumb Code    78  app_timer.o(i.app_timer_start)
    app_uart_get                             0x00000f15   Thumb Code    66  app_uart_fifo.o(i.app_uart_get)
    app_uart_init                            0x00000f69   Thumb Code   188  app_uart_fifo.o(i.app_uart_init)
    app_uart_put                             0x00001045   Thumb Code    90  app_uart_fifo.o(i.app_uart_put)
    app_util_critical_region_enter           0x000010b1   Thumb Code    10  app_util_platform.o(i.app_util_critical_region_enter)
    app_util_critical_region_exit            0x000010bb   Thumb Code    10  app_util_platform.o(i.app_util_critical_region_exit)
    app_util_disable_irq                     0x000010c5   Thumb Code    14  app_util_platform.o(i.app_util_disable_irq)
    app_util_enable_irq                      0x000010d9   Thumb Code    20  app_util_platform.o(i.app_util_enable_irq)
    clocks_start                             0x00001459   Thumb Code    24  host.o(i.clocks_start)
    esb_init                                 0x0000181d   Thumb Code   184  esbprocess.o(i.esb_init)
    esb_packet_received                      0x000018f5   Thumb Code   110  host.o(i.esb_packet_received)
    esb_packet_send                          0x00001979   Thumb Code   102  esbprocess.o(i.esb_packet_send)
    fputc                                    0x00001a9d   Thumb Code    16  retarget.o(i.fputc)
    gpio_init                                0x00001aad   Thumb Code   164  gpioprocess.o(i.gpio_init)
    main                                     0x00001e05   Thumb Code    68  host.o(i.main)
    nrf_drv_uart_init                        0x00001e91   Thumb Code   118  nrf_drv_uart.o(i.nrf_drv_uart_init)
    nrf_esb_disable                          0x00001fa5   Thumb Code    56  nrf_esb.o(i.nrf_esb_disable)
    nrf_esb_event_handler                    0x00001ff5   Thumb Code   106  esbprocess.o(i.nrf_esb_event_handler)
    nrf_esb_init                             0x000020b9   Thumb Code   200  nrf_esb.o(i.nrf_esb_init)
    nrf_esb_read_rx_payload                  0x000021b1   Thumb Code   164  nrf_esb.o(i.nrf_esb_read_rx_payload)
    nrf_esb_set_base_address_0               0x0000225d   Thumb Code   102  nrf_esb.o(i.nrf_esb_set_base_address_0)
    nrf_esb_set_base_address_1               0x000022d9   Thumb Code   170  nrf_esb.o(i.nrf_esb_set_base_address_1)
    nrf_esb_set_prefixes                     0x00002399   Thumb Code   166  nrf_esb.o(i.nrf_esb_set_prefixes)
    nrf_esb_set_rf_channel                   0x00002455   Thumb Code    36  nrf_esb.o(i.nrf_esb_set_rf_channel)
    nrf_esb_skip_tx                          0x00002481   Thumb Code    74  nrf_esb.o(i.nrf_esb_skip_tx)
    nrf_esb_start_rx                         0x000024d5   Thumb Code   128  nrf_esb.o(i.nrf_esb_start_rx)
    nrf_esb_start_tx                         0x0000257d   Thumb Code    36  nrf_esb.o(i.nrf_esb_start_tx)
    nrf_esb_stop_rx                          0x000025a9   Thumb Code    74  nrf_esb.o(i.nrf_esb_stop_rx)
    nrf_esb_write_payload                    0x00002605   Thumb Code   220  nrf_esb.o(i.nrf_esb_write_payload)
    nrfx_gpiote_in_event_enable              0x000029f5   Thumb Code   164  nrfx_gpiote.o(i.nrfx_gpiote_in_event_enable)
    nrfx_gpiote_in_init                      0x00002aa1   Thumb Code   232  nrfx_gpiote.o(i.nrfx_gpiote_in_init)
    nrfx_gpiote_init                         0x00002b95   Thumb Code   162  nrfx_gpiote.o(i.nrfx_gpiote_init)
    nrfx_prs_acquire                         0x00002c59   Thumb Code    72  nrfx_prs.o(i.nrfx_prs_acquire)
    nrfx_uart_0_irq_handler                  0x00002ca1   Thumb Code    12  nrfx_uart.o(i.nrfx_uart_0_irq_handler)
    nrfx_uart_init                           0x00002cb5   Thumb Code   128  nrfx_uart.o(i.nrfx_uart_init)
    nrfx_uart_rx                             0x00002d3d   Thumb Code   286  nrfx_uart.o(i.nrfx_uart_rx)
    nrfx_uart_tx                             0x00002e61   Thumb Code   134  nrfx_uart.o(i.nrfx_uart_tx)
    nrfx_uart_tx_in_progress                 0x00002eed   Thumb Code    30  nrfx_uart.o(i.nrfx_uart_tx_in_progress)
    nrfx_uarte_0_irq_handler                 0x00002f11   Thumb Code    12  nrfx_uarte.o(i.nrfx_uarte_0_irq_handler)
    nrfx_uarte_init                          0x00002f25   Thumb Code   120  nrfx_uarte.o(i.nrfx_uarte_init)
    nrfx_uarte_rx                            0x00002fa5   Thumb Code   306  nrfx_uarte.o(i.nrfx_uarte_rx)
    nrfx_uarte_tx                            0x000030dd   Thumb Code   162  nrfx_uarte.o(i.nrfx_uarte_tx)
    nrfx_uarte_tx_in_progress                0x00003185   Thumb Code    26  nrfx_uarte.o(i.nrfx_uarte_tx_in_progress)
    uart_event_handle                        0x00003ea1   Thumb Code   284  uartprocess.o(i.uart_event_handle)
    Region$$Table$$Base                      0x000046e0   Number         0  anon$$obj.o(Region$$Table)
    Region$$Table$$Limit                     0x00004700   Number         0  anon$$obj.o(Region$$Table)
    UICR_ADDR_0x20C                          0x1000120c   Data           4  gpioprocess.o(.ARM.__AT_0x1000120C)
    KeyDebunseTick                           0x20000000   Data           1  gpioprocess.o(.data)
    RxLedFlashCnt                            0x20000004   Data           4  host.o(.data)
    TriggerPressed                           0x20000008   Data           1  host.o(.data)
    TriggerPressedFlag                       0x20000009   Data           1  host.o(.data)
    nrf_esb_config                           0x2000000c   Data          24  esbprocess.o(.data)
    rx_callback                              0x20000024   Data           4  esbprocess.o(.data)
    radio_tx_busy                            0x20000028   Data           1  esbprocess.o(.data)
    radio_started                            0x20000029   Data           1  esbprocess.o(.data)
    PacketSendCnt                            0x2000002c   Data           4  esbprocess.o(.data)
    PacketSendOKCnt                          0x20000030   Data           4  esbprocess.o(.data)
    PacketSentNGCnt                          0x20000034   Data           4  esbprocess.o(.data)
    PacketReceiveOKCnt                       0x20000038   Data           4  esbprocess.o(.data)
    PacketReceiveNGCnt                       0x2000003c   Data           4  esbprocess.o(.data)
    nrf_drv_uart_use_easy_dma                0x20000048   Data           1  nrf_drv_uart.o(.data)
    __stdout                                 0x20000088   Data           4  retarget.o(.data)
    __stdin                                  0x2000008c   Data           4  retarget.o(.data)
    SystemCoreClock                          0x200000dc   Data           4  system_nrf52.o(.data)
    tx_payload                               0x20000100   Data         255  esbprocess.o(.bss)
    rx_payload                               0x200001ff   Data         255  esbprocess.o(.bss)
    __initial_sp                             0x20003f50   Data           0  arm_startup_nrf52.o(STACK)



==============================================================================

Memory Map of the image

  Image Entry point : 0x00000201

  Load Region LR_IROM1 (Base: 0x00000000, Size: 0x000047e0, Max: 0x00080000, ABSOLUTE)

    Execution Region ER_IROM1 (Exec base: 0x00000000, Load base: 0x00000000, Size: 0x00004700, Max: 0x00080000, ABSOLUTE)

    Exec Addr    Load Addr    Size         Type   Attr      Idx    E Section Name        Object

    0x00000000   0x00000000   0x00000200   Data   RO         2939    RESET               arm_startup_nrf52.o
    0x00000200   0x00000200   0x00000000   Code   RO         3035  * .ARM.Collect$$$$00000000  mc_w.l(entry.o)
    0x00000200   0x00000200   0x00000004   Code   RO         3309    .ARM.Collect$$$$00000001  mc_w.l(entry2.o)
    0x00000204   0x00000204   0x00000004   Code   RO         3312    .ARM.Collect$$$$00000004  mc_w.l(entry5.o)
    0x00000208   0x00000208   0x00000000   Code   RO         3314    .ARM.Collect$$$$00000008  mc_w.l(entry7b.o)
    0x00000208   0x00000208   0x00000000   Code   RO         3316    .ARM.Collect$$$$0000000A  mc_w.l(entry8b.o)
    0x00000208   0x00000208   0x00000008   Code   RO         3317    .ARM.Collect$$$$0000000B  mc_w.l(entry9a.o)
    0x00000210   0x00000210   0x00000000   Code   RO         3319    .ARM.Collect$$$$0000000D  mc_w.l(entry10a.o)
    0x00000210   0x00000210   0x00000000   Code   RO         3321    .ARM.Collect$$$$0000000F  mc_w.l(entry11a.o)
    0x00000210   0x00000210   0x00000004   Code   RO         3310    .ARM.Collect$$$$00002712  mc_w.l(entry2.o)
    0x00000214   0x00000214   0x00000024   Code   RO         2940    .text               arm_startup_nrf52.o
    0x00000238   0x00000238   0x00000024   Code   RO         3038    .text               mc_w.l(memcpya.o)
    0x0000025c   0x0000025c   0x00000024   Code   RO         3040    .text               mc_w.l(memseta.o)
    0x00000280   0x00000280   0x0000001a   Code   RO         3044    .text               mc_w.l(memcmp.o)
    0x0000029a   0x0000029a   0x0000002c   Code   RO         3323    .text               mc_w.l(uidiv.o)
    0x000002c6   0x000002c6   0x00000002   PAD
    0x000002c8   0x000002c8   0x00000024   Code   RO         3338    .text               mc_w.l(init.o)
    0x000002ec   0x000002ec   0x0000001e   Code   RO          232    i.Action_Key1       host.o
    0x0000030a   0x0000030a   0x00000002   PAD
    0x0000030c   0x0000030c   0x0000021c   Code   RO         1121    i.GPIOTE_IRQHandler  nrfx_gpiote.o
    0x00000528   0x00000528   0x00000018   Code   RO         2253    i.NVIC_ClearPendingIRQ  app_timer.o
    0x00000540   0x00000540   0x00000018   Code   RO         2554    i.NVIC_ClearPendingIRQ  nrf_esb.o
    0x00000558   0x00000558   0x00000018   Code   RO         2555    i.NVIC_DisableIRQ   nrf_esb.o
    0x00000570   0x00000570   0x00000016   Code   RO         2254    i.NVIC_EnableIRQ    app_timer.o
    0x00000586   0x00000586   0x00000016   Code   RO         2556    i.NVIC_EnableIRQ    nrf_esb.o
    0x0000059c   0x0000059c   0x00000018   Code   RO         2255    i.NVIC_SetPendingIRQ  app_timer.o
    0x000005b4   0x000005b4   0x00000018   Code   RO         2557    i.NVIC_SetPendingIRQ  nrf_esb.o
    0x000005cc   0x000005cc   0x00000028   Code   RO         2256    i.NVIC_SetPriority  app_timer.o
    0x000005f4   0x000005f4   0x00000028   Code   RO         2558    i.NVIC_SetPriority  nrf_esb.o
    0x0000061c   0x0000061c   0x00000038   Code   RO          233    i.PacketSend        host.o
    0x00000654   0x00000654   0x00000058   Code   RO            4    i.Pin_Trigger_handler_1  gpioprocess.o
    0x000006ac   0x000006ac   0x00000070   Code   RO            5    i.Pin_Trigger_handler_2  gpioprocess.o
    0x0000071c   0x0000071c   0x00000078   Code   RO         2559    i.RADIO_IRQHandler  nrf_esb.o
    0x00000794   0x00000794   0x00000034   Code   RO         2257    i.RTC1_IRQHandler   app_timer.o
    0x000007c8   0x000007c8   0x00000064   Code   RO         2560    i.SWI0_EGU0_IRQHandler  nrf_esb.o
    0x0000082c   0x0000082c   0x00000008   Code   RO         2258    i.SWI1_EGU1_IRQHandler  app_timer.o
    0x00000834   0x00000834   0x00000010   Code   RO         2947    i.SystemCoreClockUpdate  system_nrf52.o
    0x00000844   0x00000844   0x00000298   Code   RO         2948    i.SystemInit        system_nrf52.o
    0x00000adc   0x00000adc   0x00000028   Code   RO         2561    i.TIMER3_IRQHandler  nrf_esb.o
    0x00000b04   0x00000b04   0x00000038   Code   RO          234    i.Timer_1S          host.o
    0x00000b3c   0x00000b3c   0x00000010   Code   RO          598    i.UARTE0_UART0_IRQHandler  nrfx_prs.o
    0x00000b4c   0x00000b4c   0x0000005c   Code   RO         2897    i.UART_Init         uartprocess.o
    0x00000ba8   0x00000ba8   0x00000020   Code   RO         3093    i.__0printf$1       mc_w.l(printf1.o)
    0x00000bc8   0x00000bc8   0x0000000e   Code   RO         3350    i.__scatterload_copy  mc_w.l(handlers.o)
    0x00000bd6   0x00000bd6   0x00000002   Code   RO         3351    i.__scatterload_null  mc_w.l(handlers.o)
    0x00000bd8   0x00000bd8   0x0000000e   Code   RO         3352    i.__scatterload_zeroinit  mc_w.l(handlers.o)
    0x00000be6   0x00000be6   0x00000002   PAD
    0x00000be8   0x00000be8   0x00000154   Code   RO         3100    i._printf_core      mc_w.l(printf1.o)
    0x00000d3c   0x00000d3c   0x0000000e   Code   RO         2562    i.addr_conv         nrf_esb.o
    0x00000d4a   0x00000d4a   0x00000002   PAD
    0x00000d4c   0x00000d4c   0x0000005c   Code   RO         1499    i.app_error_fault_handler  app_error_weak.o
    0x00000da8   0x00000da8   0x0000001c   Code   RO         1439    i.app_error_handler_bare  app_error.o
    0x00000dc4   0x00000dc4   0x0000001e   Code   RO         1537    i.app_fifo_get      app_fifo.o
    0x00000de2   0x00000de2   0x00000024   Code   RO         1538    i.app_fifo_init     app_fifo.o
    0x00000e06   0x00000e06   0x00000022   Code   RO         1540    i.app_fifo_put      app_fifo.o
    0x00000e28   0x00000e28   0x0000003c   Code   RO         2261    i.app_timer_create  app_timer.o
    0x00000e64   0x00000e64   0x0000005c   Code   RO         2262    i.app_timer_init    app_timer.o
    0x00000ec0   0x00000ec0   0x00000054   Code   RO         2265    i.app_timer_start   app_timer.o
    0x00000f14   0x00000f14   0x00000054   Code   RO         1624    i.app_uart_get      app_uart_fifo.o
    0x00000f68   0x00000f68   0x000000dc   Code   RO         1625    i.app_uart_init     app_uart_fifo.o
    0x00001044   0x00001044   0x0000006c   Code   RO         1626    i.app_uart_put      app_uart_fifo.o
    0x000010b0   0x000010b0   0x0000000a   Code   RO         1710    i.app_util_critical_region_enter  app_util_platform.o
    0x000010ba   0x000010ba   0x0000000a   Code   RO         1711    i.app_util_critical_region_exit  app_util_platform.o
    0x000010c4   0x000010c4   0x00000014   Code   RO         1712    i.app_util_disable_irq  app_util_platform.o
    0x000010d8   0x000010d8   0x00000018   Code   RO         1713    i.app_util_enable_irq  app_util_platform.o
    0x000010f0   0x000010f0   0x0000013c   Code   RO         2563    i.apply_address_workarounds  nrf_esb.o
    0x0000122c   0x0000122c   0x0000007c   Code   RO          658    i.apply_config      nrfx_uart.o
    0x000012a8   0x000012a8   0x0000007c   Code   RO          907    i.apply_config      nrfx_uarte.o
    0x00001324   0x00001324   0x0000000c   Code   RO         2564    i.bytewise_bit_swap  nrf_esb.o
    0x00001330   0x00001330   0x00000020   Code   RO         1122    i.channel_free      nrfx_gpiote.o
    0x00001350   0x00001350   0x00000010   Code   RO         1123    i.channel_handler_get  nrfx_gpiote.o
    0x00001360   0x00001360   0x00000080   Code   RO         1124    i.channel_port_alloc  nrfx_gpiote.o
    0x000013e0   0x000013e0   0x0000000c   Code   RO         1125    i.channel_port_get  nrfx_gpiote.o
    0x000013ec   0x000013ec   0x0000006c   Code   RO         2565    i.clear_events_restart_rx  nrf_esb.o
    0x00001458   0x00001458   0x0000001c   Code   RO          235    i.clocks_start      host.o
    0x00001474   0x00001474   0x00000090   Code   RO         2268    i.compare_reg_update  app_timer.o
    0x00001504   0x00001504   0x00000064   Code   RO         2269    i.elapsed_ticks_acquire  app_timer.o
    0x00001568   0x00001568   0x00000054   Code   RO         2949    i.errata_108        system_nrf52.o
    0x000015bc   0x000015bc   0x00000054   Code   RO         2950    i.errata_12         system_nrf52.o
    0x00001610   0x00001610   0x00000054   Code   RO         2951    i.errata_136        system_nrf52.o
    0x00001664   0x00001664   0x00000030   Code   RO         2952    i.errata_16         system_nrf52.o
    0x00001694   0x00001694   0x00000020   Code   RO         2953    i.errata_182        system_nrf52.o
    0x000016b4   0x000016b4   0x00000054   Code   RO         2954    i.errata_31         system_nrf52.o
    0x00001708   0x00001708   0x00000030   Code   RO         2955    i.errata_32         system_nrf52.o
    0x00001738   0x00001738   0x00000054   Code   RO         2956    i.errata_36         system_nrf52.o
    0x0000178c   0x0000178c   0x00000030   Code   RO         2957    i.errata_37         system_nrf52.o
    0x000017bc   0x000017bc   0x00000030   Code   RO         2958    i.errata_57         system_nrf52.o
    0x000017ec   0x000017ec   0x00000030   Code   RO         2959    i.errata_66         system_nrf52.o
    0x0000181c   0x0000181c   0x000000d8   Code   RO          350    i.esb_init          esbprocess.o
    0x000018f4   0x000018f4   0x00000084   Code   RO          236    i.esb_packet_received  host.o
    0x00001978   0x00001978   0x0000007c   Code   RO          351    i.esb_packet_send   esbprocess.o
    0x000019f4   0x000019f4   0x00000058   Code   RO         2270    i.expired_timers_handler  app_timer.o
    0x00001a4c   0x00001a4c   0x00000018   Code   RO         1543    i.fifo_get          app_fifo.o
    0x00001a64   0x00001a64   0x0000000a   Code   RO         1544    i.fifo_length       app_fifo.o
    0x00001a6e   0x00001a6e   0x0000000a   Code   RO         1627    i.fifo_length       app_uart_fifo.o
    0x00001a78   0x00001a78   0x00000012   Code   RO         1545    i.fifo_peek         app_fifo.o
    0x00001a8a   0x00001a8a   0x00000012   Code   RO         1546    i.fifo_put          app_fifo.o
    0x00001a9c   0x00001a9c   0x00000010   Code   RO         2482    i.fputc             retarget.o
    0x00001aac   0x00001aac   0x000000b0   Code   RO            6    i.gpio_init         gpioprocess.o
    0x00001b5c   0x00001b5c   0x00000048   Code   RO         2566    i.initialize_fifos  nrf_esb.o
    0x00001ba4   0x00001ba4   0x00000088   Code   RO          660    i.interrupts_enable  nrfx_uart.o
    0x00001c2c   0x00001c2c   0x0000009c   Code   RO          909    i.interrupts_enable  nrfx_uarte.o
    0x00001cc8   0x00001cc8   0x0000013c   Code   RO         2271    i.list_insertions_handler  app_timer.o
    0x00001e04   0x00001e04   0x00000060   Code   RO          237    i.main              host.o
    0x00001e64   0x00001e64   0x00000016   Code   RO         1126    i.nrf_bitmask_bit_is_set  nrfx_gpiote.o
    0x00001e7a   0x00001e7a   0x00000016   Code   RO         1127    i.nrf_bitmask_bit_set  nrfx_gpiote.o
    0x00001e90   0x00001e90   0x0000008c   Code   RO          546    i.nrf_drv_uart_init  nrf_drv_uart.o
    0x00001f1c   0x00001f1c   0x00000044   Code   RO         1628    i.nrf_drv_uart_rx   app_uart_fifo.o
    0x00001f60   0x00001f60   0x00000044   Code   RO         1629    i.nrf_drv_uart_tx   app_uart_fifo.o
    0x00001fa4   0x00001fa4   0x00000050   Code   RO         2567    i.nrf_esb_disable   nrf_esb.o
    0x00001ff4   0x00001ff4   0x00000084   Code   RO          352    i.nrf_esb_event_handler  esbprocess.o
    0x00002078   0x00002078   0x00000040   Code   RO         2571    i.nrf_esb_get_clear_interrupts  nrf_esb.o
    0x000020b8   0x000020b8   0x000000f8   Code   RO         2573    i.nrf_esb_init      nrf_esb.o
    0x000021b0   0x000021b0   0x000000ac   Code   RO         2576    i.nrf_esb_read_rx_payload  nrf_esb.o
    0x0000225c   0x0000225c   0x0000007c   Code   RO         2579    i.nrf_esb_set_base_address_0  nrf_esb.o
    0x000022d8   0x000022d8   0x000000c0   Code   RO         2580    i.nrf_esb_set_base_address_1  nrf_esb.o
    0x00002398   0x00002398   0x000000bc   Code   RO         2582    i.nrf_esb_set_prefixes  nrf_esb.o
    0x00002454   0x00002454   0x0000002c   Code   RO         2585    i.nrf_esb_set_rf_channel  nrf_esb.o
    0x00002480   0x00002480   0x00000054   Code   RO         2587    i.nrf_esb_skip_tx   nrf_esb.o
    0x000024d4   0x000024d4   0x000000a8   Code   RO         2588    i.nrf_esb_start_rx  nrf_esb.o
    0x0000257c   0x0000257c   0x0000002c   Code   RO         2589    i.nrf_esb_start_tx  nrf_esb.o
    0x000025a8   0x000025a8   0x0000005c   Code   RO         2590    i.nrf_esb_stop_rx   nrf_esb.o
    0x00002604   0x00002604   0x000000f0   Code   RO         2593    i.nrf_esb_write_payload  nrf_esb.o
    0x000026f4   0x000026f4   0x00000028   Code   RO          661    i.nrf_gpio_cfg      nrfx_uart.o
    0x0000271c   0x0000271c   0x00000028   Code   RO          910    i.nrf_gpio_cfg      nrfx_uarte.o
    0x00002744   0x00002744   0x00000028   Code   RO         1128    i.nrf_gpio_cfg      nrfx_gpiote.o
    0x0000276c   0x0000276c   0x0000001a   Code   RO          663    i.nrf_gpio_cfg_input  nrfx_uart.o
    0x00002786   0x00002786   0x0000001a   Code   RO          912    i.nrf_gpio_cfg_input  nrfx_uarte.o
    0x000027a0   0x000027a0   0x00000030   Code   RO            7    i.nrf_gpio_cfg_output  gpioprocess.o
    0x000027d0   0x000027d0   0x00000018   Code   RO          664    i.nrf_gpio_cfg_output  nrfx_uart.o
    0x000027e8   0x000027e8   0x00000018   Code   RO          913    i.nrf_gpio_cfg_output  nrfx_uarte.o
    0x00002800   0x00002800   0x00000032   Code   RO         1130    i.nrf_gpio_cfg_sense_set  nrfx_gpiote.o
    0x00002832   0x00002832   0x00000016   Code   RO            8    i.nrf_gpio_pin_clear  gpioprocess.o
    0x00002848   0x00002848   0x00000018   Code   RO         1132    i.nrf_gpio_pin_read  nrfx_gpiote.o
    0x00002860   0x00002860   0x00000016   Code   RO          665    i.nrf_gpio_pin_set  nrfx_uart.o
    0x00002876   0x00002876   0x00000016   Code   RO          914    i.nrf_gpio_pin_set  nrfx_uarte.o
    0x0000288c   0x0000288c   0x00000028   Code   RO         1134    i.nrf_gpio_ports_read  nrfx_gpiote.o
    0x000028b4   0x000028b4   0x0000000c   Code   RO         1135    i.nrf_gpiote_event_addr_get  nrfx_gpiote.o
    0x000028c0   0x000028c0   0x0000001c   Code   RO         1136    i.nrf_gpiote_event_clear  nrfx_gpiote.o
    0x000028dc   0x000028dc   0x00000016   Code   RO         1137    i.nrf_gpiote_event_is_set  nrfx_gpiote.o
    0x000028f2   0x000028f2   0x00000002   PAD
    0x000028f4   0x000028f4   0x0000000c   Code   RO         1138    i.nrf_gpiote_int_enable  nrfx_gpiote.o
    0x00002900   0x00002900   0x0000000c   Code   RO          666    i.nrf_uart_errorsrc_get_and_clear  nrfx_uart.o
    0x0000290c   0x0000290c   0x0000000e   Code   RO          667    i.nrf_uart_event_check  nrfx_uart.o
    0x0000291a   0x0000291a   0x0000000e   Code   RO          668    i.nrf_uart_event_clear  nrfx_uart.o
    0x00002928   0x00002928   0x0000000a   Code   RO          669    i.nrf_uart_hwfc_pins_set  nrfx_uart.o
    0x00002932   0x00002932   0x00000006   Code   RO          670    i.nrf_uart_int_disable  nrfx_uart.o
    0x00002938   0x00002938   0x00000006   Code   RO          671    i.nrf_uart_int_enable  nrfx_uart.o
    0x0000293e   0x0000293e   0x00000012   Code   RO          672    i.nrf_uart_int_enable_check  nrfx_uart.o
    0x00002950   0x00002950   0x00000006   Code   RO          673    i.nrf_uart_task_trigger  nrfx_uart.o
    0x00002956   0x00002956   0x0000000a   Code   RO          674    i.nrf_uart_txrx_pins_set  nrfx_uart.o
    0x00002960   0x00002960   0x0000000c   Code   RO          915    i.nrf_uarte_errorsrc_get_and_clear  nrfx_uarte.o
    0x0000296c   0x0000296c   0x0000000e   Code   RO          916    i.nrf_uarte_event_check  nrfx_uarte.o
    0x0000297a   0x0000297a   0x0000000e   Code   RO          917    i.nrf_uarte_event_clear  nrfx_uarte.o
    0x00002988   0x00002988   0x0000000c   Code   RO          918    i.nrf_uarte_hwfc_pins_set  nrfx_uarte.o
    0x00002994   0x00002994   0x00000006   Code   RO          919    i.nrf_uarte_int_disable  nrfx_uarte.o
    0x0000299a   0x0000299a   0x00000006   Code   RO          920    i.nrf_uarte_int_enable  nrfx_uarte.o
    0x000029a0   0x000029a0   0x0000000a   Code   RO          921    i.nrf_uarte_rx_amount_get  nrfx_uarte.o
    0x000029aa   0x000029aa   0x0000000c   Code   RO          922    i.nrf_uarte_shorts_disable  nrfx_uarte.o
    0x000029b6   0x000029b6   0x00000006   Code   RO          923    i.nrf_uarte_task_trigger  nrfx_uarte.o
    0x000029bc   0x000029bc   0x0000000e   Code   RO          924    i.nrf_uarte_txrx_pins_set  nrfx_uarte.o
    0x000029ca   0x000029ca   0x00000002   PAD
    0x000029cc   0x000029cc   0x00000018   Code   RO         2272    i.nrfx_coredep_delay_us  app_timer.o
    0x000029e4   0x000029e4   0x00000008   Code   RO          675    i.nrfx_get_irq_number  nrfx_uart.o
    0x000029ec   0x000029ec   0x00000008   Code   RO          925    i.nrfx_get_irq_number  nrfx_uarte.o
    0x000029f4   0x000029f4   0x000000ac   Code   RO         1145    i.nrfx_gpiote_in_event_enable  nrfx_gpiote.o
    0x00002aa0   0x00002aa0   0x000000f4   Code   RO         1146    i.nrfx_gpiote_in_init  nrfx_gpiote.o
    0x00002b94   0x00002b94   0x000000b0   Code   RO         1149    i.nrfx_gpiote_init  nrfx_gpiote.o
    0x00002c44   0x00002c44   0x00000014   Code   RO          926    i.nrfx_is_in_ram    nrfx_uarte.o
    0x00002c58   0x00002c58   0x00000048   Code   RO          599    i.nrfx_prs_acquire  nrfx_prs.o
    0x00002ca0   0x00002ca0   0x00000014   Code   RO          676    i.nrfx_uart_0_irq_handler  nrfx_uart.o
    0x00002cb4   0x00002cb4   0x00000088   Code   RO          678    i.nrfx_uart_init    nrfx_uart.o
    0x00002d3c   0x00002d3c   0x00000124   Code   RO          679    i.nrfx_uart_rx      nrfx_uart.o
    0x00002e60   0x00002e60   0x0000008c   Code   RO          684    i.nrfx_uart_tx      nrfx_uart.o
    0x00002eec   0x00002eec   0x00000024   Code   RO          686    i.nrfx_uart_tx_in_progress  nrfx_uart.o
    0x00002f10   0x00002f10   0x00000014   Code   RO          927    i.nrfx_uarte_0_irq_handler  nrfx_uarte.o
    0x00002f24   0x00002f24   0x00000080   Code   RO          929    i.nrfx_uarte_init   nrfx_uarte.o
    0x00002fa4   0x00002fa4   0x00000138   Code   RO          930    i.nrfx_uarte_rx     nrfx_uarte.o
    0x000030dc   0x000030dc   0x000000a8   Code   RO          933    i.nrfx_uarte_tx     nrfx_uarte.o
    0x00003184   0x00003184   0x00000020   Code   RO          935    i.nrfx_uarte_tx_in_progress  nrfx_uarte.o
    0x000031a4   0x000031a4   0x000001d8   Code   RO         2594    i.on_radio_disabled_rx  nrf_esb.o
    0x0000337c   0x0000337c   0x00000050   Code   RO         2595    i.on_radio_disabled_rx_ack  nrf_esb.o
    0x000033cc   0x000033cc   0x000000a4   Code   RO         2596    i.on_radio_disabled_tx  nrf_esb.o
    0x00003470   0x00003470   0x00000040   Code   RO         2597    i.on_radio_disabled_tx_noack  nrf_esb.o
    0x000034b0   0x000034b0   0x00000170   Code   RO         2598    i.on_radio_disabled_tx_wait_for_ack  nrf_esb.o
    0x00003620   0x00003620   0x00000014   Code   RO         1166    i.pin_configured_set  nrfx_gpiote.o
    0x00003634   0x00003634   0x0000001c   Code   RO         1167    i.pin_in_use_by_gpiote  nrfx_gpiote.o
    0x00003650   0x00003650   0x00000018   Code   RO         1168    i.pin_in_use_by_port  nrfx_gpiote.o
    0x00003668   0x00003668   0x00000020   Code   RO         1169    i.pin_in_use_by_te  nrfx_gpiote.o
    0x00003688   0x00003688   0x0000000c   Code   RO         1170    i.pin_in_use_clear  nrfx_gpiote.o
    0x00003694   0x00003694   0x00000050   Code   RO         2599    i.ppi_init          nrf_esb.o
    0x000036e4   0x000036e4   0x00000018   Code   RO          601    i.prs_box_get       nrfx_prs.o
    0x000036fc   0x000036fc   0x0000001c   Code   RO         2600    i.reset_fifos       nrf_esb.o
    0x00003718   0x00003718   0x0000000c   Code   RO         2273    i.rtc1_compare0_set  app_timer.o
    0x00003724   0x00003724   0x0000000c   Code   RO         2274    i.rtc1_counter_get  app_timer.o
    0x00003730   0x00003730   0x00000018   Code   RO         2275    i.rtc1_init         app_timer.o
    0x00003748   0x00003748   0x0000003c   Code   RO         2276    i.rtc1_start        app_timer.o
    0x00003784   0x00003784   0x00000058   Code   RO         2277    i.rtc1_stop         app_timer.o
    0x000037dc   0x000037dc   0x0000003e   Code   RO          689    i.rx_byte           nrfx_uart.o
    0x0000381a   0x0000381a   0x0000001c   Code   RO          690    i.rx_done_event     nrfx_uart.o
    0x00003836   0x00003836   0x0000001c   Code   RO          938    i.rx_done_event     nrfx_uarte.o
    0x00003852   0x00003852   0x00000022   Code   RO          691    i.rx_enable         nrfx_uart.o
    0x00003874   0x00003874   0x000000e8   Code   RO         2601    i.rx_fifo_push_rfbuf  nrf_esb.o
    0x0000395c   0x0000395c   0x000001b4   Code   RO         2602    i.start_tx_transaction  nrf_esb.o
    0x00003b10   0x00003b10   0x00000020   Code   RO         2603    i.sys_timer_init    nrf_esb.o
    0x00003b30   0x00003b30   0x0000000a   Code   RO         2278    i.ticks_diff_get    app_timer.o
    0x00003b3a   0x00003b3a   0x0000000c   Code   RO         2279    i.timeout_handler_exec  app_timer.o
    0x00003b46   0x00003b46   0x00000002   PAD
    0x00003b48   0x00003b48   0x00000050   Code   RO         2280    i.timer_list_handler  app_timer.o
    0x00003b98   0x00003b98   0x0000000a   Code   RO         2281    i.timer_list_handler_sched  app_timer.o
    0x00003ba2   0x00003ba2   0x00000002   PAD
    0x00003ba4   0x00003ba4   0x00000068   Code   RO         2282    i.timer_list_insert  app_timer.o
    0x00003c0c   0x00003c0c   0x00000088   Code   RO         2283    i.timer_list_remove  app_timer.o
    0x00003c94   0x00003c94   0x00000058   Code   RO         2284    i.timer_start_op_schedule  app_timer.o
    0x00003cec   0x00003cec   0x00000098   Code   RO         2286    i.timer_timeouts_check  app_timer.o
    0x00003d84   0x00003d84   0x0000000a   Code   RO         2287    i.timer_timeouts_check_sched  app_timer.o
    0x00003d8e   0x00003d8e   0x00000002   PAD
    0x00003d90   0x00003d90   0x00000048   Code   RO          238    i.timers_init       host.o
    0x00003dd8   0x00003dd8   0x0000002c   Code   RO          239    i.timers_start      host.o
    0x00003e04   0x00003e04   0x00000036   Code   RO          692    i.tx_blocking       nrfx_uart.o
    0x00003e3a   0x00003e3a   0x00000026   Code   RO          693    i.tx_byte           nrfx_uart.o
    0x00003e60   0x00003e60   0x00000020   Code   RO          694    i.tx_done_event     nrfx_uart.o
    0x00003e80   0x00003e80   0x00000020   Code   RO          939    i.tx_done_event     nrfx_uarte.o
    0x00003ea0   0x00003ea0   0x00000194   Code   RO         2898    i.uart_event_handle  uartprocess.o
    0x00004034   0x00004034   0x000000d4   Code   RO         1630    i.uart_event_handler  app_uart_fifo.o
    0x00004108   0x00004108   0x00000038   Code   RO          547    i.uart_evt_handler  nrf_drv_uart.o
    0x00004140   0x00004140   0x0000014c   Code   RO          695    i.uart_irq_handler  nrfx_uart.o
    0x0000428c   0x0000428c   0x00000038   Code   RO          548    i.uarte_evt_handler  nrf_drv_uart.o
    0x000042c4   0x000042c4   0x00000104   Code   RO          940    i.uarte_irq_handler  nrfx_uarte.o
    0x000043c8   0x000043c8   0x00000054   Code   RO         2604    i.update_radio_addresses  nrf_esb.o
    0x0000441c   0x0000441c   0x0000004c   Code   RO         2605    i.update_radio_bitrate  nrf_esb.o
    0x00004468   0x00004468   0x00000050   Code   RO         2606    i.update_radio_crc  nrf_esb.o
    0x000044b8   0x000044b8   0x00000040   Code   RO         2607    i.update_radio_parameters  nrf_esb.o
    0x000044f8   0x000044f8   0x00000034   Code   RO         2608    i.update_radio_protocol  nrf_esb.o
    0x0000452c   0x0000452c   0x00000014   Code   RO         2609    i.update_radio_tx_power  nrf_esb.o
    0x00004540   0x00004540   0x00000030   Code   RO         2610    i.update_rf_payload_format_esb  nrf_esb.o
    0x00004570   0x00004570   0x0000002c   Code   RO         2611    i.update_rf_payload_format_esb_dpl  nrf_esb.o
    0x0000459c   0x0000459c   0x0000003c   Code   RO         2288    i.user_op_alloc     app_timer.o
    0x000045d8   0x000045d8   0x0000000c   Code   RO         2289    i.user_op_enque     app_timer.o
    0x000045e4   0x000045e4   0x00000003   Data   RO           10    .constdata          gpioprocess.o
    0x000045e7   0x000045e7   0x00000001   PAD
    0x000045e8   0x000045e8   0x00000004   Data   RO          241    .constdata          host.o
    0x000045ec   0x000045ec   0x0000002e   Data   RO          697    .constdata          nrfx_uart.o
    0x0000461a   0x0000461a   0x00000002   PAD
    0x0000461c   0x0000461c   0x00000030   Data   RO          942    .constdata          nrfx_uarte.o
    0x0000464c   0x0000464c   0x0000003e   Data   RO         1172    .constdata          nrfx_gpiote.o
    0x0000468a   0x0000468a   0x00000002   PAD
    0x0000468c   0x0000468c   0x00000020   Data   RO         1632    .constdata          app_uart_fifo.o
    0x000046ac   0x000046ac   0x00000004   PAD
    0x000046b0   0x000046b0   0x00000006   Data   RO         2291    .constdata          app_timer.o
    0x000046b6   0x000046b6   0x0000000a   PAD
    0x000046c0   0x000046c0   0x00000020   Data   RO         2900    .constdata          uartprocess.o
    0x000046e0   0x000046e0   0x00000020   Data   RO         3348    Region$$Table       anon$$obj.o


    Execution Region RW_IRAM1 (Exec base: 0x20000000, Load base: 0x00004700, Size: 0x00003f50, Max: 0x00010000, ABSOLUTE)

    Exec Addr    Load Addr    Size         Type   Attr      Idx    E Section Name        Object

    0x20000000   0x00004700   0x00000001   Data   RW           11    .data               gpioprocess.o
    0x20000001   0x00004701   0x00000003   PAD
    0x20000004   0x00004704   0x00000006   Data   RW          242    .data               host.o
    0x2000000a   0x0000470a   0x00000002   PAD
    0x2000000c   0x0000470c   0x00000034   Data   RW          354    .data               esbprocess.o
    0x20000040   0x00004740   0x00000009   Data   RW          549    .data               nrf_drv_uart.o
    0x20000049   0x00004749   0x00000003   PAD
    0x2000004c   0x0000474c   0x00000008   Data   RW          603    .data               nrfx_prs.o
    0x20000054   0x00004754   0x0000001b   Data   RW         1633    .data               app_uart_fifo.o
    0x2000006f   0x0000476f   0x00000001   PAD
    0x20000070   0x00004770   0x00000004   Data   RW         1716    .data               app_util_platform.o
    0x20000074   0x00004774   0x00000014   Data   RW         2292    .data               app_timer.o
    0x20000088   0x00004788   0x00000008   Data   RW         2483    .data               retarget.o
    0x20000090   0x00004790   0x00000048   Data   RW         2613    .data               nrf_esb.o
    0x200000d8   0x000047d8   0x00000001   Data   RW         2901    .data               uartprocess.o
    0x200000d9   0x000047d9   0x00000003   PAD
    0x200000dc   0x000047dc   0x00000004   Data   RW         2960    .data               system_nrf52.o
    0x200000e0        -       0x00000020   Zero   RW          240    .bss                host.o
    0x20000100        -       0x000001fe   Zero   RW          353    .bss                esbprocess.o
    0x200002fe   0x000047e0   0x00000002   PAD
    0x20000300        -       0x0000002c   Zero   RW          696    .bss                nrfx_uart.o
    0x2000032c        -       0x00000024   Zero   RW          941    .bss                nrfx_uarte.o
    0x20000350        -       0x0000004c   Zero   RW         1171    .bss                nrfx_gpiote.o
    0x2000039c        -       0x00000020   Zero   RW         1631    .bss                app_uart_fifo.o
    0x200003bc        -       0x0000010c   Zero   RW         2290    .bss                app_timer.o
    0x200004c8        -       0x00001278   Zero   RW         2612    .bss                nrf_esb.o
    0x20001740        -       0x00000810   Zero   RW         2899    .bss                uartprocess.o
    0x20001f50        -       0x00002000   Zero   RW         2937    STACK               arm_startup_nrf52.o



  Load Region LR$$.ARM.__AT_0x1000120C (Base: 0x1000120c, Size: 0x00000004, Max: 0x00000004, ABSOLUTE)

    Execution Region ER$$.ARM.__AT_0x1000120C (Exec base: 0x1000120c, Load base: 0x1000120c, Size: 0x00000004, Max: 0x00000004, ABSOLUTE, UNINIT)

    Exec Addr    Load Addr    Size         Type   Attr      Idx    E Section Name        Object

    0x1000120c   0x1000120c   0x00000004   Data   RO            9    .ARM.__AT_0x1000120C  gpioprocess.o


==============================================================================

Image component sizes


      Code (inc. data)   RO Data    RW Data    ZI Data      Debug   Object Name

        28          0          0          0          0       2473   app_error.o
        92         10          0          0          0      27461   app_error_weak.o
       170          0          0          0          0       6142   app_fifo.o
      1948        238          6         20        268      52202   app_timer.o
       770        108         32         27         32      21730   app_uart_fifo.o
        64         10          0          4          0       3446   app_util_platform.o
        36          8        512          0       8192        928   arm_startup_nrf52.o
         0          0          0          0          0      35216   boards.o
       472         80          0         52        510       5404   esbprocess.o
       446        108          7          1          0      61133   gpioprocess.o
       514         76          4          6         32      12157   host.o
       252         42          0          9          0      17872   nrf_drv_uart.o
      5080        858          0         72       4728      35065   nrf_esb.o
      1708        110         62          0         76      63065   nrfx_gpiote.o
       112         14          0          8          0       3713   nrfx_prs.o
      1680         46         46          0         44      63579   nrfx_uart.o
      1506         46         48          0         36      30265   nrfx_uarte.o
        16          0          0          8          0       2910   retarget.o
      1372        142          0          4          0       8567   system_nrf52.o
       496        138         32          1       2064      30399   uartprocess.o

    ----------------------------------------------------------------------
     16776       2034        800        224      15984     483727   Object Totals
         0          0         32          0          0          0   (incl. Generated)
        14          0         19         12          2          0   (incl. Padding)

    ----------------------------------------------------------------------

      Code (inc. data)   RO Data    RW Data    ZI Data      Debug   Library Member Name

         0          0          0          0          0          0   entry.o
         0          0          0          0          0          0   entry10a.o
         0          0          0          0          0          0   entry11a.o
         8          4          0          0          0          0   entry2.o
         4          0          0          0          0          0   entry5.o
         0          0          0          0          0          0   entry7b.o
         0          0          0          0          0          0   entry8b.o
         8          4          0          0          0          0   entry9a.o
        30          0          0          0          0          0   handlers.o
        36          8          0          0          0         68   init.o
        26          0          0          0          0         80   memcmp.o
        36          0          0          0          0         68   memcpya.o
        36          0          0          0          0        108   memseta.o
       372         14          0          0          0        184   printf1.o
        44          0          0          0          0         80   uidiv.o

    ----------------------------------------------------------------------
       604         30          0          0          0        588   Library Totals
         4          0          0          0          0          0   (incl. Padding)

    ----------------------------------------------------------------------

      Code (inc. data)   RO Data    RW Data    ZI Data      Debug   Library Name

       600         30          0          0          0        588   mc_w.l

    ----------------------------------------------------------------------
       604         30          0          0          0        588   Library Totals

    ----------------------------------------------------------------------

==============================================================================


      Code (inc. data)   RO Data    RW Data    ZI Data      Debug   

     17380       2064        800        224      15984     463811   Grand Totals
     17380       2064        800        224      15984     463811   ELF Image Totals
     17380       2064        800        224          0          0   ROM Totals

==============================================================================

    Total RO  Size (Code + RO Data)                18180 (  17.75kB)
    Total RW  Size (RW Data + ZI Data)             16208 (  15.83kB)
    Total ROM Size (Code + RO Data + RW Data)      18404 (  17.97kB)

==============================================================================

